:020000040000FA
:10000000F8580020D11B000045750000BD1B000002
:10001000BD1B0000BD1B0000BD1B00000000000058
:10002000000000000000000000000000491D00006A
:10003000BD1B000000000000151D0000BD1B0000DE
:10004000C51E0000C51E0000C51E0000C51E000024
:10005000C51E0000C51E0000C51E0000C51E000014
:10006000C51E0000C51E0000C51E0000C51E000004
:10007000C51E0000C51E0000C51E0000C51E0000F4
:10008000C51E0000C51E0000C51E0000C51E0000E4
:10009000C51E0000C51E0000C51E0000C51E0000D4
:1000A000C51E0000C51E0000C51E0000C51E0000C4
:1000B000C51E0000C51E0000C51E0000C51E0000B4
:1000C000C51E0000C51E0000C51E0000C51E0000A4
:1000D000C51E0000C51E0000C51E000053B94AB968
:1000E000002908BF00281CBF4FF0FF314FF0FF3040
:1000F00000F00CB8ADF1080C6DE904CE00F008F882
:10010000DDF804E0DDE9022304B07047704700BF6A
:100110002DE9F04786468C460846089E15467446EB
:100120001946002B40F0C2808542B2FA82F245D9CE
:100130004AB1C2F1200300FA02FC2EFA03F3954003
:1001400043EA0C0C94404FEA154EA8B2BCFBFEF8F3
:10015000230C0EFB18CC08FB00F943EA0C4399452D
:1001600028D9EB1808F1FF3704D2994502D9A8F134
:1001700002072B44A3EB0903A4B2B3FBFEFC0EFB66
:100180001C330CFB00F044EA0344A04214D92C19A0
:100190000CF1FF3304D2A04202D9ACF102032C448B
:1001A000241A43EA07401EB1D44000233460736030
:1001B000BDE8F0874746DDE76346F1E792BB431BA6
:1001C00001214FEA154EAFB2B3FBFEFC200C0EFB33
:1001D0001C330CFB07F840EA0343984562D9EB183F
:1001E0000CF1FF3004D2984502D9ACF102002B4447
:1001F000A3EB0803A4B2B3FBFEFC0EFB1C330CFB09
:1002000007F744EA0344A7424ED92C190CF1FF33F7
:1002100004D2A74202D9ACF102032C44E41B43EA06
:100220000040C0E7C2F1200320FA03F1954090405E
:100230002EFA03F303434FEA154EAFB2B1FBFEFCB7
:100240000EFB1C10190C0CFB07F841EA0041884515
:1002500004FA02F422D969180CF1FF3004D288455F
:1002600002D9ACF102002944A1EB08019BB2B1FB19
:10027000FEFC0EFB1C110CFB07F743EA01439F42F7
:100280000ED9EB180CF1FF3104D29F4202D9ACF128
:1002900002012B44DB1B41EA004192E76046E3E7A1
:1002A0006146F7E76046A3E76346B7E7834206D9AE
:1002B00016B9002108467BE7C6E900E0F9E7B3FA82
:1002C00083F78FB9834201D3724508D8BEEB02048D
:1002D00060EB030301209C461EB9002168E7384605
:1002E000FAE7C6E9004CF8E7C7F1200CBB4022FA58
:1002F0000CF41C432EFA0CF120FA0CF3B840014325
:100300004FEA14490EFA07F5B3FBF9F81FFA84FE19
:1003100009FB18300B0C08FB0EFA43EA00439A4520
:1003200002FA07F240D9E31808F1FF3004D29A45E7
:1003300002D9A8F102002344A3EB0A0389B2B3FB5C
:10034000F9F809FB183308FB0EFE41EA03418E451C
:100350002CD9611808F1FF3304D28E4502D9A8F1D7
:100360000203214443EA0040A0FB0298A1EB0E01E6
:100370004145CE46434602D306D14D4504D2B9EBA2
:10038000020E68EB04030138002EA6D0B5EB0E0276
:1003900061EB030101FA0CFC22FA07F34CEA0303B8
:1003A000F940C6E9003198E74046C5E74346D9E73A
:1003B0007FB5284B284AC3F800262848C3F80426EE
:1003C0004921C3F80826C3F80C26C3F81026C3F841
:1003D0001426C3F81826C3F81C2607F02FF800F0DF
:1003E0006BF801A800F018FD1D4B1B68834204D078
:1003F0001C48452107F022F8FEE7039A1A484921D4
:1004000007F01CF81948492107F018F869469DF8CB
:10041000080000F02FF8009B039C1C44019B1D89E1
:1004200003F024FC661900F091FD00F053FD00F08C
:100430007BFD635983F30888002383F31488BFF39B
:100440006F8FBFF36F8F736898470948452106F097
:10045000F5FFFEE7000001403546526E8A9C000021
:1004600088080020A39C0000C69C0000F59C0000AA
:100470001A9D000008B5024638B105480023452101
:1004800006F0DCFF6FF0150008BD0860FCE700BF58
:100490003D9D000021B1012906D06FF01500704785
:1004A000044B53F830007047024B03EBC00358680D
:1004B000704700BF9898000002484FF4C05104F004
:1004C0002BB900BFB21600202DE9F04FF9B0DDE9DD
:1004D000848ADFF8F891869CD9F8006038A817461E
:1004E0001D4608F084FC002138A804F04BFAB8F14E
:1004F000000F07D0BAF1000F04DD5246414638A87C
:1005000008F07EFC3B897A89D7F80CB013449B44F1
:100510004FF00008C34564D80DA938A808F0AFFC17
:1005200038A808F068FC24B120220DA9204607F065
:100530004EF8002300932A464FF6FF73394607A86A
:1005400006F041FD804600285BD128460C9C06F051
:10055000E9FD844255D8DFF878B1DFF878A14FF093
:10056000FF340DF1160305AA06A907A806F079FDC8
:10057000002846DB40F0A280069907A806F0BDFDE2
:1005800050B9BDF81600544A4FF6FF7132F8023BDD
:100590008B4236D09842F9D1BDF81670102F3AD060
:1005A000202F6DD0012FDCD1BDF81430202B28D89E
:1005B000069938AA284606F04FFF044608BB9DF866
:1005C00014300293202B09D8DAF80030434F0393FC
:1005D000039B9C421DA836DB08F00DFC4FF0FF3456
:1005E000BFE7839B829AABEB080A9A4528BF9A46DD
:1005F00053464146284606F02FFF28B138A808F098
:10060000FAFBD9F800605CE08299524638A808F0FD
:10061000F7FBD0447EE7BDF81470202FF1D1069986
:100620003B4638AA284606F017FF0028E9D13A468B
:1006300038A90DA806F06FFDDBF800308342E0D149
:100640004FF001088DE708F0D2FB00211DA804F04F
:1006500099F97A6857F8081B12681DA808F0D0FBB2
:1006600015A91DA808F00BFC029A38A915A806F0D8
:100670009EFF18B91DA808F0BEFB72E70134A7E77A
:10068000631C3FF46EAFDAF80030A342A6DDBDF87C
:100690001430B3F5807FB4D1069938AA284606F005
:1006A000DBFE0028ADD1E4B2BDF81430009438AAC6
:1006B00039460DA800F014F806468FE7B8F1000F90
:1006C0009FD0304679B0BDE8F08F00BFBC04002059
:1006D00088080020A09800005C9C0000A4980000FE
:1006E0002DE9F04FDFF8E4A1ADF5417D07462AA8DA
:1006F0009DF828B3DAF800501E468946904608F067
:100700002FFB092201212AA804F0B8F8704B53F8F6
:100710003B40059403EBCB0380AA5B681B681C4439
:100720002146302305A807F005FC002840F0C580CD
:10073000059B809A13449C4240F0BF802CAA21461E
:1007400005A807F00BFC002840F0B7800DF1B80BAE
:100750005A46214605A807F001FC0390002840F006
:10076000AC802CA807F0A8FF059A2B90944240F08B
:10077000A480039BCDF804B000931A462CA92AA8A4
:1007800008F0ABFA002840F098802AA804F08CF812
:10079000002840F092802CA807F08EFF2B902AA80A
:1007A00008F0E8FA864240F08880B6F5807FDAF8F3
:1007B000005040F08280B9F1200F7ED180AA4146DE
:1007C0002AA804F097F80446002876D19DF8FF3255
:1007D000BC2B72D106900DF59079DF260FA808F09A
:1007E00006FB00210FA804F0CDF820220DF2DF2136
:1007F0000FA808F005FB042206A90FA808F000FBCB
:1008000007A90FA808F03BFB202E9DF81B30B0462F
:10081000A8BF4FF0200801334846424607A9A6EB7F
:1008200008068DF81B3006F0D2FE002EC144D5DC40
:100830000FA808F0E0FA48AB80AA184600219C46B1
:10084000067812F801EB013186EA0E06DF2900F87E
:10085000016BF5D11A7802F07F021A7013F8016B60
:100860005EBB0134BE2CF9D19CF8BE30012B24D1E3
:100870000FA808F0BCFA31460FA804F083F8154918
:1008800008220FA808F0BCFA394620220FA808F069
:10089000B7FA20220DF2DF110FA808F0B1FA07A96C
:1008A0000FA808F0ECFA0FA808F0A5FA20220DF224
:1008B000DF2107A806F02FFC05462AA808F05CFAFD
:1008C00028460DF5417DBDE8F08F00BFBC04002037
:1008D000A4980000639D00002DE9F0413F4F88B0CF
:1008E000064600200D463C68FFF7D4FD06A9C0B2BD
:1008F00000F0B2FEB8B92946FFF7CCFD2C2407A9B9
:10090000C0B204FB056400F0A7FE80B12C226A434C
:10091000B318DDF818801869C10618D5304B1C686B
:10092000069806F098FD204608B0BDE8F0810798CB
:1009300006F0DBFD8046079806F08DFD631EE21C85
:1009400013F8011F4145E1D19A42F9D1E6E7B158C8
:10095000244A254E914225D1DA681989891821D275
:100960005A8952181ED2D8F808309A421AD240F644
:100970000C63184216D14FF0FF33079307A807F016
:100980005AF9F8B14FF4807300210193174B00938B
:100990002246CDE90311029143460846FFF794FD34
:1009A000044617E03C683368A342B9D09DB106986D
:1009B0000021826806F07AFD0D4A0E48452106F0B6
:1009C0003DFDABE7079B802BDCD10B48492106F0AE
:1009D00035FD3468E7E7094AEFE700BFBC040020B3
:1009E000B80400203DB8F39688080020B22E0020FD
:1009F000739D0000A49D00007D9D00006B9D000084
:100A00002DE9F84FDFF870B01C4C1D4D884691461B
:100A10009A4600260B9B9E4201D300200FE00B9BC1
:100A2000154A9F1BB7F5806F28BF4FF480673B4680
:100A300006EB0A01404606F00FFD10B10120BDE8AB
:100A4000F88F0A993B465A467118484606F019FD38
:100A50000028F3D1C4F800563E44C4F80456C4F844
:100A60000856C4F80C56C4F81056C4F81456C4F806
:100A70001856C4F81C56CDE78C0800200000014031
:100A80003546526E2DE9F04FB64B43620F4603F5E3
:100A90008063002103658BB004460846FFF7FAFC2B
:100AA00004F120010546C0B200F0D6FD0346E8B9C6
:100AB0000121FFF7EFFC04F14C010546C0B200F044
:100AC000CBFD0346E0B9204606F051FB0546C8B908
:100AD00000221146204606F034FB054650B3A248DA
:100AE0000022572106F0AAFC01235BE00022CDE999
:100AF00000239E4800232A46452106F09FFCFEE77E
:100B00000122F4E79A488022572106F097FC01233E
:100B10009D4284F85830DBD194F858308DF81F305E
:100B2000042B42D8012B42D800F0DF80FF2384F849
:100B30005830DAE0204600F07FF90028D4D006A82B
:100B400006F036FB06F03DFB014620B906AA20461A
:100B500006F0F7FAC8E79DF81F60012E17D1284666
:100B600003F012F9831E022B05460DD831462046AC
:100B7000FFF7B2FE7F4B1B68984205D07E4B1D6885
:100B8000A84214BF0525012584F85850C4E7012167
:100B90002046FFF7A1FE774B1B6898420CBF9DF8DB
:100BA0001F30052384F85830B6E7052BBCE706F064
:100BB000BBFA804606F0B8FA012181460020FFF713
:100BC00069FC04A9C0B200F047FD002800F096803F
:100BD0000026049806F03FFC00226848492106F0F0
:100BE0002DFC6748492106F029FC236A04A91878DE
:100BF00000F032FD05A9062000F02EFD0025D4F8F6
:100C000028B0AA46D34512D0636A049803EBCA03FE
:100C100029465A68039206F049FC039A1544B542E6
:100C2000C0F09C80E56DB6FBF5F605FB0655E06D62
:100C300006F073FAA26A636A013A196803EBC20309
:100C400000225E68324490429C46A3F10803F8D823
:100C5000DCF800300498591A06F028FC06F064FA13
:100C60004921A0EB0902474806F0E8FB06F05CFAD0
:100C70002B46002249210646434806F0DFFB0023AD
:100C8000DDE90421019500932046FFF7B9FE20BB62
:100C9000049803F003F80546F8B906F045FA49212F
:100CA000821B3A4806F0CAFB236D05985A6829460C
:100CB00006F0FCFBD4E91423013B02EBC30052F81D
:100CC0003310136842680598C91A06F0EFFB0498C0
:100CD00006F0C1FB059806F0BEFB06F025FA492197
:100CE000A0EB08022A4806F0A9FB94F85830FF2B25
:100CF00052D12848452106F0A1FBFEE7A36BA58E43
:100D000004981D4405AA0423294606F0A5FB0028E3
:100D10007FF45EAFBDF81420E68E049846F6081303
:100D20009A4218D1BDF816309E427FF451AF042389
:100D300005AA711906F090FB00287FF449AFBDF8B1
:100D4000142046F607139A427FF442AFBDF81630DE
:100D50001E442E443DE7002EF1D039E70AF1010A86
:100D600050E700BF8C0C00205B9E0000CC9D000073
:100D7000199E000088080020B8040020879E00000B
:100D8000BC9E0000DA9E0000F29E00003C9F000026
:100D9000539F00006C9F00000022012B1B4D059209
:100DA00014D01146204606F0CCF978B12D681022F7
:100DB000002106A806F016FCE06C06F04CFB206A49
:100DC00006F049FB28460BB0BDE8F08F0021204615
:100DD000FFF782FD0E4E33689842E7D12B689842A8
:100DE000E4D00C4B1B689842E0D0059B013305937F
:100DF000059B012B00D0FEE7206A06F0E2F838716F
:100E0000236A5B683C603568BB60D0E7BC040020A7
:100E100088080020B804002038B5064D044660223A
:100E20000021284606F0DEFB21462846FFF72AFE71
:100E300038BD00BF8C140020F8B5D0F828C0466D2E
:100E4000BCF1800F01D8802E36D91F48572106F0FB
:100E5000F5FA0020F8BDAC4216D1476A07EBC2078D
:100E600001327F683C44076D07EBC30701337F689D
:100E70003D449445EFD89E42EDD8944501D19E4221
:100E800020D012485721E2E70CD2476A07EBC2078D
:100E900002297F683C4402D10D485721D7E701322F
:100EA0000121E6E7076D07EBC30701297F683D4491
:100EB000F2D001330221DCE700210B460A460D4641
:100EC0000C46D6E70120C5E7789F0000DE9F0000B2
:100ED000A79F0000BFF36F8F72B6124B4FF0FF3227
:100EE000C3F88020C3F88420C3F88820C3F88C207E
:100EF000C3F89020C3F89420C3F89820C3F89C202E
:100F0000C3F88021C3F88421C3F88821C3F88C2159
:100F1000C3F89021C3F89421C3F89821C3F89C2109
:100F2000704700BF00E100E00749D1F8902000239E
:100F3000C2F307221846934200DB7047C1F898308D
:100F4000C1F8A0000133F6E700ED00E01A4B70B5E0
:100F50004FF0FF3401265E60C3F84843C3F80843EE
:100F600003F5C043154D5E60C3F84843C3F808431A
:100F700003F5983302205E60C3F84843C3F8084382
:100F8000C5F8084300F0FEFE00236E60C5F84C3142
:100F9000D5F84C21C5F81031D5F81021C5F84431E9
:100FA000D5F84421C5F80035054BC3F808454FF086
:100FB0008043C3F8084370BD00B0004000200040EB
:100FC00000F00140014B1B68184700BFC00400201F
:100FD000014B1860704700BFC004002007B50B46E6
:100FE000002102460091034800F006F803B05DF8C6
:100FF00004FB00BFC50F00002DE9F04F8DB01D466A
:10100000531E8246019103934FF00009039B5878C9
:10101000252803F1010419D11E4600204FF0FF38A6
:10102000023603460290444631780396392954D853
:101030001F2914D8002900F0EE8101992520D047FE
:1010400001993078D04709F10209DFE7002800F064
:10105000E2810199D04709F101090394D6E7A1F192
:101060002002192AE9D801A757F822F0D51000006C
:101070003B1000003B100000D51000003B100000AA
:10108000551100003B1000003B1000003B10000019
:101090003B100000A1110000D51000003B10000023
:1010A000B5110000611100003B1000006F1100003D
:1010B0008F1100008F1100008F1100008F110000B0
:1010C0008F1100008F1100008F1100008F110000A0
:1010D0008F11000008460136A6E7582900F0EB8082
:1010E000A1F16302D7B2172FA7D8172AA5D801A755
:1010F00057F822F05D130000DB1100003B100000E8
:101100003B1000003B100000BB110000DB11000091
:101110003B1000003B100000BB1100003B10000022
:101120003B1000003B100000911200003B1000003B
:101130003B100000311300003B100000DB110000E9
:101140003B1000003B100000911200003B1000001B
:10115000BB11000001992520D04709F1010955E78D
:10116000029A02F0FE0202924FF00008B3E7002C50
:101170000DDAB8F1000F0DDA029A002A00F043816F
:1011800024EAE4740A2202FB0414303CA3E7B8F119
:10119000000FF5DB0A2202FB0812A2F130089AE7E1
:1011A000B8F1000F55F8042B80F22F81002A80F24D
:1011B0002E815442022202928DE7682903D1682BC6
:1011C00006D1482387E76C2902D16C2B00F02181DE
:1011D000002B7FF432AF0B467DE77A2B06D17529C1
:1011E00055F8046B14D14FF0000B0CE06C2BF6D0CB
:1011F0004C2BF4D1073525F007037529D3E9006B93
:1012000003F1080506D120283BD1854F013C09E0B8
:101210004FEAE67BBBF1000FF5DA7642814F6BEBCC
:101220004B0B013C0DF12D03059300230493304635
:1012300059460A220023FEF751FF059B303203F87E
:10124000012DB4460593049B5A46BCF10A0F8B4608
:1012500072F1000203F1FF3106460491E7D2C3F1B7
:10126000010B30330DEB0306B8F1000FA6F10406B5
:101270006DDA029BD9077DD4A8EB0B03A4EB0B041A
:1012800013E02B280ABF684F684F04F1FF34C9E709
:1012900070290FD155F8042B0023FAB9634F644E1F
:1012A000053C6FF004034FF0050B029A920770D4CF
:1012B000A04666E078216C2B03D155F8042B00235F
:1012C00008E04C2BF9D1073525F007031D465B6874
:1012D00055F8082B232825D1880621D5554F023CE7
:1012E00001F06001A1F1390B0DF12D0E002602F085
:1012F0000F01092988BF594430310EF8011D102A09
:101300004FEA121141EA03714FEA131C73F1000313
:1013100006F1FF3008D2C6F1010B06F13003A1E758
:10132000454FDCE7414FDBE706460A466346DEE70A
:1013300055F8046B304606F033F9B8F1000F8346D8
:1013400002DB4045A8BFC346384F4FF00008A8EB6A
:101350000B03002B92DDA4EB0804A6E755F8043B31
:101360008DF81830314F013C4FF0FF334FF0010B37
:1013700006AE9AE7A046EAE7029301992020D047FB
:10138000029BB8F10108F7D524EAE472013C9144CC
:10139000A41AB84606E0049302920199D047029A33
:1013A000049B9046424612F8010B0028F3D11A46DE
:1013B000013A15D5002BACBFC7EB03077F425B4654
:1013C000013B15D5BBF1000FA8BF5F444F44264633
:1013D000013E14D5002CA8BF3F1907EB080915E6FC
:1013E0000493029201993020D047049B029ADFE7D0
:1013F0000293019916F8010BD047029BE0E701998F
:101400002020D047E4E70122D5E6904663E6144663
:1014100061E64C235FE648460DB0BDE8F08F00BFA3
:1014200057A500002BA100002DA1000035A700004A
:1014300035A100002FA1000032A100002DE9F047E6
:10144000058B04462807904611D4022905F00705AC
:1014500040F0CC80204605F0F5FE78B10138218BB4
:10146000042811D8DFE800F0C2106D85950001292D
:101470000CBF45F0100545F02005258388F3118841
:10148000BFF36F8FBDE8F08701F0070AAA4500F0AF
:10149000A5800027B9463E46A368002B00F0BC801B
:1014A00041F00801218388F31188BFF36F8FA16891
:1014B000002900F0BA800D68002900F0B680D1F84C
:1014C0000480334652462046C047002D76D02B6814
:1014D00029461D46F0E701F007035A1F012A1BD8D1
:1014E000002221F00701062B276889B2C4E90022F7
:1014F00009D13B4603E0628B013262831B68002BFB
:10150000F9D141F002012183204605F09BFE00281D
:101510007AD041F0200176E0042B0AD121F00701B6
:1015200089B22183204605F08DFE10B141F02001E3
:101530002183218B01F0070AAA454FD00027B94625
:10154000AAE7236921F0070141F00601062DD3F82F
:10155000009021832DD1B9F1000F3FD041F0080157
:10156000218388F31188BFF36F8F3A492046C8471B
:1015700029E021F00701236941F0040189B2042D1B
:10158000D3F804902183E6D000273E464FF0040AAA
:1015900082E721F00701236941F0050189B2052D99
:1015A000D3F808902183D6D000273E464FF0050A95
:1015B00072E700273E464FF0060A6DE72B4687E7A5
:1015C000B9F1000FD1D1EFF31188202383F31288F2
:1015D000BFF36F8F238B23F008032383258BEA0649
:1015E0002ED525F01003238305F007056669218BAE
:1015F000002EBFF670AF00232768C4E9003321F046
:10160000070141F001012183218B01F0070AAA455E
:101610004FF000097FF440AF002F9CD041F008014B
:10162000218388F31188BFF36F8F002FC8D03D68E6
:10163000394633465246204605F030FE2F46F4E741
:10164000AB067FF51BAF25F02003238305F00705CC
:1016500000E700BFC972000070B5114B1C680D4651
:10166000DCB1104B196800238B4202DB6FF00100E4
:1016700070BD224612F8106B864202D00133144628
:10168000F2E7E06810B96FF01200F1E707F0BCFD77
:101690000028F8D02C600020EAE76FF00C00E7E7A4
:1016A000C4040020B098000070B588B005460C4610
:1016B000C0B269461646FFF7CFFF00281BDB009833
:1016C000C8B143680293836822680195CDE9033667
:1016D0000023CDE906230593C56805F0BCFE6DB176
:1016E0002846084901AA06F012FA079808B9059B8E
:1016F000236008B070BD6FF01500FAE76FF01200BC
:10170000F7E700BFF974000008B5054805F083FD50
:10171000044805F080FDBDE80840034805F07BBDA6
:1017200041A1000072A10000A5A1000037B5054647
:101730000C46C9B18B680093D1E9002312484521BA
:1017400005F07CFE63690093D4E903230F4845212B
:1017500005F074FEE2690E48452105F06FFEA269AE
:101760000C48452105F06AFE012D06D1EFF30582F4
:101770000948103A452105F061FE2146284603B08C
:10178000BDE8304004F0A8BAD3A1000007A20000D1
:101790003BA200004FA2000082A2000030BFFFF772
:1017A000FDBF00BF074A936893F90E10002907DBBD
:1017B000526993421FBF044A536843F080535360F9
:1017C000704700BF7816002000ED00E010B5204CF7
:1017D0002048452105F032FEA36A990136D51E48FE
:1017E000452105F02BFE1E20A36ADA0104D51B4813
:1017F000452105F023FE1F20154CA36A1B0304D5C9
:101800001748452105F01AFE2120A36A590304D583
:101810001448452105F012FE22200D4CA36A9A03BC
:1018200004D51148452105F009FE2320A36ADB03F6
:1018300004D50E48452105F001FE2420044A936A90
:101840006FEA03436FEA1343936210BD1D20CBE799
:1018500000ED00E09AA20000B7A20000CFA20000B5
:10186000EEA2000011A300003BA300005AA3000059
:1018700070B5284C06460D462748452105F0DEFD8B
:10188000A36AD9043BD52548452105F0D7FD17208B
:10189000A36A1A0504D52248452105F0CFFD18207A
:1018A0001C4CA36A9B0511D51E48452105F0C6FDB9
:1018B000A26BA36A180408D51B48452105F0BEFD9C
:1018C0001EB1A36A23F40043A3621920114CA36A3A
:1018D000590504D51548452105F0B0FD1A20A36A25
:1018E000DA050ED51248452105F0A8FD1B20094A4E
:1018F000936A43F47F43936200232B7070BD1620DC
:10190000C6E7A36A9B04F2D50A48452105F096FD77
:101910001C20ECE700ED00E08AA30000A5A3000076
:10192000BBA30000D3A30000F1A300000BA40000A0
:101930002BA4000048A4000070B5294C06460D46B3
:101940002848452105F07AFDA36AD80646D52648E1
:10195000452105F073FD1120A36A190704D523481A
:10196000452105F06BFD12201D4CA36A9A0711D585
:101970001F48452105F062FD626BA36A1B0608D56E
:101980001C48452105F05AFD1EB1A36A23F08003CF
:10199000A3621320124CA36ADE0704D51648452122
:1019A00005F04CFD1420A36A9C0604D5134845217C
:1019B00005F044FD15200A4B9A6AD10658BF9A6A71
:1019C0009A6A920642BF5A6A22F400525A629A6A8E
:1019D00042F0FF029A6200232B7070BD1020BBE71B
:1019E00000ED00E07CA4000097A40000BBA3000071
:1019F000CFA40000ECA4000007A5000048A400004C
:101A00002DE9F0415C4B5F688AB00546C7F30804D6
:101A1000002686F31188BFF36F8F02F07F43B3F186
:101A20007F4F07D102F00C03082B14D153484521F6
:101A300005F004FD002635464FF00008E31E8DF842
:101A40000780092B00F28680DFE803F00A797D75B4
:101A500084848484848110074CBF0D460126EBE703
:101A60004748454C452105F0E9FC8DF80780E36ABD
:101A70009A0705D54348452105F0E0FC002432E0F3
:101A8000E36A002B02DA40484521F5E7E36A5B0090
:101A9000F4D53E48452105F0D1FC6369AA6943F4B9
:101AA00080736361BFF34F8FBFF36F8F636932F849
:101AB000022C23F480736361BFF34F8FBFF36F8FEA
:101AC0004DF602739A4208D0A36ADBB22BB30DF134
:101AD00007010120FFF730FF2FE02A682C4845213D
:101AE00005F0ACFC2C689DF807309BB920222946F4
:101AF00002A805F06CFD099B002E38D0C3F3080244
:101B000022B96FEA53236FEA4323099302A92046BF
:101B1000FFF70CFE0AB0BDE8F081A36A13F47F4F13
:101B200005D00DF107010120FFF7A2FE05E0A36A31
:101B3000B3F5803FA2D3FFF749FE0446D3E70DF18A
:101B400007010020C6E70DF107010020ECE711486E
:101B5000452191E71049114A114817F4F87F08BF51
:101B60000A46A4F11003452105F068FC86E723F43A
:101B7000FF7323F00103C8E700ED00E059A5000062
:101B800089A50000A5A50000CBA50000DEA50000EA
:101B900002A6000023A600002BA5000040A500001F
:101BA0004CA60000044B5A6942F010025A615A696F
:101BB00022F008025A61704700ED00E0EFF3088060
:101BC000EFF3098101B57246FFF71AFF01BD00BFAF
:101BD000002080F31488BFF36F8F02F0EBFF00202A
:101BE0000D490860BFF34F8F0C4880F3088800F060
:101BF00019F8202080F3118809484FF4006140183B
:101C000080F30988EFF314800221084380F31488DD
:101C1000BFF36F8F00F0F0F894ED00E0F85800206B
:101C2000B82F002072B6002383F31388144B4FF0B3
:101C3000FF32C3F88020C3F88420C3F88820C3F89B
:101C40008C20C3F89020C3F89420C3F89820C3F8E0
:101C50009C20C3F88021C3F88421C3F88821C3F8ED
:101C60008C21C3F89021C3F89421C3F89821C3F8BC
:101C70009C2162B6BFF34F8FBFF36F8F704700BFD9
:101C800000E100E0084B9B6883420BD1EFF3058332
:101C900043B1064B5A6842F080525A605A6A22F4A5
:101CA00000425A6207F012BC7816002000ED00E0F6
:101CB000094A93686FF00A01D966084998664B682B
:101CC00043F080534B60002383F31188BFF36F8F81
:101CD0009368D86E704700BF7816002000ED00E0D2
:101CE000EFF31183202383F31288BFF36F8F074A2A
:101CF00053699360064A4FF00061516000219A6E6B
:101D0000996682F31188BFF36F8F704778160020B1
:101D100000ED00E00B498A684FF030001044EFF30B
:101D2000098C80E8F01F74467046FFF7D9FFA6467D
:101D300004498A6802F1300090E8F01F8CF30988AA
:101D400070470000781600201EF0040F0CBFEFF360
:101D50000880EFF30980816911F8021C0229FFD085
:101D600001B505F0EBFB01BD40B2002807DB044ADA
:101D70004109012300F01F00834042F821307047E1
:101D800000E100E040B200280CDB4309064900F006
:101D90001F0020330122824041F82320BFF34F8FE0
:101DA000BFF36F8F704700BF00E100E0054B4209B1
:101DB00000F01F0053F82220012303FA00F0104026
:101DC000704700BF00E100E040B20028A8BF00F16A
:101DD000604001F10101B8BF064B4FEA4111ACBFB1
:101DE00000F5614000F00F00C9B2B4BF195480F88B
:101DF0000013704714ED00E00B4A08B50B4B22F0BE
:101E00007F029A60BFF34F8FBFF36F8FD3F88820A4
:101E100022F47002C3F8882004F024F804F0B2FE23
:101E200000F044F804F05EF80000000000ED00E06F
:101E300042F8203C009B42F81C3C0A49019B42F8B6
:101E4000183C029B42F8143C21F001014FF08073D2
:101E500042F8043C42F8081C0023203A02658366DD
:101E6000704700BF317200000A4B00B50E46986003
:101E700015462C4686F309884FF00000064B98471C
:101E800020464FF000014FF000024FF00003034CDA
:101E9000204700BF781600205B75000031720000FB
:101EA000014B10221A61704700ED00E00448002346
:101EB0002021C2180133272B82F80013F9D1704773
:101EC00000E100E008B5EFF30583064A103B02EBA2
:101ED000C30152F8330049688847BDE80840FFF75E
:101EE00061BC00BFE4960000014B1860704700BF62
:101EF000C8040020024B0122C3F84025002070478F
:101F000000E0014020B1034B800143F0010318477A
:101F1000704700BF90980000084B70B5C31A0D467B
:101F200007499B10044659430648402205F06FFBC1
:101F30002B4601462046BDE870401847001500209A
:101F4000B76DDBB64496000073B50C4C0C4A4023C9
:101F5000041B00930D460B460A49A4106143064634
:101F6000094805F07FFB011E05DA30462B4602B01A
:101F7000BDE87040184702B070BD00BF00150020DA
:101F8000CD760000B76DDBB644960000002270B538
:101F9000012104461046FFF717FF114802F0F2FF37
:101FA000104B984218D1206900F0DEF902F0FCFFD6
:101FB00026690D49304605F094F900280BDB012510
:101FC00035642469084904F11C0005F08AF90028E9
:101FD00001DBE564002070BD6FF00400FBE700BF8B
:101FE000C52000000000AD0B349900001FB5002291
:101FF0000123CDE90223094ACDF800D06B46CDF884
:1020000004D005F05CFB002805DB4FF48042002380
:10201000684604F0A7F805B05DF804FBDF76000021
:1020200010B5074C23782BB94FF4A57007F0E7F8EB
:1020300001232370BDE81040002002F0C7BF00BF9D
:10204000B22F002010B5EFF31184202383F3128800
:10205000BFF36F8F074A136823F00201DB0711609B
:1020600002D4012006F0CCFF84F31188BFF36F8FF8
:1020700010BD00BF5015002030B4104B0C2202FBE5
:10208000003301460020D3E90E529863EFF311802C
:10209000202484F31288BFF36F8F1C6C04F0C004FB
:1020A00044F002041C6480F31188BFF36F8F1DB1EC
:1020B0002B46034830BC184730BC70470015002041
:1020C00044960000012810B504460AD004280CD01C
:1020D00078B9084B1B6C5B070BD1BDE81040FFF7CC
:1020E000CBBF00F04FF92046F7E7BDE8104000F005
:1020F00057B910BD0015002010B4EFF31182202352
:1021000083F31288BFF36F8F1748016841F0020410
:102110000460C80707D482F31188BFF36F8F0120D2
:1021200010BC02F053BF4FF08041D1F80C04D1F83D
:102130000C14C907EFD5EFF3118083F31288BFF3B6
:102140006F8F0A490B6C03F0C00343F002030B646A
:1021500080F31188BFF36F8F82F31188BFF36F8F05
:10216000002010BCFFF788BF50150020001500208C
:10217000024AC3B21C2003FB002070470015002058
:10218000F8B52849BFF35B8F0646012251E8003FAE
:1021900041E800200028F9D1BFF35B8F33B9224911
:1021A00022484B60CB608A6005F0AEF8731E012BAD
:1021B0001DD807F0B4F80446D0B91D4B1B78BBB14D
:1021C0004FF080430222C3F8082305464FF08047B2
:1021D000D7F81824D7F81834D20312D59B0701D0AA
:1021E000012E0ED1BCB185F31188BFF36F8FF8BDFE
:1021F000EFF31185202383F31288BFF36F8F01243F
:10220000E4E71CB1284605F0BCF9E1E700212120F4
:1022100004F0FCFBDCE74FF080430222C3F8042308
:10222000E5E700BFFC140020EC1400201C15002082
:10223000B62F00200D4BBFF35B8F012253E8001F28
:10224000002903D143E800200028F7D1BFF35B8FBA
:102250000AD107490023CB60064B4B6003238B60F8
:10226000054B186805F050B8704700BF7015002086
:10227000581500203D2300005415002007B500220A
:102280000023CDE9002308484FF40032002304F076
:1022900043FE064B186805F08EF8054B00221A60C5
:1022A00003B05DF804FB00BF300600205415002089
:1022B00070150020F7B51C4E1C4CB7681C4DFB6810
:1022C0003C213046984740B1002323702B8002F018
:1022D000EFFE0123237003B0F0BD0C213B696A4679
:1022E000304698470028EFD1124A019B93FBF2F346
:1022F000009A217803EB82031BB2B5F90020002974
:10230000E4D09A1A002AB8BF524212B2012ADDDC88
:10231000094A1368013901332170136003B0BDE825
:10232000F040FFF7ABBF00BFD0960000B32F0020F6
:10233000B016002090D003006815002008B50748AB
:1023400006F062FF28B902F0B3FE054B01221A70B5
:1023500008BDBDE80840034804F03CB8D096000032
:10236000B32F0020CC040020034B044A1860002344
:102370001360034A13607047541500206C15002049
:1023800068150020024B00221A70FFF753BF00BFF0
:10239000B32F0020014807F0F8B800BF3006002036
:1023A000024A136801331360FFF768BF6C15002001
:1023B00008B5074806F028FF38B10648FFF794FD36
:1023C0000448FEF705FE002008BD6FF01200FBE791
:1023D0006C960000D92300000A2838B5074D044642
:1023E00004D1AB680D215B6828469847AB68034869
:1023F0005B68E1B29847204638BD00BF6C9600008C
:1024000000487047AC9900002DE9F04F91B00446A8
:1024100004AF00694FF0FF32012106F03FFF66680C
:10242000306806F0F1FEA8B1F06878B9206905F0CF
:102430006BF9204605F00BFB021E12DA76484521A7
:1024400004F0FCFF206905F05DF903E006F0DCFE16
:102450000028EBD16FF0120528463437BD46BDE8A1
:10246000F08F204605F0BFF9051E27DDE8071BD4D5
:10247000206905F047F9206905F046F90323019327
:1024800007F11403009300231A469F21204605F00C
:1024900041F98046206905F035F9B8F1000F18D0F0
:1024A0005E484246452111E05D48572104F0C6FFD1
:1024B00000220023204605F0A7F90546206905F013
:1024C00021F9002DD7DA57482A46452104F0B6FFF6
:1024D000C0E7337EA3B3206905F016F9204605F066
:1024E00082F9051E27DD337E25EA03053D76434646
:1024F000CDE9008880220621204605F00BF905462B
:1025000030B1206905F0FEF847482A464521DDE74D
:10251000012107F118030093019103468022204610
:1025200005F0F8F805460028EBD1002200232046EC
:1025300005F06AF90546206905F0E4F8002DE3D1BD
:102540002069C7F80CD005F0DFF818230193FB18B9
:102550000093052200235A21204605F0DBF80646A9
:10256000206905F0CFF846B130483246452104F0E5
:1025700065FF2E4832464521A8E7BA692C4B9A429E
:1025800006D02C48452104F059FF6FF01506F0E7FE
:10259000BA7F7B7F284801320292FA7F01923A7F0C
:1025A00000922268492104F049FFBB7F012B9CBFA8
:1025B0000133DBB207F1200A94BFDB001023534440
:1025C000BB605546BB68AB423CD12569D7F80CD0FF
:1025D0002E6A2B4605F108000022597D21B1997D14
:1025E0000AB1914200D20A4602339842F5D1002A3C
:1025F00000F02981012393405A1ED10440F1EC8060
:102600004FF480520D48452104F018FF6FF0150279
:102610000B4845215AE700BF91A60000FEA6000026
:10262000AEA60000D0A600001CA7000036A7000040
:102630005346445050A700006DA7000011A80000A9
:102640007DA80000EB792E78A9798C4846EA03260C
:102650006B791B0243EA014329790B430393EB781F
:1026600002936B780193AB780093A5EB0A02334693
:10267000D210492104F0E2FEB6F57F4F40F0988079
:1026800095F803906E79C7F804D0B9F1140F28BFFC
:102690004FF014094FEA89094B46242B38BF2423F5
:1026A000073303F4FF63ADEB030DAB79206936020A
:1026B00046EA03462B790DF110081E4305F024F875
:1026C0003302CDE9008905225A21204605F022F87F
:1026D0000646206905F016F8002E75D1D8F80430AA
:1026E000D4F810B0002B0BF1150963DA23F0004386
:1026F0000122A3F12006C3F1200102FA06F622FA14
:1027000001F10E4302FA03F3DB0843EA4676B6F51D
:10271000801F34BF6B214D2122685948009134BF7E
:10272000B30A330D492104F089FE002108224846EE
:1027300004F058FF01214A464046396005F013FA7B
:1027400039680131C9B2052909F10209F3D1EB78E1
:102750000A2B88BFD8F82820CBF8206083BF01233C
:10276000C2F3031293404FF48073ABF81E3020691C
:1027700004F0CAFF0023CDE9003380220621204661
:1027800004F0C8FF0646B8B9CDE900000346802230
:10279000B721204604F0BEFF064668B92269137DC2
:1027A00043F001031375206904F0ACFFD7F804D09F
:1027B000083507E70133A7E7206904F0A3FF314894
:1027C0003246452104F03AFE2F483246492104F0B2
:1027D00035FED7F80CD0CCE6C6F30B0333B12B484B
:1027E00033464FF48052492104F028FE4FF48053C1
:1027F000360BAB626E62206904F086FF636893F863
:102800002030DA072ED50023CDE900338022B9210C
:10281000204604F07FFF054630BB6368256993F8C6
:102820002030DB0712D4284604F06CFF206904F046
:102830006BFF204605F00BF90546206904F062FFA6
:1028400005EAE57508E66FF08502E1E606F09BFE15
:102850004FF47A72A0FB020302FB0131C00B40EA85
:10286000414028612069DFE7206904F04BFF002D1B
:10287000DCDA15F1860FD9D0EEE500BF94A7000091
:10288000BAA70000D2A70000F8A7000047A80000E0
:10289000024B0B6001231360704700BFA01500209E
:1028A00000487047C899000070B50D462846194683
:1028B00016461C4605F01AF940B9084823462A4630
:1028C000452104F0BBFD6FF0150070BD24B1224618
:1028D0002946304604F07BFE0020F6E7ACA8000055
:1028E00010B5012211460648064C06F0D7FC06F04A
:1028F0000AFC206006F003FC6060002010BD00BFF1
:10290000A8150020A0150020F8B50E46144606F0C4
:10291000F6FB21460546304605F0E8F8374650B349
:10292000B6FBF5F305FB136323B9B4FBF5F305FB25
:10293000134343B1124823463246452104F07EFD3D
:102940006FF0150002E0A54201D90020F8BD4FF05C
:10295000FF324FF0FF330B4803F004FC06F0CFFBCF
:102960000546384602F08EFF641B2F44F9D1054816
:1029700003F0D4FBE9E70448234632464521DDE76E
:10298000CEA80000A8150020ACA80000F8B50E469F
:102990003046194617461C4605F0A8F840B91848B5
:1029A00023463246452104F049FD6FF01500F8BD7D
:1029B00046EA040515F0030504D0124823463246C2
:1029C0004521F0E7A4B110484FF0FF324FF0FF333C
:1029D00003F0C8FB24F00304AC4206EB050009D168
:1029E0000A4AD2F80034DB07FBD5074803F096FB10
:1029F0000020DCE7795902F065FF0435ECE700BF01
:102A0000ACA80000F2A80000A815002000E00140DA
:102A100038B545682B69B3B11035284602F016FE6B
:102A2000044680B90146284602F0DCFD084B984276
:102A30000BD108492246284602F0BCFD224605215A
:102A40000620FFF7C1F9002038BD6FF00400FBE756
:102A50000000AD0B592A0000430970B507D10B4B9C
:102A6000596821B101250C68094E854001B970BD36
:102A70008A682A4002D04B68304698471CB12368C8
:102A800021461C46F2E72346FAE700BFB8150020AE
:102A9000589600002DE9F043476840F20636D0060C
:102AA0003B7B87B002EA060654BFC2F34010032006
:102AB00001F01F05B6F5837F144645EA43158DF8EE
:102AC000030043D00FD8062E18D007D8B6B1022E77
:102AD0003ED06FF0150007B0BDE8F083B6F5807FFB
:102AE000F7D101260AE040F20222964232D0B6F532
:102AF000407F31D0B6F5007FEBD1022601232203BF
:102B000003FA01F12AD57B68C3F808153B695BBB62
:102B100005F01F026D0974D1920002F1A04284F405
:102B20008031D2F80037C1F30041C4F3404423F4AC
:102B3000E16344EA410423F007031C4344EA8004B0
:102B400044EA0624C2F800470020C4E70726D5E778
:102B50000426D3E70526D1E70326CFE7630344BF66
:102B60007B68C3F80C15D1E710370DF10202294636
:102B7000384602F025FD14F4403F80460CD129462A
:102B8000384606F0AFFA214B9845DDD19DF802108A
:102B9000384602F065FDD7E701AB4FF0000903AA04
:102BA00029463846CDE90439CDE90199CDF80C9094
:102BB00002F0DAFB154B98428BD114F4003315D098
:102BC0009DF803308DF80E3084F48034C4F3004453
:102BD0004B4603AA294638468DF80C608DF80D4007
:102BE00002F072FC094B9842CDD072E7CDE9043374
:102BF00003AA0DF1030329463846039302F0B4FB00
:102C0000F0E702F5E07253F82230FFDE0000AD0B72
:102C1000F0B54068057B01F01F0444EA45140569DE
:102C200087B0002D60D0B2F5001F00F1100506D16D
:102C30002146284606F058FA002007B0F0BD01AE44
:102C40000027B2F5800F0197776038D1B3F1007F8C
:102C500014BF052304238DF804300023CDE9046359
:102C60000393836823FA01F111F0010119D1B2F144
:102C7000A07F16D104F01F03620903F5E07339D178
:102C80004FF0A04252F82330DB070AD40DF10306BF
:102C900032462146284602F093FC184B984219D040
:102CA000029603AA2146284602F05EFB144B984286
:102CB0001DD101222146284602F0DEFCBCE7B3F11B
:102CC000C06F05D0B3F1007F14BF01230223C2E718
:102CD0000323C0E73146284602F0C8FC084B98425F
:102CE000DED06FF00B00A8E76FF08500A5E76FF06E
:102CF0001500A2E751F82330FFDE00BF0400AD0B42
:102D00000000AD0B37B5134D284606F07DFA88B9A3
:102D10002A681148452104F091FB6FF01204204607
:102D200003B030BD2A680D4800941A23452104F0F1
:102D300085FBF4E72A69A968136823F080631360B0
:102D40000B684FF420221A2128469847041EE9DB1D
:102D50000024E4E75896000047A9000063A900009A
:102D60002DE9F0435B4E5C4F00EB810140F2FF1513
:102D7000814202D10020BDE8F083046814F4804F42
:102D8000C4F3C32CC4F3080340F09080240E16F85B
:102D90000CC0AB4208BF4FF0FF33192C00F2898002
:102DA000DFE804F00D13191C1F251C878787873661
:102DB00063878787878787878787667B7E81C2F857
:102DC0000C355C1C5ED10430D2E7C2F814355C1CB3
:102DD000F9D000245FE0C2F80835F2E7C2F81035F8
:102DE000F5E75C1CC2F80835EDD0002404E05C1C5B
:102DF000C2F80C35E7D001245FEA531E5CD14FF0D6
:102E000001084FF0A04E08FA03F9CEF80C950AE03D
:102E1000C2F80835BCF1000FD9D15C1CD3D0002416
:102E2000A0464FF0060CD0F8009009F4004EBEF119
:102E3000000F1CBF4FF00008012403F01F0E5B09B8
:102E400042D14FEA8E0E0EF1A04EC9F34129DEF8B1
:102E500000373B4043EA890343EA0C2343EA080373
:102E600043EA4403CEF80037ADE7C2F80C35D1E7AA
:102E7000C2F86035B3F1FF3F0468A4D0C4F3004446
:102E8000002CB8D05C091BD101244FF0A04E04FAED
:102E900003F8CEF80885A046C5E7C2F86435E9E72F
:102EA000C2F86835E6E7C2F86C35E3E76FF0150065
:102EB00061E76FF085005EE70023C3F80C35FFDEA5
:102EC0000023C3F80835FAE70EF5E07E002353F837
:102ED0002E30F4E7ABA90000F0F8FCFF014B012213
:102EE0001A60704700C000400C2903690BD15B6A6F
:102EF000064907484B4393FBF0F100FB1133116087
:102F00005360002070476FF08500704790D0030039
:102F100040420F00044B00690022C3F80021D3F89F
:102F2000003103F0FBB800BF00C000407FB5056969
:102F3000AB6A63B33C2901D00C292BD105F11006F3
:102F40004FF0FF324FF0FF33304603F033F8134BAE
:102F50000193A86A0323002469460394029304F0B2
:102F6000D3F94FF0FF324FF0FF33284603F0FAF861
:102F7000A86A04F020FA0A4BD3F808256A620122F5
:102F80005A60304603F08EF8204604B070BD6FF0F2
:102F90000A00FAE76FF08500F7E700BFDD2E0000BA
:102FA00000C0004010B504690020FFF7E1F8A062FE
:102FB0004FF0FF320021204606F070F904F11000B6
:102FC00006F065F9002201210C20FEF7FDFE0C2021
:102FD000FEF7CAFE024B0122C3F80423002010BDF5
:102FE00000C000402DE9F041044647680D4606F058
:102FF00096F94FF0200888B9264B1B7873B16426E8
:10300000606804F06AFEF0B9012005F0EBFF013EB4
:10301000F6D10021212003F0F9FCF0E7EFF311864F
:10302000314688F31288BFF36F8F606804F055FE55
:10303000A8B986F31188BFF36F8FEFE786F3118885
:10304000BFF36F8FE5E7EFF31186314688F31288FF
:10305000BFF36F8F606804F040FE0028EED0BB69BC
:103060001D706368BA691B680020C3F844250122FB
:10307000C3F84825C3F82001D3F82041C3F858010C
:10308000D3F858019A6081F31188BFF36F8FBDE8C0
:10309000F08100BFB62F0020F7B5054600220121C0
:1030A0000220FEF791FE0220FEF75EFE6B681968B3
:1030B0001A69C1F824255A7D1B7D1343C1F86C356C
:1030C0006E68D6E9004313F001034FD02F6907F172
:1030D000080005F093FF324B984207D03148452154
:1030E00004F0ACF96FF0040003B0F0BD387A04F1DD
:1030F0000C0204F5907105F077FF387A012707FA82
:1031000000F001F0D7FE0823C4F80035B369C4F815
:1031100044350023C4F84835A760D4F85831002B53
:10312000FBD00021C4F800156B68DC6801AA2046BA
:1031300004F0A6FD002805DB019B226819791868B8
:10314000FFF70EFE6A6813680821C3F80015117AAC
:1031500051B9D269C3F834250122C3F83825C3F820
:103160001011D3F810111A600020BDE70822C4F82E
:103170000025B269C4F84425C4F848350123A3608A
:10318000D4F82031002BFBD00023C4F82031D4F830
:1031900020310123E3604FF48073C4F80433BCE7AB
:1031A0000000AD0BCBA900002DE9F341456806698D
:1031B0002F6A01AA0021384604F062FD041E18DBC4
:1031C000019B3A6819791868FFF7CAFD041E10DBE5
:1031D000696A481C18D005F1280000F0BBFA10F10C
:1031E000130F044609D12748452104F027F96FF051
:1031F0001204204602B0BDE8F081411D04D12248EE
:10320000452104F01BF9F4E7EB699847B5680127FD
:10321000D6E9023203EBC2039D4204D3304604F0E8
:10322000BEFD0024E5E7286805F0EEFF38B92A68FE
:103230002B7912681548452104F000F9D7E7286872
:103240002979EB88D0F810C0D0F80880DCF800406D
:10325000DA0754BF43F4B01383F4D01323F480127D
:1032600007FA01FEDB074CBF4EEA040424EA0E0411
:10327000CCF80040D8F800309847041EB9DB083578
:10328000C6E700BF0DAA00003DAA00005FAA00002B
:103290007FB50546406829698A6C0B6D0ABBABB1E6
:1032A0004C6C8B6516461A46C96C0291CDE90046F6
:1032B00011B3002B18BF134600226946039302F096
:1032C0003DFC0E4B98420AD06FF004032C69236337
:1032D00004F1200002F022FF002384F85C3004B0E7
:1032E00070BD4C6C13B19A4228BF1A46002C8A65F7
:1032F00014BF16460026D7E70B46DDE70000AD0BEE
:1033000038B503780C4663B98D6D5DB94B6D1C699A
:103310006FF07303236304F1200002F0FFFE84F8D2
:103320005C5038BD8B6C2BB19D4211D92148452191
:1033300004F084F8236DA26D2BB19A4220D91D4868
:10334000452104F07BF8606DBDE83840FFF7A0BF71
:103350005B1B8B6473B94B6B08334B638B6B013B0B
:103360008B6301F1480204F13400383104F0F0FCC1
:103370006064DFE74B6C002BDCD02B444B64D9E757
:103380009B1A23657BB9E36B0833E363236C013B32
:10339000236404F1500204F1400104F13C0004F004
:1033A000D7FCE064CFE7E36C002BCCD01344E3649C
:1033B000C9E700BF88AA00002DE9F04F89B00F4689
:1033C0000093436801938B880469990406469146EB
:1033D0002DD44FF0FF324FF0FF3304F1100002F014
:1033E000C1FE6760D6F81080D6F804A098F85D306A
:1033F00023B1D8F800309F4200F0C380B7F804C072
:103400001CF4006F1AD0B148452104F017F86FF092
:10341000850523689B8813F4005304D1636004F18D
:10342000100002F07BFE284609B0BDE8F08FA369CA
:10343000002BCED163689F42CBD1D3E71CF0010FA4
:1034400007D03268A248452103F0F8FF6FF0150558
:10345000DFE71CF0080F04D09E48452103F0EEFF83
:10346000F4E7CCF34513082B02D09B484521F5E740
:103470003D689A4B9D4202D899484521EEE70AF1F2
:10348000080BBBE80F000DF10C0EAEE80F00DBF8E7
:103490000030CEF80030934B9D4251D9924B9D4263
:1034A00051D9924B9D4251D9914B9D4251D9914B4B
:1034B0009D4251D9904B9D422CBF4FF000454FF09B
:1034C00080451CF0020F05950CF0040347D0002B3B
:1034D00014BF032302238DF81830CCF300138DF8AA
:1034E0001930DAF80030D3F808251CF0020FCCF3BD
:1034F00040014FEA52104FF0010334D1002840F050
:10350000218193404FF0A042C2F80C3598F85D300D
:103510002BB1504602F0DAFA002388F85D30774A82
:10352000434603A9504602F09DFA754B9842024665
:1035300022D07448452103F081FF6FF0040568E74D
:103540004FF00075BDE74FF08065BAE74FF00065BA
:10355000B7E74FF08055B4E74FF00055B1E7003BB7
:1035600018BF0123B7E7002840F0EF8093404FF0E9
:10357000A042C2F80835C9E7012388F85D30C8F8D1
:103580000070012384F85C30019B596A4A1C09D001
:1035900003F1280000F00EF9743003D15A48572186
:1035A00003F04CFFB9F1000F72D1C4F8349000233E
:1035B000A36304F1480204F1380104F1340004F07B
:1035C000C7FB009B6064002B6AD1E3630023236484
:1035D00004F1500204F1400104F13C0004F0B8FB96
:1035E000E06420680023236348B183683BB1012174
:1035F000083004F0C0FB2368186905F000FE30466F
:10360000FFF746FE0022A06B1346834250D10023F1
:10361000256C1946A94252D19342274638BF13461A
:103620004FF4FA5202FB03F557F8203B4FF0000825
:103630001B68B5FBF3F54FF4004CC835414640F22A
:10364000E7304FF47A720023E5FB0C01FCF746FDEE
:1036500002460B46384602F085FD002858D02B481C
:10366000452103F0EBFE0198C4F8588002F02EFAD1
:1036700084F85D8036696FF07305356306F12000CC
:1036800002F04CFD86F85C80384602F091FD43E084
:10369000D9F800306363002B89D0D9F8043087E76C
:1036A000009B1B68E363002B90D0009B5B688EE758
:1036B000616B01EBC301013349680A44A5E7E06B84
:1036C00000EBC100013140680344A3E7ABAA00004E
:1036D000CAAA0000F1AA000015AB000047E80100EB
:1036E00049AB00008FD003001FA107003F420F002D
:1036F0007F841E00FF083D0000127A0001330000A5
:103700000000AD0B7FAB0000ABAB0000DAAB0000FC
:10371000256B15F1740FA6D02368002B3FF479AE0A
:103720009A68002A3FF475AE998811F480567FF4A8
:1037300070AE186905F063FD20683146083004F06A
:103740001AFB66E6C1F80C15FFDE0023C3F8083546
:10375000FAE700BFF0B587B001238DF802300223ED
:103760008DF804306B4403930F4601AB0DF1030158
:103770000024049305460291059401F077FF0C4B59
:10378000984206460FD103AA3946284601F0ECFDBF
:10379000B0420BD09DF80310284601F061FF6FF096
:1037A000040007B0F0BD6FF01200FAE72046F8E71A
:1037B0000000AD0B2DE9F0410D46064605F096FCE4
:1037C000002207462946304601F056FF6B0905F0F6
:1037D0001F0429D1A40004F1A044164BD4F80027FB
:1037E000134043F00C03C4F8003704F00EFB80468E
:1037F0003368DB597BB100273046294605F074FC5D
:10380000D4F800270B4B134043F00403C4F80037EF
:103810003846BDE8F08104F0F8FAA0EB080006286D
:10382000E6D96FF07307E7E704F5E074002353F877
:103830002430FFDEF0F8FCFF70B5012383400E4A10
:10384000BFF35B8FDC4352E8001F01EA040542E846
:103850000056002EF7D1BFF35B8F4FF480328240C9
:103860000648C0F80823BFF35F8FBFF36F8F0B428A
:1038700014BF0120002070BD001600200010014080
:1038800070B40E49D1E90034D01AC31844F10004D1
:1038900022F07F46C1E90034A6F50013B3F5400FCE
:1038A00009D2074B1B681A0A1B069C19054B42F1EB
:1038B0000005C3E9004570BC03F03EBA780600205D
:1038C000041600208006002011B3BFF35B8F012394
:1038D000104A834052E800CF4CEA030C42E800C192
:1038E0000029F7D1BFF35B8F0B4A4FF4803383403D
:1038F000C2F80433094BBFF35B8F1B68BFF35B8FC8
:10390000C340DB0742BF064B4FF40032C3F800212F
:10391000704700BF0016002000100140FC15002079
:1039200000E100E00D4B1868010A0006BFF35F8F4D
:103930000B4BD3F80435181841F10001B3F5801F83
:103940000AD2084BD3E90023904271EB030303D260
:1039500010F1807041F10001704700BF0416002093
:1039600000100140800600202DE9F04F85B016467A
:103970001F469DF840A00446FFF75EFF0190FFF749
:10398000D1FFB04271EB070354D23E4B301A67EBC4
:103990000101984271F100014FD23B4B03EB04133C
:1039A000D3E902239F4208BF96425ED037494FF4C5
:1039B000803804F1500508FA04F8AD00C1F84883D6
:1039C0002046ADB204F015FA26F07F4B05F1804594
:1039D00004F5A87305F58835DC464FF0030902931A
:1039E000029A2CF07F4341F82230C1F84483D1F889
:1039F0000435274A6FF00200C01A604420F07F406F
:103A0000904232D9286868B1D1F804350393A3EB0A
:103A10000B0020F07F40B0F5000F26D9204604F0BF
:103A2000E8F9039BBAF1000F07D109EB030C09F188
:103A30000109D5E7BAF1000F09D06FF0150520464E
:103A40000199FFF741FF284605B0BDE8F08F01233B
:103A5000104ABFF35B8FA34052E8000F184342E8BF
:103A600000010029F8D1BFF35B8F07490E982301AD
:103A700001EB0412C8500F9B5360C2E90267002596
:103A8000DDE700BF01008000680600200010014053
:103A9000FDFF7F00FC1500207FB51C4C1C4BC4F8BB
:103AA0000833C4F848331B4B00254FF0FF304FF06C
:103AB000FF31C4F80855C3E902014FF48033C4F85C
:103AC0000433154B02264FF400320121C4F804637D
:103AD0001120C3F880212A46FEF776F91120FEF75F
:103AE00043F90E4A0123A360236013600C4B0D4A77
:103AF0000093CDE9015500232846FFF735FF3046F6
:103B0000FEF73EFB284604B070BD00BF0010014028
:103B100003000F006806002000E100E0001600200E
:103B200081380000FFFF7F002DE9F7432F4CD4F8C8
:103B3000043399070BD5D4F8043143B12C4A002340
:103B4000C4F80431D4F80431136801331360D4F895
:103B50000433DA0329D5BFF35B8F264B53E8002FDC
:103B600022F0010143E800100028F7D1BFF35B8F7A
:103B7000D30702D4D4F84031BBB10025C4F840517A
:103B8000D4F84031FFF7CEFEEFF31182202383F308
:103B90001288BFF36F8F184BD3E90267B042B94167
:103BA00006D282F31188BFF36F8F03B0BDE8F083B4
:103BB0004FF0FF384FF0FF39C3E90289D3E9001015
:103BC0001D604FF48033C4F84833C4F84051D4F832
:103BD000403182F31188BFF36F8F0029E5D0009048
:103BE00032463B4628468847DFE700BF00100140C9
:103BF00004160020FC1500206806002030B5431C88
:103C0000124C85B005D08442A8BF0446012CB8BF31
:103C10000124FFF787FE0E4B0C4DD3E90013401A29
:103C2000B0F5000F10D22218AA4228BF2A46521817
:103C30004FF0000007490091CDE9010043F1000376
:103C4000FFF792FE05B030BD2A46F0E7FFFF7F0088
:103C5000780600208138000008B5FFF763FE024BAC
:103C60001B68C01A08BD00BF7806002010B5084CBC
:103C7000012363601120FEF785F8064BC4F8083372
:103C8000C4F84833044B4FF40032C3F8802110BD10
:103C90000010014003000F0000E100E030B5816832
:103CA00085B0103921F00704054603F01EFC1022F0
:103CB0000146684603F096FC07491022684603F067
:103CC00086FC10236A462146284603F0DAFB0038BA
:103CD00018BF012005B030BD7A9C000030B50D46FC
:103CE000816887B0102302AA1039044603F0B4FBA0
:103CF000002802DA012007B030BD102202A92046B8
:103D000004F09BF800283AD11E49102202A803F0C3
:103D10004EFC00280CBF012302232B70204604F028
:103D200078F8012301460DF10702204603F094FBC9
:103D30000028DFDB9DF8073003F00F021B096A70D3
:103D40002B7101220DF10701204604F076F810B91D
:103D50006B78042B03D901236B7000232B71A268AD
:103D6000183A22F00702083AA91C204604F078F815
:103D70000028BFD1E91C204604F08EF8BBE70323DE
:103D8000CBE700BF7A9C0000F0B5354F460085B008
:103D90000546694657F8260004F084F8044610B139
:103DA000FF2005B0F0BD013602A957F8260004F047
:103DB00079F8012837D12B482A46492103F03EFBE8
:103DC000294B02938DF80C409DF800609DF8087017
:103DD000264C00222078314604F021F850B3607858
:103DE000394604F01CF828B3A378042B03D09DF8BF
:103DF000031099421ED1E378042B03D09DF80B10D9
:103E0000994217D12379042B10D16279022A1DD14E
:103E1000174B18482A46492103F010FB6079831E8E
:103E2000022BBED9BCE70028CED0B9E79DF802101E
:103E30009942EAD00132032A04F10604CAD10E489D
:103E40002A46492103F0FAFA0120AAE7032A05D0FD
:103E50000A4B0B49042A08BF0B46DAE7094BD8E79F
:103E6000289B00004FAC000003010303E4AC0000FA
:103E700031AC00009AAC0000BEAC000036AC0000D3
:103E800048AC00002CAC0000044B1B6858404308B1
:103E90005B4240421843C017704700BF081600201D
:103EA0008842F0B504D0094F04380025AA4200D159
:103EB000F0BD3E6850F8044F5E4024EA060451F815
:103EC00025601E40344304600135EFE708160020EA
:103ED0002DE9F04F8DB01D46189B179F1A9E059235
:103EE000B3F12A3F83468A4640F08D8039461698C2
:103EF00004F047F8012838BF0120470900F01F04EB
:103F00007B01502B4FF0010934BF4B4603230A932A
:103F100009FA03F30B930A9B059805FA03F306EBE2
:103F20008303069303EB8503079304F002FA4FEA39
:103F30008508089042460021304603F053FB079B5A
:103F4000C6F800900393089B199ACDE90153059B8D
:103F5000009331462B46304606EB080904F0FAF987
:103F600051464246484603F032FB02234946099334
:103F70000B9B099A934248D142463146584603F07A
:103F800026FB4FF00009CA46079B0393089BCDE927
:103F90000153059B00935A462B465946584604F058
:103FA000D9F9002C47D1013F1F24169B53F8273025
:103FB000E34003F0010343EA49090A9B0AF1010ABD
:103FC000534503D0002CDFD1002FDDD1189BB3F176
:103FD0002A3F32D10698424609FB086103F0F7FAFE
:103FE000079B0393089B069ACDE90153059B009319
:103FF00059462B46584604F0ADF9002CC1D1BFB943
:104000000DB0BDE8F08F00247AE7079B0393089B6F
:1040100001EB080ACDE90153059B00934A462B4664
:10402000504604F097F9099B0133099351469FE7E5
:10403000A146A246A8E7013CB7E731464FF0000A87
:104040000A4B18681B68584080EA090080EA0A0099
:10405000FFF71AFF2A46C3430698FFF721FF099B83
:104060000AF1010A53454144EAD1B9E70816002094
:10407000054B1B68013143400132084022EA03022C
:104080000243501E00B27047081600202DE9F04F81
:1040900099B083460F46184600211646039304F054
:1040A000CAFB002800F08981784B14930024012575
:1040B00015AB039913933046CDE90B45CDE90D457A
:1040C000CDE90F45CDE9114504F03EFBA04228DAC9
:1040D000BBF1000F05D1E7B90024204619B0BDE8B7
:1040E000F08F2146584604F0B7FA04460028F2D073
:1040F0000BA804F0FEF90DA804F0FBF90FA804F0DA
:10410000F8F911A804F0F5F90C2115A800F038FB16
:10411000E3E73146384604F06AFA04460028E7D15E
:10412000DAE731460BA804F062FA04460028DFD132
:1041300003990DA804F05BFA04460028D8D1F18851
:10414000ADF8385002310FA8ADF8305004F0DFF967
:1041500004460028CCD101460FA804F07DFA04469D
:104160000028C5D1F18811A8023104F0D0F9044625
:104170000028BDD10DA804F09BFA00F01F001F28F5
:1041800073D0C0F11F0319460BA8019304F0B6FACF
:1041900004460028ACD101990DA804F0AFFA0446FA
:1041A0000028A5D1BDF83250BDF83A80A5EB080A29
:1041B0004FEA4A1949460DA804F0A0FA044600281F
:1041C00096D14FEA8A0A0DA90BA804F0ECFA002850
:1041D0004DDA49460DA804F0AEFA0446002887D10E
:1041E00008F1FF3305939B0005F1FF3A069305F1B3
:1041F000804508F18043023B013D9B00A5EB08058B
:104200000893AB000293059B9A4541D8BBF1000F80
:104210000DD00FA9584604F0EAF9002840F0C980F3
:10422000039AB388928813FB02F3ABF80430002F93
:104230003FF45EAF01990BA804F07DFA002840F02E
:10424000B880B388ADF830300BA9384604F0CFF908
:104250000146002840F0AF80384604F0ECFA002810
:104260007FF446AF0123BB8042E701949AE70F9A9F
:1042700052F80A300BA9013342F80A3008460DAA59
:1042800004F0BFFB044600289DD031E70100030085
:104290000D9B069A04931344DDF82C900793049B1E
:1042A00059F82A109A580F9D4FEA8A08A8F104037A
:1042B0000993029B91421D4476D2A8F10400002389
:1042C00059F80000FBF70AFF002914BF4FF0FF3335
:1042D0000346BAF1010F2B6016BF09EB0803002358
:1042E00053F8083C1593A8F1040359F803301693CA
:1042F00059F8083017932B68DDF8108001332B60D4
:10430000089B98442B68013B2B60002111A804F006
:10431000A3F900284DD1059B002B48D0D8F80020E8
:10432000119B1A60079A12685A6011A92A680846F8
:1043300004F06BFB00283CD113A911A804F033FA58
:104340000028DFDC2A680DA911A804F05EFB80BB01
:10435000029B4FEAC308414611A804F0CFF940BBC5
:104360000BA9084611AA04F04CFB014618BB0BA888
:1043700004F061FA002812DA0DA911A804F037F947
:10438000B8B9414611A804F0B9F990B90BA911AA1E
:10439000084604F033FB60B92B68013B2B60029B9D
:1043A0000AF1FF3A043B2DE74FF0FF3391E7059AFE
:1043B000B6E704469CE60C469AE66FF00B048CE6E2
:1043C0002DE9F74F90461F4A1568454006460F46AF
:1043D000ED43002B14BF9A468A4600240C9B04F13F
:1043E00004094B4505D20C9B9C4220D303B0BDE889
:1043F000F08F042208EB04010DEB020003F0E7F854
:10440000019A06EA020B04220AEB04010DEB0200FA
:1044100003F0DDF8019A2A4042EA0B0201920422DD
:1044200038190DEB020103F0D2F84C46D6E718F824
:1044300004301AF8042033402A4013433B5501341A
:10444000D1E700BF08160020082804D00928034837
:1044500018BF002070470248704700BFF6AC00004C
:10446000F9AC000001680E4A9142034615D1C169BA
:10447000A2F11022A2F1EF1291420ED18268012A1C
:104480000BD8C26812B101698A4206D0586928B1B6
:104490009B691B1A5842584170470120704700BF62
:1044A00055AA00FF70B50D4B9E68A6B13046FFF7C8
:1044B000D9FF044678B9F3686BB935690DB9204660
:1044C00070BD2846FFF7CEFF28B9EB68B34202D192
:1044D0002E462D69F2E70124F1E700BF0C160020FB
:1044E0002DE9F8433F4F3C68D4B1BC68C4B1002803
:1044F0004AD0002948D001FB00F5B5FBF0F0884216
:1045000042D1281D40D8A9070DD025F00306043656
:10451000FC6803E06368B34238D2A469002CF9D187
:104520002046BDE8F8832E46F2E7FB6041E006F145
:1045300020016318203A5A600022C3E902242A4865
:1045400022691A6160502949D96102B1D360626958
:104550005A61A1699961AAB193619A6902B15361E3
:104560004FF00109C4E9016923610023C4E905335F
:104570003B69DB072ED5FFF795FF58B31C4B484628
:104580001B6826E0FB60E8E70024C9E7A3681BB1CD
:10459000174B01201B6898476268921B232A04F17D
:1045A0002008C4D80123A360D4E90523002ABCD085
:1045B0009361A3690BB162695A610023C4E90533B1
:1045C0003B69DA0706D5FFF76DFF18B1084B1B688A
:1045D000012098472A4600214046444603F002F84D
:1045E0009EE700BF0C16002055AA00FF669911EE49
:1045F000A005002070B50546002800F08880444ED4
:104600003368002B00F08380B268002A7FD0834299
:1046100003D872681344984203D33E4B01201B68B1
:104620009847A5F120042046FFF71CFF18B1394B2D
:1046300001201B68984755F8183C012B03D0354BD7
:1046400001201B689847002345F8183C55F8143C96
:104650003BB39A682ABB55F81C2C02F120015A681A
:104660000A445A6055E905321A6155F8145C2B6901
:1046700003B1DD6020220021204602F0B3FF28694B
:1046800010B18368002B2ED033699B073FD5FFF70D
:1046900009FF00283BD01F4BBDE870401B6801207C
:1046A000184755F8100C00282AD0836843BB42688D
:1046B000636813442033636003692361D4E90523ED
:1046C0009AB9CBB9436963618269A261B3B19C6154
:1046D000A36903B15C61236903B1DC60202200217E
:1046E00002F080FFD0E72C46E1E79361A369002B3D
:1046F000E8D062695A61E5E7F360F7E7F460E7E75D
:10470000F36845F8083C03B15C61F460BCE770BD38
:104710000C160020A005002038B514220C460546D2
:104720000021134802F05EFF1249134800F040F8E0
:10473000232C1CD915F003031FBF043CE418C3F15C
:104740000403ED1822460021284602F04BFF084BD7
:104750000A499D60C3E90054203C6C609A6811606E
:104760009A68DA60A1F11021A1F1EF11D16138BD91
:104770000C160020F5450000E144000055AA00FF9A
:1047800010B50A46044619B1024B00211B68984730
:1047900010BD00BF9C050020014B1B68184700BFDF
:1047A000A8050020014B1B68184700BFA405002086
:1047B000024B1860024B002019607047A8050020CA
:1047C000A4050020F8B500F1080647680446304605
:1047D0000D4603F071FF87424BD16368B3F5807FCC
:1047E00047D80021304604F026F8002841DD00219A
:1047F000304603F04DFFE0B345B9294604F11000FF
:1048000004F019F8002834DD0020F8BD04F120057B
:104810000021284604F00FF800282ADD0021284650
:1048200003F036FF28B304F128050021284604F0E0
:1048300002F800281DDD0021284603F029FFC0B141
:10484000002104F1100003F0F6FF002811DD002123
:1048500004F1300003F0EFFF00280ADD002104F12D
:10486000380003F0E8FF002803DD002104F14000D8
:10487000C6E70148C9E700BF80BFFFFF012938B57F
:104880000546144601D0074838BD22B90123C5E9C1
:104890001C340020F8E71046FFF7D6FD0028F5D1BC
:1048A000F1E700BF00BFFFFF70B500210446FFF72E
:1048B00089FF054610B10E4D284670BD04F108066B
:1048C000304603F0F5FE7F28F5D9103429462046FE
:1048D00003F0DEFE0028EED0204603F0E9FE0128BA
:1048E000E9D93146204603F05EFF0028E4DBE2E729
:1048F00000BEFFFFF0B50C4685B000210546164608
:10490000FFF760FF002839D102A803F0EDFD214632
:104910006A6802A803F0D6FE044618B102A803F0A4
:10492000E8FD0CE005F10804214602A803F03BFF76
:10493000002807DB02A803F0DCFD6FF00304A4F5F8
:10494000854418E005F1480302A96F68009305F15A
:1049500010022346084604F0A8F904460028DDD1D9
:104960003A46314602A803F0C3FE044602A803F00B
:10497000C0FD002CE3D1204605B0F0BD004CFAE7A5
:1049800080BFFFFF01292DE9F041034641D8224AAB
:10499000224F2348234E244D244C9966002918BFEA
:1049A0009046234A18BF964602F1794202F57402F6
:1049B00002F5016218BF94461E4A18BF17461E4AE8
:1049C00018BF164602F1D14208BF804602F5C01258
:1049D0001A4802F51E620CBF864615461848194A49
:1049E0000CBF844614461848A2F11162A2F50C22AD
:1049F000A2F28E2218BF02460020C3E91000C3E9CC
:104A0000128EC3E914C7C3E91665C3E91842BDE8AD
:104A1000F0816FF07300FAE7D89E05C13AF54FA513
:104A200067E6096A7F520E518C68059BABD9831FDC
:104A300007D57C3639590EF7310BC0FF85AE67BB01
:104A400072F36E3CA78FF964A44FFABE2DE9F04FC4
:104A5000CFB000F1640300F144070DF58A790093AB
:104A600001914A463B4653F8041F42F8041F00993F
:104A70009942F8D104ADDFF800A14FF000082C46B0
:104A8000B8F10F0F61D8019B042203EB880103A842
:104A900002F09DFD039804F0A8F9A860D4E94763EB
:104AA000D4F818C15AF8041B73404FEAFC22D4F81A
:104AB000206182EABC1203EA0C0382EA7C62734042
:104AC0001344D4F82421D4F8106113440B44D4E9DE
:104AD000421E034441EA0E024FEA713080EAB100FF
:104AE000324001EA0E0B80EAB15042EA0B02024466
:104AF000D4F81401626018441344D4F82021C4F897
:104B0000242108F10108D4F81C212360B8F1400FDA
:104B1000C4E947C2C4E944E6C4E94231C4F8180113
:104B200005F10405ACD157F8043F59F8042F13449C
:104B30003B60009BBB42F6D104A84FF49471FFF791
:104B40001FFE00204FB0BDE8F08F2B6855F8382CC1
:104B500055F8341C4FEAF34080EA734080EA932012
:104B600055F8143C134418444FEAB14383EAF11357
:104B700083EAD103184490E7309B00004FF0704364
:104B800093F8E02F062A09D1D3F8E83FC3F30313C3
:104B9000033B042B02D8024AD05C704700207047C8
:104BA0000BAD0000024AD2F80034002BFBD0704756
:104BB00000E0014010B504F006FA40B14FF0805318
:104BC0008E4AD3F82433C3F30423C2F84035FFF7E9
:104BD000D5FF10B18A4B8B4A5A6704F0F4F948B1FB
:104BE0004FF080534FF08042D3F84432C3F3423346
:104BF000C2F83C35FFF7C2FF30B1834AD2F8FC302F
:104C000023F08073C2F8FC3004F0DDF940B14FF0BE
:104C100080430022C3F80C21C3F81021C3F83825C3
:104C2000FFF7ACFF20B14FF080430322C3F8A0256B
:104C3000FFF7A4FF60B1754B0522C3F810260122CF
:104C4000C3F888260022C3F818263F22C3F814268A
:104C50004FF08053D3F83021511C09BF4FF07043FF
:104C6000D3F8343193F8E02FD3F8E83F08BFC3F30B
:104C70000313062A4DD1033B042B03D8644AD35CAB
:104C8000002B46D04FF08052624BD2F80414C3F888
:104C90002015D2F80814C3F82415D2F80C14C3F860
:104CA0002815D2F81014C3F82C15D2F81414C3F830
:104CB0003015D2F81814C3F83415D2F81C14C3F800
:104CC0004015D2F82014C3F84415D2F82414C3F8C0
:104CD0004815D2F82814C3F84C15D2F82C14C3F890
:104CE0005015D2F83014C3F85415D2F83414C3F860
:104CF0006015D2F83814C3F86415D2F83C14C3F820
:104D00006815D2F84014C3F86C15D2F84424C3F8DF
:104D1000702504F058F948B14FF080534FF08042AD
:104D2000D3F8583203F04F03C2F8E43E04F04BF9D5
:104D300048B14FF08043D3F80024D20744BF6FF04E
:104D40000102C3F800244FF08053D3F83021062A23
:104D500026D1D3F83431033B042B02D82E4AD35C3E
:104D600063B12E4AD2F83C3743F48063C2F83C3733
:104D70004FF08053D3F83031062B11D14FF08053D0
:104D8000D3F83431033B042B02D8254AD35C3BB122
:104D90004FF01023D3F808224FF08043C3F8582572
:104DA0004FF01023D3F80022002A03DBD3F804329B
:104DB000002B22DA1B4901234FF01020C1F80435E3
:104DC0001524FFF7EFFEC0F80042FFF7EBFEC0F836
:104DD0000442FFF7E7FE0023C1F80435FFF7E2FEC7
:104DE000BFF34F8F0849104BCA6802F4E0621343C7
:104DF000CB60BFF34F8F00BFFDE710BD0030014017
:104E000000C007400DF0ADBA00ED00E000500040DA
:104E100006AD000000C0004001AD000000100040E1
:104E2000FCAC000000E001400400FA0530B5046865
:104E3000CCB1BFF35B8FB4FA84F3C3F11F03DBB2D1
:104E400001229A4024EA020250E8005FA54204D100
:104E500040E8002CBCF1000FF6D1BFF35B8FE6D128
:104E600002480B7030BD0248FCE700BF0000AD0BEC
:104E70000200AD0B10B50368CB40DB0714D401234F
:104E80008B400268BFF35B8F43EA020150E8004F9A
:104E9000944204D140E8001CBCF1000FF6D1BFF3EE
:104EA0005B8FEED1014810BD0148FCE70000AD0B5F
:104EB0000400AD0B014BC3F80405704700F001403E
:104EC000F7B5044618B1012823D003B0F0BD4FF068
:104ED00080430222C3F808230122DA60C3F80401E8
:104EE000D3F80431064601238DF8073042F21075DD
:104EF0004FF08047D4B1012CE7D1D7F80C3403F43C
:104F00008033AEBB83B3012004F06CF8013DF4D1D3
:104F10002AE04FF080430022C3F808035860C3F82A
:104F20000021D3F800310DF10706DCE7D7F818347B
:104F300003F480333EB9002BC7D0012004F052F8AF
:104F4000013DF3D1C1E7D7F8182402F00302326023
:104F5000002BBAD09DF80700012803D104F042F8D5
:104F6000013DC7D1012CB0D1054B00225A71ACE7ED
:104F7000D7F80C2402F001023270002BEAD1F3E7DB
:104F800020160020054B1A792AB99A71012218605F
:104F90009A80034870470348704700BF20160020DE
:104FA0000000AD0B0C00AD0B08B5074B1B682BB117
:104FB0000020FCF7FBFE08B9FCF7D6FE4FF080435B
:104FC0000022C3F8182508BD2016002038B5B0B15E
:104FD000012851D14FF080420023C2F80031D2F8AD
:104FE00000212E4A03F18043012119602C4B1B68DC
:104FF000002B4CD04FF08043C3F804033CE04FF04B
:105000008043D3F81814D3F81824CC0326D590077E
:1050100002D00020FFF754FF4FF080430022C3F876
:105020001825C3F804211F4AD3F80431D2F8FC0034
:1050300040F08073C2F8FC301B4B1C6844F0010147
:1050400019605D685968491BB1F50A5FFAD31C60A5
:10505000C2F8FC000823154A0220C3E7D3F8142441
:10506000D107D9D5D3F81C249207D2D10C4A1268A3
:105070001AB10222C3F8042338BDD3F80421002A50
:10508000FBD00022C3F80421D3F80431F4E71368FD
:10509000002BFCD0002313601368EDE700010040F3
:1050A0002016002000ED00E0001000E004010040A8
:1050B0004FF08043D3F80C14D3F80C24C80325D543
:1050C000D10723D5D3F81824D2031FD5114A9179DB
:1050D00001F0FF00E1B9C3F80C01D3F80C11022074
:1050E00001219171C3F8340C1961126822B10822B0
:1050F000C3F8042308487047D3F80C21002AFBD0DA
:105100000022C3F80C21D3F80C31F3E703487047B1
:1051100003487047201600200000AD0B0500AD0BC2
:105120000B00AD0B10B54FF08043D3F800216AB1EE
:105130000022C3F80021D3F800210122C3F808237C
:10514000184B587910B95A711B6898474FF0804333
:10515000D3F804215AB10022C3F80421D3F8042162
:105160000222C3F808230F4B01201B6898474FF019
:105170008043D3F80C21A2B1D3F80423120710D531
:105180000022C3F8342CC3F80C21D3F80C110821E9
:10519000C3F80813034B9A71BDE810401B68042044
:1051A000184710BD2016002070B500F108030C4C04
:1051B00034F81330DA0505460E4607D5C3F343230A
:1051C00004EBC30254F8333052689847A3682BB1FC
:1051D000E26831462846BDE87040184770BD00BF00
:1051E000AC05002010B4C0B2114A083032F81030BB
:1051F000D9051BD5C3F3432123F4F85322F810300B
:1052000002F10E04002034F8023F13F4807F03D033
:10521000C3F34323994209D001302028F3D100235E
:1052200042F83130034810BCFFF724BE10BC704771
:10523000AC05002004060020F0B505460020044619
:10524000012607468C420BD1114BD3F87C2132B199
:105250000022C3F87C21D3F87C3140F00040F0BD3F
:10526000E3B29B0003F580729B0806FA03F31D422C
:105270000BD002F1804202F5C042D2F800C0BCF16E
:10528000000F02D01760126818430134DAE700BF3C
:1052900000600040C0B2064B083033F810008306AF
:1052A00043BF400B800000F580704FF4BE70704724
:1052B000AC050020CBB20246083308460C4931F851
:1052C0001330990611D599070FD410685B0B012193
:1052D0009940C0F80813126802EB8303D3F8102535
:1052E00022F00302C3F810257047002103F0DDBE51
:1052F000AC050020F7B5CDB2174E0835074636F895
:105300001530DB070C4624D5FFF7D4FF36F81530EF
:105310009A0606D55B0B3A6803F5A273002142F8A2
:1053200023102046FFF75EFF002301A826F8153062
:10533000019403F067FE019B00EB8300074BD0F85C
:105340000027134043F00203C0F80037044803B0BD
:10535000F0BD0448FBE700BFAC050020F0F8FCFFFF
:105360000000AD0B0400AD0B2DE9FF4113680746AB
:105370000C461546FBB1CEB2DFF83C81083638F852
:10538000162002F02202222A22D00022CDE9002299
:105390008DF80E208DF80F200DF10E010DF10F028A
:1053A000204603F039FE38F8163023F0020343F0AC
:1053B000010328F816306B684BB393F800C05A68A5
:1053C0003D4EE3B2083336F81310880702D5B2B168
:1053D0003A481FE021F02001C904C90C26F8131037
:1053E0006AB1BCF1030FF3D86A6838685268127862
:1053F000BCF1000F11D102F5A27240F822C036F8BC
:10540000132022F01C0242EA8C0226F81320AB681B
:1054100043BB2B4804B0BDE8F08100EB820041EAB9
:105420004231D0F810E52EF0030EC0F810E53F68C9
:1054300007EB820741F02001D7F8100526F813107A
:1054400020F4473020F44070C7F810052002D7F848
:1054500010E500F4F85040EA0C4040EA0E00C7F8AE
:105460001005CCE7D3E900672046FFF7BBFE002E0E
:10547000CFD0114DD5E90023964203D19F4201D1EF
:10548000002209E00F480DF10F01FFF7CFFC0C4B94
:105490009842BFD19DF80F2045F83260E4B205EB89
:1054A000C20308345F6035F8143043EA422343F402
:1054B000807325F81430ACE7AC0500200400AD0B78
:1054C0000000AD0B040600202DE9FF4107460C4605
:1054D0001E4612B3CDB2DFF8D080083538F815304B
:1054E000980701D4990621D413F01C0F02D05378E9
:1054F000012B1BD001238DF80F300023CDE90023B1
:105500000DF10F01931C2046013203F085FD38F8A0
:10551000153043F0030328F81530002E42D0E1B2D5
:10552000214D083135F81120930703D41F4804B0EA
:10553000BDE8F08196F800E0D7F800C022F0200224
:105540000EF5A270D2040023D20C4CF8203025F8BE
:10555000112096F801C0BCF1000F23D03868B6784E
:1055600000EB8E004FEA0C4CD0F8103523F4981362
:1055700023F4F853C0F81035230203F4F8530CF465
:10558000403C3605D0F8107543EA0C0306F480164B
:1055900042EA4E32334342F020023B4325F81120C9
:1055A000C0F810350248C2E7AC0500200400AD0B7E
:1055B0000000AD0B014BC3E902127047AC0500209F
:1055C000C9B20831044B33F81130990643BF5B0B65
:1055D0000248137002487047AC0500200000AD0B74
:1055E0000400AD0B70B5164D95F8604006462CBB17
:1055F0002146402205F1100001F0F4FF30682E6DC5
:1056000021468E420ED10023C0F87C31D0F87C3187
:1056100040F30730FCF7A8FB01230A4885F8603007
:10562000AB6570BDCBB29B0003F580727C2B08BFCD
:10563000845001F1010108BF8358E2E70248F0E716
:10564000AC0500200000AD0B0C00AD0B034B93F834
:105650006000003818BF0120704700BFAC05002073
:105660000148FFF707BC00BF000600200148FFF714
:10567000DDBB00BF0006002073B503680C46D3F8FD
:1056800004130029A4BF4FF00041C3F80413E3B290
:105690001D49083331F8133099061AD513F0020664
:1056A00017D15B0B9C00056804F580716E5069583A
:1056B00001682144D1F8104544F00104C1F81045B7
:1056C0002AB10168012202FA03F3C1F8043302B0DF
:1056D00070BDC3F38203042B12D0052B12D001A896
:1056E000019403F08FFC019AD0F81035D34003F0F9
:1056F0000103991C204602B0BDE8704003F0D5BC00
:105700000321F7E70221F5E7AC0500202DE9F34777
:10571000544B554FD3F80403396DC0B240F00040EC
:10572000FFF78AFD051E18DA0023F96D009368461D
:1057300003F0CAFC4FF0010897F85C30DA075AD43E
:10574000396D4FF00040FFF777FDF96D684603F0C3
:10575000BBFC0028F0D125F000450124002D69D1C3
:1057600002B0BDE8F08794FAA4F4B4FA84F4E00837
:1057700004F1080304F0070237F813901DF8003015
:10578000019408FA02F223EA02030DF8003001A89E
:1057900003F038FC019B03F5E0734FEA990150F8E0
:1057A0002360C9F3820A4B07D146C6F3014626D5CA
:1057B00020465146FFF7F8FC01A8019403F022FCB3
:1057C000019B03F5E073F6B250F82330C3F30143B5
:1057D0009E4207D10021204603F067FC3146204657
:1057E00003F063FC01A8019403F00CFC019B08FA90
:1057F00003F3C0F82035009C002CB4D1A0E7022EA2
:105800000CD10321204603F050FC0AF00503012BC4
:10581000E8D149462046FFF7C7FCE3E702212046CE
:1058200003F043FCBAF1030FF3D0032EDAD1BAF13F
:10583000020FEDE795FAA5F3B3FA83F304FA03F246
:105840009B0003F1804303F5C04325EA0205D3F82A
:105850001005D3F81015C0F30420C1F30141FFF780
:10586000A3FC7BE700600040AC050020044AD2F8AE
:105870000034DB07FBD50160BFF35F8F704700BFCB
:1058800000E001404FF080531A69B0FBF2F302FBD5
:10589000130373B9084B0222C3F80425C3F80805A3
:1058A000D3F80024D207FBD500220448C3F804250E
:1058B00070470348704700BF00E001400000AD0B97
:1058C0000A00AD0B10B5054C0123C4F80435FFF7F1
:1058D000CDFF0023C4F8043510BD00BF00E0014037
:1058E00001460148FFF7A2BA1006002007B5019053
:1058F00001A803F00CFC019B00EB8300054BD0F8E2
:105900000027134043F00303C0F8003703B05DF8ED
:1059100004FB00BFF0F8FCFF73B5CB7B0446002B03
:1059200038D10B7B0878012B77D803F007FC0B7874
:10593000019301A803F0EBFB019B00EB83003C4BC0
:10594000D0F80027134043F00103C0F8003748782F
:10595000FF2804D003F0F2FB4878FFF7C7FF8B78ED
:10596000FF2B0FD001A88D7B019303F0D0FB019B8F
:1059700000EB83002E4BD0F80027134043EA850349
:10598000C0F80037C878FF2804D003F0CAFBC878F5
:10599000FFF7ACFF23792748CA78282505FB0303C6
:1059A0009A770B7C9BB94B7825680E78FF2B18BF34
:1059B0001A468B78C5F8086508BF4FF0FF32FF2BF9
:1059C00008BF4FF0FF33C5F80C25C5F81035236824
:1059D0008A68C3F824254B7B0A7B2568003B18BFE7
:1059E0000123022A1CD0032A1DD0012A01D143F031
:1059F0000203C5F8543523794979282202FB0303B1
:105A0000D97723795343C35883B1206840F30730D3
:105A100002B0BDE87040FCF7A7B903F082FB86E74F
:105A200043F00403E5E743F00603E2E702B070BD8C
:105A3000F0F8FCFF2816002007B5019001A803F03C
:105A400066FB019B00EB8300054BD0F80027134059
:105A500043F00203C0F8003703B05DF804FB00BF59
:105A6000F0F8FCFF2DE9F04190F80480144C4FF061
:105A7000280C0CFB08FC04EB0C06074696F81CE00F
:105A8000BEF1000F19D144F80C20736041B1CB7BFB
:105A900086F82530CB78B3774B79F377FFF73CFF67
:105AA0003A6808480123C2F80035282202FB08445E
:105AB000002262772377BDE8F0810348FBE700BF4F
:105AC000281600200000AD0B0C00AD0B70B5067958
:105AD000194C056828237343E35833B145F3073065
:105AE000FCF750F90423C5F808330023C5F8003546
:105AF000282303FB064393F82530BBB9D5F80805E6
:105B0000FFF79AFFD5F81005421C01D0FFF794FF6C
:105B1000D5F80C05431C01D0FFF78EFF282303FBAB
:105B20000643987FFF2801D0FFF786FF282303FB59
:105B300006440023237770BD281600202DE9F84382
:105B40000779394C28237B439046E2180E46517F53
:105B50008146002966D1E3580BB10123537796E8BB
:105B60000F00282505FB074505F10C0C8CE80F00FC
:105B7000A87F0023FF2885F8243001D003F0DEFA47
:105B80002823B8F1000F06D003FB07430022274863
:105B90005A77BDE8F883D9F8005003FB0743042285
:105BA000C5F80823C3F82080C5F80881D5F8082176
:105BB00072689AB133681B78C5F81C357368012B7D
:105BC0000ED933685B78C5F81C3528237B43E6582B
:105BD00076B10423C5F804331548DAE7DB7FEBE739
:105BE000F368012BF1D9282303FB0743DB7FEAE7A6
:105BF00007EB870104EBC101D5F80831002BFBD07E
:105C0000C5F808612846D5F8083103F0A4FA002841
:105C1000F2D1282303FB0744A07FFF28DCD003F048
:105C200080FAD9E70348B4E7281600200300AD0B3B
:105C30000000AD0B0B00AD0B02494FF0402003F00C
:105C4000BDBA00BF281600200149024803F0B6BAC9
:105C5000501600200030024010B5144CA82200213C
:105C6000204601F0BFFC03232361114A6361114BFD
:105C7000A261E3614FF4806323620023A362636245
:105C8000E36222660C4A62661022A2662367E3661C
:105C90006367BFF35F8F094A12F8011DE1540133B6
:105CA000102BF9D1BFF35F8F10BD00BF100400208F
:105CB00010AD0000100000200000002029AD000001
:105CC00010B545210446034801F0B8FB204603F017
:105CD000A6FA00BF2AAD0000F7B504460D46EFF363
:105CE0001187202383F31288BFF36F8F1A4A042889
:105CF00098BF1A4B9668127C94BF53F82030184B0B
:105D0000009245210246174801F098FB3DB1EB692E
:105D1000C3F308031BB11448452101F08FFB36B1D2
:105D2000304603F005FB034608B1027802B90F4B79
:105D30000F483246452101F081FB29462046FFF7F6
:105D4000BFFF87F31188BFF36F8F304603B0BDE804
:105D5000F040FBF797BF00BF78160020309C000092
:105D60003EAD000054AD000081AD00004CAD000020
:105D7000A7AD000038B5094B53F82040013053F867
:105D80002050A54200D838BD636823B1204603F0F7
:105D90004EFA0834F5E723689847FAE7449C000078
:105DA00070B52B4B2B4C2C4D012286B003201A7062
:105DB000FFF7E0FFFBF7A8FC03F055FA0420FFF71C
:105DC000D9FF2646AE4204F1300410D300F060FD46
:105DD000204C224EAC4226D300F06EFDFAF7E8FAD2
:105DE0001F4A137B23F00103137306B070BD54F8F0
:105DF0000C3C059354F8103C049354F8143C039362
:105E000054F8183C029354F81C3C019354F8203C7D
:105E1000009354E90A2354E90C0100F01FFB54F8E5
:105E2000303C5E65CDE7D4E90A23B3F1FF3F08BFFC
:105E3000B2F1FF3F05D052EA0301206803D103F01D
:105E400079FA3034C6E73146183000F0FBFEF8E747
:105E5000B62F00201C9800001C98000063940000DE
:105E6000F806002008B50348034A0021121A03F07F
:105E7000F6F908BD68060020B82F002070B5144E52
:105E8000144D1549702386B003FB006601220023E0
:105E9000CDE904230F22CDE902320193142303FB41
:105EA00000554FF4A072044602FB00110B4B009505
:105EB000304600F0D3FA737B2C7423F00403737321
:105EC000074BEE60013403EBC4236B6006B070BD7A
:105ED0008806002078160020B8370020699200005C
:105EE000B82F0020BFB50020FFF744FF294B83F3F4
:105EF0000888294C294E6369294F43F40073636174
:105F00000025E02384F82230E57725766576A576AE
:105F100084F82050636A43F4E023636284F82350DA
:105F2000FBF740FEFBF7BCFF4FF0FF33A362E362D9
:105F30001C4BB36040F201129A815D6603F063F975
:105F40000120FFF717FF0220174CFFF713FF00F0A7
:105F5000D3FC164B74610593012315490095CDE9D7
:105F600003534FF400523B46CDE90155204600F063
:105F700075FA627B064622F004022046627303F043
:105F800015FA2846FFF77AFF3A4631462046FBF7D6
:105F90006BFF00BFB837002000ED00E0781600204E
:105FA000A15D000068070020F80600200EAE00008A
:105FB000F83800202DE9F341044617461E46EFF35A
:105FC0001188202383F31288BFF36F8FC368334A8D
:105FD0007BB180689168884219D057EA060318D1CE
:105FE00088F31188BFF36F8F6FF00F0002B0BDE828
:105FF000F081916891F90E1021610133E36093689B
:10600000A36088F31188BFF36F8F0020EEE721694A
:10601000F2E791F90E1090F90E309942A8BF194697
:106020006FF07E029142B8BF11468B422DDD03F026
:1060300026F90546CDE9007619482246414600F08A
:1060400073FB0028E1D0EFF31186202383F312883D
:10605000BFF36F8FA068D0B1236821699C420AD03A
:106060004BB193F90E309942A8BF19466FF07E03E9
:106070009942B8BF194603F002F940B108483146C9
:1060800000F0C2FB6FF00A00B0E70025D2E7002D58
:10609000F4D186F31188BFF36F8FF3E778160020F1
:1060A000B72F002038B58368044663B3194A926855
:1060B00093422BD1C368012B03D9013BC36000205D
:1060C00038BDEFF31185202383F31288BFF36F8F60
:1060D0000169806803F0D3F8204603F0DCF9A06082
:1060E00058B190F90E2022610022C26603F05EF9D9
:1060F0000948294600F088FBE1E7E06085F3118854
:10610000BFF36F8FDBE76FF01500D9E74FF0FF307B
:10611000D6E700BF78160020B72F002038B5044618
:10612000EFF31185202383F31288BFF36F8F03F001
:10613000B2F948B10022C26603F038F9294608488E
:10614000BDE8384000F060BBD4E902329A4218BF83
:106150000133A36085F31188BFF36F8F38BD00BF93
:10616000B72F002013B5EFF31181202484F3128898
:10617000BFF36F8F846844B1013C846081F3118860
:10618000BFF36F8F002002B010BD52EA030406D1A6
:1061900081F31188BFF36F8F6FF00F00F3E7CDE944
:1061A00000230246014800F0BFFAECE7B72F0020B9
:1061B00070B50446EFF31185202383F31288BFF3F3
:1061C0006F8F6FF00A06204603F065F918B1C666B6
:1061D00003F0ECF8F7E7A06029460248BDE87040FC
:1061E00000F012BBB72F00202DE9F043DFF82C811F
:1061F00085B005464FF0FF364FF0FF37EFF31189BA
:10620000202383F31288BFF36F8F2C6F8CB9022188
:1062100005F1880003F04EF800285DD10023CDE998
:106220000067029305F1780249463D4800F012FCF0
:10623000E4E76A6F23682B67944208BF6B67D5F861
:10624000883043F00203C5F88830E36823F0040384
:1062500043F00103E360636889F31188BFF36F8F34
:1062600020469847EFF31189202383F31288BFF368
:106270006F8FE368D90623F0010237D4E260E36848
:106280009A071AD5D8F8000023F00203E360A0B102
:106290000268002188B143689C4237D1036869BB1A
:1062A000D8F80420C8F80030824201D1C8F8043080
:1062B000002340F8083BFFF731FFD5F8883023F082
:1062C0000203C5F8883089F31188BFF36F8FDB05AF
:1062D00094D400F019FB91E705F18004002201211C
:1062E000204603F015F90028F8D197E723F01103B1
:1062F000E36004F11000FFF711FFC0E70B60D8F86E
:106300000430834208BFC8F80410D1E722B11368F3
:10631000014610461A46BDE71346F9E798160020D5
:10632000B72F0020F8B5C3689A0704460F46C3F399
:1063300040062CD45B071AD40B680BB983680B603A
:10634000E368DD0744BFA3683B603D684CBF02269D
:106350000126002D38D01E4B9B68AB420AD0D5F8E1
:106360008830D807C3F3800214D46FF012060023DC
:106370003B6024E002F0D3FFD5F888300028F0D14C
:10638000D907C3F3C002F0D552B15B0708D46FF050
:106390000F06ECE7002AFAD1C3F3C003002BF6D1B5
:1063A000002323606B6F63B9C5E91C44284602F0E3
:1063B0008CFFE36843F00403E3603B68A36030466E
:1063C000F8BD1C606C67F1E76FF01506CFE700BF02
:1063D000781600200146014802F091BFF80700201E
:1063E000F0B589B004460020C4E91C000E9D04F1FC
:1063F0007800C4E91E0004F18000C4E920004DB318
:106400002879002840F2011008BF0120C4F8880054
:1064100000204FF0FF364FF0FF37CDE90330CDE9D4
:106420000100CDE906670C4B0094204600F040F8CF
:1064300055B1296811B1204602F077FF6B791BB185
:10644000237B43F001032373204609B0BDE8F040ED
:1064500002F070BF0120D9E7E96100007FB50C9E12
:10646000067307320426467300F158050B9E8673A7
:1064700022F00702C0E916558E1800250A9A856099
:10648000C0E90655C5730292099A0192089A0092D2
:1064900032460446FBF7CCFC044B65659B6803B1B0
:1064A0005B6E6366304604B070BD00BF7816002096
:1064B000F0B587B000250595109D04950F9D0395B7
:1064C0000E9D0295DDE912760D9D01950C9D0095BE
:1064D0000446FFF7C3FFB6F1FF3F08BFB7F1FF3F28
:1064E00005D056EA070305D1204600F09FF9204663
:1064F00007B0F0BD03493A46334604F1180000F0F6
:10650000A1FBF4E76394000038B50D4D2B4653F81A
:10651000184F9C4200D004B9EC68AB6838B95A7B7C
:10652000D20604D1A26912B9DA897F2A05D89C4221
:1065300002D0204600F0CEFA23466B6138BD00BF82
:106540007816002008B590F90D20437B002A0146FB
:1065500004DA03F07F03437302F0EEFE044B986805
:10656000431A58425841BDE80840FFF7CDBF00BF6D
:106570007816002070B490F90D30427B002B29DB97
:10658000D30627D183692BBB134962F07F02427384
:106590000A4652F8184F944218BF2346CC6923B9D3
:1065A000C0E900242060C8610CE090F90E5093F916
:1065B0000E60B5420AD0AE4208DD5A68C0E900322A
:1065C0001060586070BC0020FFF79EBF9C42E7D06F
:1065D0001B68E4E770BC7047781600202DE9F04195
:1065E000002A427B0E460CBF1021082111420446AE
:1065F0000FD141EA0203D20918D1437308291BD0F5
:106600000120FFF781FFBFF35F8F637B23F06003FF
:106610006373264B9B68A34241D1EFF30583002BA4
:106620003DD13046BDE8F041FBF742BB03F07F03AC
:10663000437302F081FEE1E7A36813B1204602F044
:1066400083FE04F1180002F085FFA56D04F15807E0
:10665000AF4211D04FF0000875B1284602F074FE29
:1066600005F1180002F076FFC5F86C802846FFF7A8
:1066700081FFA56DAF42EFD10C4DAB689C42BFD1FD
:10668000EFF30583002BBBD00120FFF73DFF084B44
:10669000AB6040F201129A8100225A66B3E786F39A
:1066A0001188BFF36F8FBDE8F08100BF781600201E
:1066B0006807002070B590F90D20437B002A014641
:1066C00004DA03F07F03437302F036FE4B7B154A76
:1066D00063F07F0310464B7350F8183FD469834230
:1066E00008BF002323B9C1E900042160D1610CE097
:1066F00091F90E5093F90E60B5420ED0AE420CDD0A
:106700005868C1E90030016059609068431A5842E6
:10671000BDE870405841FFF7F7BE9C42E3D01B68CC
:10672000E0E700BF78160020F8B5124B0C46114682
:10673000114A98681060DDE90676EFF31182202295
:1067400082F31288BFF36F8F9D68284602F006FE21
:10675000B6F1FF3F08BFB7F1FF3F06D007493A4601
:10676000334605F1180000F06DFA2046BDE8F84008
:10677000FBF79EBA78160020A01600206394000054
:10678000F8B50446EFF31186202383F31288BFF394
:106790006F8F437BDA0649B219D18569BDB903F021
:1067A0007F03437302F0C8FD437B164A817363F095
:1067B0007F034373134653F8180F984218BF0546DA
:1067C000D0695DB9C4E900300460D46111E0A173FF
:1067D000002086F31188BFF36F8FF8BD95F90E7016
:1067E000B9420BD08F4209DD6B68C4E900531C60CD
:1067F0006C600120FFF788FE0120EAE7A842E1D0A3
:106800002D68DEE77816002049B9EFF3058030B92E
:10681000054B5A699B689A4201D0FBF749BA81F34C
:106820001188BFF36F8F70477816002010B5EFF313
:106830001184202282F31288BFF36F8F427B5107AD
:1068400004D484F31188BFF36F8F10BD22F00402CB
:106850004273FFF78FFE21460248BDE81040FFF764
:10686000D3BF00BFB72F0020034648B9EFF305821E
:1068700032B9064A51699268914201D0FBF718BAC1
:1068800083F31188BFF36F8F704700BF7816002025
:10689000EFF31181202383F31288BFF36F8F054B31
:1068A0009A68D37B013BD37381F31188BFF36F8F59
:1068B000704700BF7816002038B5EFF3118520240B
:1068C00084F31288BFF36F8F0A4B9A68D37B01332E
:1068D000D3730020FFF718FE85F31188BFF36F8F85
:1068E000EFF3118084F31288BFF36F8FBDE8384057
:1068F000FFF7BABF78160020024B03F11802C3E974
:106900000622704778160020F8B5EFF31185202392
:1069100083F31288BFF36F8F19498868437B03F0B4
:106920007F03437302F008FD8B685A7B084662F0D0
:106930007F025A7350F8182FCC69824208BF002298
:1069400022B9C3E900042360CB610CE093F90E6027
:1069500092F90E70BE420ED0B7420CDD5168C3E909
:1069600000210B6053600120FFF7CEFD2846BDE8F3
:10697000F840FBF79DB9A242E3D01268E0E700BF00
:106980007816002050EA01032DE9F04105460E4635
:1069900003D1FFF7B9FF00202BE0831C71F1FF3317
:1069A00029DB02F0ECFD2C18EFF31188202383F390
:1069B0001288BFF36F8F124F124BB8681860FFF741
:1069C000C1FDB86810492A463346183000F03AF93C
:1069D000BA68537B43F0100353734046FBF768F9E2
:1069E00002F0CDFD201A63EB0303012873F10003CD
:1069F000D1DBBDE8F0816FF00104241AD4E700BFB9
:106A000078160020A016002063940000B1F1FF3F2B
:106A100008BFB0F1FF3F08B506D10A4B986802F0F5
:106A2000D4FC4FF0FF3008BDFFF7ACFF4FF47A7194
:106A300047F6FF730022C0FB0132D80B40EA424008
:106A4000F1E700BF78160020014B9868704700BF3F
:106A500078160020D3B5DDE90667089CCDE900670C
:106A6000FFF762FE1CB1034B9B685B69236002B0B9
:106A7000D0BD00BF78160020044BC01A044BC010D4
:106A80005843044B01221A54704700BFD807002016
:106A9000ABAAAAAAB72F0020C3897F2B12D80A4B12
:106AA0001B6863B1094B90F90E201B689A4209DB01
:106AB000437BDB0606D1064BC31A18BF012303F044
:106AC000010070470023FAE7A8160020A416002052
:106AD0008806002070B50E4B0E4C1E7C06EB46035C
:106AE00004EBC3040546204602F034FD0A4B0022A5
:106AF00028469A55FFF7D0FF48B1084B08491A6855
:106B0000013A2046D317BDE8704000F09BB870BD35
:106B100078160020D8070020B72F0020A8160020E4
:106B2000796A000038B5EFF31185202383F31288CA
:106B3000BFF36F8F104B114A9C681068A04206D1BA
:106B4000FFF7C8FF85F31188BFF36F8F38BD0021B1
:106B50001B7C11600A4AD35C002BF3D02046FFF760
:106B60009BFF0028EED0637BDB0602D12046FFF7B7
:106B7000A1FD2046E4E700BF78160020A016002003
:106B8000B72F002008B50648064A0749121A02F036
:106B900068FBBDE80840054A0549064802F061BBAC
:106BA000B80400206806002020AE000000000000AD
:106BB00020AE0000B8040020034B1B680BB9FDF7A2
:106BC0004BB80020704700BFAC16002030B570B144
:106BD0000B4B5B6898420AD0036843B1D3E90421A8
:106BE000D0E90445121941EB0501C3E90421D0E9BC
:106BF000003213605A600023C0E9003330BD00BF8B
:106C00001406002010B50E4B1C689C4204D1FFF7FF
:106C1000D3FF6FF0004010BDFFF7CEFF002CF8D07F
:106C2000D4E904321B1A62EBE072B3F1004F72F147
:106C30000001EEDA002AACBF18460020EBE700BFE7
:106C400014060020B3F1FF3F08BFB2F1FF3FF8B5D3
:106C500004461D4616465ED08160EFF3118720235F
:106C600083F31288BFF36F8F013275F1FF3324DA9B
:106C70002E49D1E900206FF001039B1A4FF0FF323B
:106C800062EB00009E1B60EB0500012E70F100031B
:106C900001DA01260020C4E90460254ED6F800C0C0
:106CA0007568B44508BF4FF0000CBCF1000F0DD162
:106CB000C4E900652C6074601CE0FFF77DFF0136BD
:106CC00045F10005361845EBE070E4E7DCE9042007
:106CD000D4E90431934271EB000E1DDAD21ADCF8CC
:106CE000043060EB0100CCE90420C4E900C31C605F
:106CF000CCF804403368B34209D09C4207D10D4B15
:106D00001C6824B9FFF77EFF2146FCF777FF87F365
:106D10001188BFF36F8FF8BD9B1A61EB0001AC4582
:106D2000C4E90431C4D0DCF800C0BEE7F00700209D
:106D300014060020AC1600202DE9F84FEFF3118C5B
:106D4000202383F31288BFF36F8FDFF8B0A0DFF842
:106D5000B0902C4FC9F80000DAF80000002450452C
:106D600008BF00200025D7E90021D9F80030E0460F
:106D700078B3D0E9046C4FEAE37EB3427EEB0C0BB0
:106D800005DAF61A6CEB0E04C0E9046421E0B218CF
:106D900041EBE671C0E90445C7E90021FFF716FFA2
:106DA00088F31188BFF36F8F83689847EFF31188DA
:106DB000202383F31288BFF36F8FD9F80030DAF8FD
:106DC00000009B1B5045C446C9F80030CBD1D7E921
:106DD00000219A1841EBE3730024C7E90023C9F8A6
:106DE0000040FFF70FFF2146FCF708FF88F31188EA
:106DF000BFF36F8FBDE8F84FFFF794BE1406002075
:106E0000AC160020F007002010B5EFF3118420230A
:106E100083F31288BFF36F8FFFF7CEFE054A034658
:106E2000D2E90001181841EBE37184F31188BFF334
:106E30006F8F10BDF0070020F8B50446EFF31187FF
:106E4000202383F31288BFF36F8F026822B187F388
:106E50001188BFF36F8FF8BDD0E90A36581C46F190
:106E60000001022871F1000127D3012B76F1000106
:106E7000BCBF012316465D1E46F1FF3602F083FBC0
:106E8000013041F10001401946EB0101012871F187
:106E9000000139DB02F077FB013041F100016FF0B6
:106EA0000102401946EB0103121A4FF0FF3161EB6A
:106EB000030318492046FFF7C5FE236B0133236304
:106EC000236A6BB187F31188BFF36F8F236A204663
:106ED0009847EFF31187202383F31288BFF36F8F56
:106EE00054F8185FA542B2D0002DB0D0284602F069
:106EF00086FA0023EB6687F31188BFF36F8F28466D
:106F0000BDE8F84002F052BA6FF001024FF0FF33D3
:106F1000CFE700BF396E00002DE9F04105461C4661
:106F200090461F46EFF31186202383F31288BFF3A8
:106F30006F8FB4F1FF3F08BFB2F1FF3F05D186F379
:106F40001188BFF36F8FBDE8F081531C74F1FF33DC
:106F500009DB012A74F10003BCBF0122002412F1F5
:106F6000FF3844F1FF37284602F0F4FADDE9060164
:106F70000023C5E90A012B63034942463B462846E4
:106F8000FFF760FEDBE700BF396E00001FB5094A5E
:106F900092E8030002AB83E803004FF480620093A1
:106FA000054906484FF0FF33FFF71AFA002005B0F5
:106FB0005DF804FB80980000F8580020F8070020D6
:106FC0007047002070472DE9F7430E461746994653
:106FD000044628B94FF0FF38404603B0BDE8F083BF
:106FE0000029F7D0002AF5D0CB680D891D44042371
:106FF0000DEB03022946384600F02EFA80460028A1
:10700000E8D1BDF80410738946F60812914225D1E3
:10701000BDF806109942DDD104230DEB030229448B
:10702000384600F019FA0028D4D1BDF8042046F6FD
:1070300007139A42CED1C4E900679DF82830A4F81E
:107040000890A3727389BDF806202B44E36073890E
:1070500013442B44043563612561BDE7002BE4D064
:10706000B8E72DE9F3410E4617461D46044620B900
:107070004FF0FF3002B0BDE8F0810368002BF7D07D
:107080004368002BF4D04FF6FF78D4E904239A42EA
:1070900016D223685B8923B1E368934204BF0433AB
:1070A00023610423216960680DEB030200F0D4F929
:1070B0000028DDD1A37A2BB1D4E903329A4201D35F
:1070C0000120D7E72389BDF80610434501F10402EA
:1070D00003D0BDF804C09C450BD115B1BDF80430F8
:1070E0002B8023690433336039802369134423617F
:1070F000C0E7236913442361C7E748B103683BB184
:1071000043682BB1C068884294BF002001207047BB
:107110004FF0FF30704700F04ABA4FF4C073584345
:107120003030704700F075BE08B502F02CFA4FF40D
:107130007A72A0FB020302FB0133C00B40EA43401A
:1071400008BD70B513460E4615460021024604469A
:1071500000F044F850B92B4604F12C0201212046DE
:1071600000F03CF810B1002E08BF002070BD37B50C
:107170000446426A802501A903200195FAF794FA92
:1071800058B9019B226DA36201A906200195FAF767
:107190008BFA054628B1092500E00125284603B0F1
:1071A00030BD019B206A636500F098F9E065F5E762
:1071B0000123036003F1012343600023C0E902338C
:1071C00070474379012B07D10368012B04D1007963
:1071D000431E5842584170470020704713B50020A5
:1071E0001446F9F757F901A9C0B2FAF735FA014682
:1071F00068B922462023019800F02EF90446019830
:1072000000F029F9201E18BF012002B010BD012096
:10721000FBE7002070470FB407B504A951F8040B31
:107220000191F9F7DBFE03B05DF804EB04B07047A1
:10723000044608B5084611461A46A047FFF704FC65
:10724000FAF720FD038B13F0070305D10368002B29
:107250000CBF002003207047022B05D1408BB0FAF1
:1072600080F0400980007047012B05D10368002B96
:107270000CBF0020052070470020704710B50C4659
:1072800000B111B96FF0150010BD081D00F0B7F87E
:107290000028F9D1A368032BF6D9F3E72DE9F041D3
:1072A0000D4607461946281D90461E4600F0B8F8C0
:1072B000044638B13346424629463846A446BDE81E
:1072C000F0416047BDE8F08110B4EFF31182202453
:1072D00084F31288BFF36F8F416110BC0121FAF76C
:1072E000ADB838B50C46054658B151B10B6843B13D
:1072F0004B6833B11C22002100F074F92C6100208E
:1073000038BD6FF01500FBE770B505460E46FFF778
:10731000B5FF041E14DBEFF31182202383F31288E0
:10732000BFF36F8F6B8B2C8B4FF6FF718B4204F08A
:10733000070407D182F31188BFF36F8F6FF00A043F
:10734000204670BD022C0CD101336B8382F311886F
:10735000BFF36F8F0023224631462846FFF79EFF7A
:10736000EEE7062C14D8DFE804F004131313041A14
:107370000400002333606B683BB9C5E90066ACB913
:1073800002212846FAF75AF8DAE71E606E60F6E73F
:1073900082F31188BFF36F8F6FF00404D0E782F39C
:1073A0001188BFF36F8F6FF08504C9E782F31188EE
:1073B000BFF36F8FC4E710B5EFF31182202383F37F
:1073C0001288BFF36F8F048B04F00704022C0AD0DD
:1073D000012C0CBF6FF004006FF0850082F3118860
:1073E000BFF36F8F08E0438B013B9BB2438323B90C
:1073F0002146FAF723F8204610BD2046EEE7034663
:1074000058B1426802F00302012A03D0032A04D1D2
:10741000026812B10020986070476FF01500704745
:107420004268816002F00302032A4FF00002034623
:107430000CBF006810465A60704770470FB407B51C
:1074400004A951F8040B0191F9F7C8FD03B05DF8E8
:1074500004EB04B070477047002930B40446184666
:107460000BDBA5680844A84207D8E068646821449B
:1074700084682468A44630BC60476FF0150030BCB7
:107480007047002930B4044618460BDBA568084451
:10749000A84207D8E0686468214484686468A44608
:1074A00030BC60476FF0150030BC704700290346C0
:1074B00010B410460BDB9C680844A04207D8D8687B
:1074C0005B68194483689B682BB110BC18476FF048
:1074D000150010BC70476FF05700FAE708B5C06898
:1074E0008368DB689847006808BD08B5C068836892
:1074F000DB689847407908BD70B54C680368A342C3
:1075000001D2012070BD8A682244934201D3002039
:10751000F8E7D1E903254E69B54203D36FF00B03B9
:107520008B61F4E71B1B42F835304368086902EBB6
:10753000C00253600B6901330B61E2E7014600684A
:10754000FAF7F4B808B5FAF729F9BDE80840FAF7F0
:1075500029B900210120FAF7E9B861B662B680F3D3
:107560001188BFF36F8F704772B6002383F31188C1
:10757000BFF36F8FBFF34F8F30BF62B6BFF36F8F14
:10758000704772B6002383F31188BFF36F8FBFF388
:107590004F8F20BF80F31188BFF36F8F62B67047A3
:1075A000034600201A5C02B970470130FAE710B5B3
:1075B0005AB10139841810F8012B11F8013FA0428B
:1075C00001D09A42F7D0D01A10BD1046FCE710B592
:1075D000431E0A44914200D110BD11F8014B03F83B
:1075E000014FF7E7C9B202440346934200D1704706
:1075F00003F8011BF9E74FF0FF3070470369C9B288
:107600000C2201FB0233186C00F00700704770B5C4
:10761000C9B20369EFF31185202484F31288BFF304
:107620006F8F0C2606FB0134246C14F0C00408D0C4
:10763000A24206D085F31188BFF36F8F4FF0FF3061
:1076400070BD71430B4401221A6485F31188BFF3A6
:107650006F8F43680B445B6898470020F0E78022F7
:10766000FFF7D5BFF8B5069F0469C9B2EFF31186DD
:10767000202585F31288BFF36F8F0C2569430C44D6
:10768000256C05F0070CBCF1010F0BD1276486F3C4
:107690001188BFF36F8FC4E90E2343685B58984786
:1076A0000020F8BD05F0C005AF4286F31188BFF396
:1076B0006F8F0CBF6FF077004FF0FF30F1E713B51D
:1076C00080240094FFF7CEFF02B010BD10B4006913
:1076D000CBB21C2403FB0400002110BC1047104651
:1076E000FEF71CBD08B5FAF755FEBDE808400020BE
:1076F00001F086BCFAF79EBD036924330B600123B9
:1077000013607047FEF70ABD4FF0FF324FF0FF33B2
:10771000FEF728BDF0B58BB044680769119ECDF81F
:1077200018D0002000908DF80400012007901098D8
:107730008DF80010D107CDE9080602F080050DD5BF
:1077400012F0040F1BBA1ED00493042204A90DF1F9
:107750000100FFF73CFF079B04330793002E06ABA5
:107760000CBF01220222CDE903230293214602230A
:10777000059351F8040BA5B183681C68002302AA85
:10778000A0470BB0F0BD3A7D0493D307DDD40322AC
:107790000DF111010DF10100FFF719FF079B0333F4
:1077A000DBE783681C6804ABE9E773B500230D1EB3
:1077B000466818BF0421CDE9003308BF06218022A6
:1077C0000446FFF7A7FF96F82030DB0609D540B93D
:1077D0003DB9CDE900000346802298212046FFF7FD
:1077E00099FF02B070BD1FB5012301930DF10F0386
:1077F000009300231A460521FFF78CFF08B99DF876
:107800000F0005B05DF804FB2DE9FF410646154663
:107810001C4601270DF10F080023CDE900871A4609
:1078200005213046FFF776FF40B99DF80F30DB07A2
:1078300004D528462146FFF7E9F8EDE704B0BDE896
:10784000F0812DE9F347054600690F1ED0F820901E
:1078500016467DDBBB184B457AD847EA0204C4F3D1
:107860000B04002C74D1FFF74FFF21462846FFF789
:107870009CFF4FF0FF3A0446002E46D101212846D6
:10788000FFF793FF002C08BF04462869FFF73AFF73
:10789000204602B0BDE8F0872869A04600F1150334
:1078A0001D305A7882B10AFA02F137EA01010BD190
:1078B00001219140B14207D8B8F1000F1CD098F8CF
:1078C0000110914238BF984602339842E9D1B8F18D
:1078D000000F13D0002398F800108122CDE9003367
:1078E00028463B46FFF716FF98F8012001239340F6
:1078F00004461F44F61A21E09846E5E76FF01504A8
:1079000001212846FFF751FFBFE7002CF8D1CDE950
:1079100000442346802206212846FFF7FBFE04464A
:107920000028EDD1B145B7D1CDE900000346802252
:10793000C7212846FFF7EEFE00260446002CDFD1C3
:1079400040F2676200232846FFF75EFF044693E794
:107950006FF015049CE72DE9F74F054600690E1EF0
:107960001F46B0F81E80036A91464EDBF2199A4218
:107970004BD8FFF7C9FE00212846FFF716FF044643
:10798000C0BB82462FB901212846FFF70EFF0446EF
:1079900034E0B845C34628BFBB4606EB0B0396FB55
:1079A000F8F2013BB3FBF8F393421CBF08FB1262F1
:1079B000A8EB020BCDE900AA00238022062128466D
:1079C000FFF7A8FE0446A8B9CDE9009B3346812203
:1079D00002212846FFF79EFE044658B901220023E3
:1079E0002846FFF711FFA7EB0B07D9445E44044676
:1079F0000028C7D001212846FFF7D7FE2869FFF7E6
:107A000081FE204603B0BDE8F08F6FF01504F8E763
:107A1000F7B5054600690C1E1E461746036A13DBC0
:107A2000A2199A4210D8FFF76FFE2346CDE90076DF
:107A3000012203212846FFF76DFE04462869FFF75F
:107A400061FE204603B0F0BD6FF01504F9E7F7B50D
:107A5000446894F82030DA07054644D5076901F0F8
:107A600092FD4FF47A76A0FB063206FB0122DB0B77
:107A700043EA42433A699B1A13D4628BA68B9B1A42
:107A8000B3420EDAF61A4FF4004740F2E730002115
:107A90004FF47A720023E6FB0701F8F71FFBFEF7AD
:107AA000B5FF94F8203013F002031CD1CDE9003368
:107AB0008022AB212846FFF72DFEA8B994F820308C
:107AC000DB0710D5E48B40F2E7314FF400450E465A
:107AD0000146E5FB04614FF47A7200233046F8F763
:107AE000FDFAFEF793FF002003B0F0BD38B5054660
:107AF0000C4601F0FEFA002D07DBA84205D9401B19
:107B000084428CBF0020012038BD0020FCE72DE915
:107B1000F047836886B01B698846914601A902AA8E
:107B200098470024A2462546029BAB4202D806B0E5
:107B3000BDE8F087019F07EBC50700267B6804932B
:107B40003A68B2420AEB060302D801359A46EBE7DF
:107B500003940593494603A8C0470028E7D0049B37
:107B600001361C44ECE74B1E5B0800EB8300C907A1
:107B7000C36958BF1B0CC3F3072113F0FF031DBFDC
:107B80000020117053706FF01500704743685B68F8
:107B9000D3F810350B600020704743685B6802EA39
:107BA000010021EA0201C3F80805C3F80C15002002
:107BB000704743685B680020C3F808157047436846
:107BC0005B680020C3F80C15704743685A68D2F808
:107BD000043521EA03000B40C2F80805C2F80C3551
:107BE0000020704710B503695868F8B1884219D170
:107BF0009C6808685860A14200D198600020086025
:107C00002AB15A680A609A68596002B999600020DE
:107C100010E0814206D10868206098688142EDD169
:107C20009C60EBE7044600680028F2D1002AE8D106
:107C30006FF0150010BD4FF08043D3F8002402F020
:107C40000103910748BF43F01003110748BF43F4F5
:107C50008073D10348BF43F08003510348BF43F012
:107C60002003510748BF43F00203910348BF43F08C
:107C70008003120348BF43F0800303600020704775
:107C800030B543681360057A446804EBC504A34229
:107C900002D36FF0010030BD5C798C4201D0083313
:107CA000F0E70020F7E743681B68D3F88004C3F8C7
:107CB0008004704742681368D3F8100150B1D2694C
:107CC000002012780A70C3F81001D3F810210122A5
:107CD0001A6070474FF0FF30704702680346D2F8D1
:107CE000580140B95B68DB0706D4D2F820010038A0
:107CF00018BF012070470120704743681B68D3F804
:107D00000423D20517D5D3F82021A2B1EFF31182B5
:107D1000202181F31288BFF36F8FD3F8201131B186
:107D20000021C3F82011D3F820110121D96082F37A
:107D30001188BFF36F8FD3F85831704700220121AB
:107D40000420FAF741B8002201212320FAF73CB8B9
:107D500010B50B6813B91360184605E003685C683A
:107D60001CB114600368186810BD083303600B6809
:107D7000013B0B60EDE703460A46006819790123D1
:107D800003FA01F103691B68194218BF82F001026E
:107D900012B18368DB68184783681B69FBE710B57D
:107DA000036804464BB19A683AB1186901F027FAA2
:107DB000206800210830FFF7DEFFA36933B9636054
:107DC00004F11000BDE81040FEF7A8B910BD10B5D1
:107DD000006903688B4206D190F85C4034B9FFF724
:107DE000DEFF204610BD6FF01500FBE76FF00F00BF
:107DF000F8E700F150039B009BB203F1804303F5C9
:107E0000883300221A601B68704708B5FBF78AFDAB
:107E100008BD8068183820F0070010387047042823
:107E200009D0052803D1481E18BF01207047431A06
:107E30005842584170470120704738B515460C46E6
:107E400061B15AB1FFF751FB2544214611F8013BBE
:107E5000834203D1A942F9D1012038BD0020FCE7BB
:107E600038B50C460123114622460546FFF7F4FAC1
:107E700000280FDB012221462846FFF7DEFF38B934
:107E80002378012B14BF022301232370002038BD67
:107E90000323FAE70120FAE78268183A22F0070282
:107EA000FFF7DEBF13B50C46C0B201A9F9F7D4FB4A
:107EB00050B921460198FBF711FF04460198FFF7DE
:107EC000CAFA204602B010BD0124FAE770B5046872
:107ED0000D1B002D02DC6FF05F0070BD94F9006097
:107EE0002378002E0ADB631C036023781360036889
:107EF000C91A13688B42EED80020EEE703F07F0327
:107F00005C1E032C13D89D42E5DD00241460046838
:107F10000134046004681568247844EA0524146078
:107F20000468013B04F101040460F3D1DFE76FF062
:107F30006300D2E770B404680E1B002E07DD2678BC
:107F40009E4208D10134046070BCFFF7BFBF6FF0E0
:107F50005F0070BC70476FF06100FAE773B50223F1
:107F6000154601AA0446FFF7E5FF40B9019E2168C6
:107F70003246284600F0A6FB23683344236002B053
:107F800070BD0139002901DA0020704750F8213016
:107F9000002BF6D0B3FA83F00131C0EB41107047EB
:107FA00039B101F18041013900EB81018142034681
:107FB00000D270471B680A681BBA12BA40F8042B3B
:107FC00041F80439F2E72DE9F0411C4613F00303B0
:107FD00018BF012303EB94038B4206460D469046DF
:107FE00013D879B18F003A460021FFF7FBFA2CB184
:107FF000381B224641463044FFF7E9FA294630460D
:10800000FFF7CEFF0020BDE8F0816FF00700FAE730
:10801000B3EB810F70B504464FEA8105104619D9BC
:108020005A1B86180021FFF7DDFA30462B46C2188E
:1080300000218B4210D1002070BD22F0030102F01C
:1080400003066158F600F140C9B281B90132AA4273
:10805000F3D1ECE71A46FAE721F0030001F003053B
:108060002058ED00E84002F8010D0131E1E76FF022
:108070000700E1E753098B42F0B402F01F0401D876
:1080800009D124B18A00F0BC0021FFF7ABBA1F2A46
:1080900003D8F0BC70471F2A0AD900EB8302051FE2
:1080A00000EB8106B24216D1CB1A00228B4217D3C5
:1080B000002CEED000EB81010022C4F120068142A9
:1080C000E7D051F8045C25FA04F3134341F8043D6A
:1080D00005FA06F2F3E752F8047B45F8047FE1E77E
:1080E00040F823200133E1E71F2AF0B54FEA52148C
:1080F00002F01F0512D96FF0030606FB04060B46BB
:108100009C4203F1FF3212D3631A8C4288BF0023D2
:108110000B4400EB8303002283420ED135B100EB08
:1081200084000022C5F120078C4209D3F0BD56F827
:10813000223040F822301346E2E743F8042DEBE703
:10814000066806FA05F3134340F8043B013426FAA7
:1081500007F2E9E7F0B50024844620469C4200D1AE
:10816000F0BD51F8245052F824702E182CBF012570
:108170000025BF194CF8247045F100000134EDE7EB
:10818000F0B50024064620469C4200D1F0BD51F8CF
:1081900024C052F82470ACEB0005AF4294BF4FF0FE
:1081A000000E4FF0010EED1B46F8245084452CBF05
:1081B00070460EF101000134E6E78B422DE9F047ED
:1081C00028BF0B469646DE08089A0446C91A03F0F3
:1081D000070875460346B44600200CF1FF3CBCF18D
:1081E000FF3F03F1200305F1200511D104EB4614F4
:1081F0000EEB46164FEA880C06EB880E25467645B0
:1082000040F081806444013980F08B80BDE8F087C4
:1082100055F8207CA2FB079710EB090953F8200CB6
:1082200047F1000710EB090043F8200C55F81C0C2F
:1082300047F10007A2FB00093F1853F81C0C49F155
:108240000009C01943F81C0C55F8180C49F1000935
:10825000A2FB000719EB000953F8180C47F10007BF
:1082600010EB090043F8180C55F8140C47F10007FF
:10827000A2FB00093F1853F8140C49F10009C0197A
:1082800043F8140C55F8100C49F10009A2FB000743
:1082900019EB000953F8100C47F1000710EB090027
:1082A00043F8100C55F80C0C47F10007A2FB00092D
:1082B0003F1853F80C0C49F10009C01943F80C0C95
:1082C00055F8080C49F10009A2FB000719EB000959
:1082D00053F8080C47F1000710EB090043F8080CAD
:1082E00055F8040C47F10007A2FB000A17EB000940
:1082F00053F8047C4AF1000017EB090740F1000035
:1083000043F8047C69E756F8043BA2FB0337C31823
:10831000286847F10007C31845F8043B47F10000FF
:108320006DE723681B1844F8043B2CBF0120002094
:1083300069E70168881C400000F008000844032336
:1083400000FB01F2C2F10202013B02FB00F0F7D197
:10835000404270472DE9F04F87B091460493109B3F
:108360000293DDE91183139D05934FEAC80283460A
:108370008A46043200212846FFF734F908F1020347
:108380002E4600240393444515D105EB8401234672
:10839000029A51F824505846FFF7F2FE6840FBF766
:1083A00073FDA6000A4600235946109607B0BDE8A3
:1083B000F04FFCF705B85AF82430D9F80020376898
:1083C0000399009302FB0377059A049B57433046B9
:1083D0004A46FFF7F2FE3046DDE9022100974346A8
:1083E000FFF7EBFE04360134CDE738B50D46012129
:1083F000044600F031F988B9E9882046890100F087
:108400007DF958B92A462146204600F02FFB28B9AD
:10841000E9882046BDE8384000F0B8B838BD4901C9
:10842000502934BF012203220123934003335843D0
:108430000130704710B586B00B9C04940A9C0394DD
:1084400000240294099C0194089C0094FBF740FDD1
:1084500006B010BD10B586B00B9C04940A9C039422
:108460004FF02A340294099C0194089C0094FBF775
:108470002FFD06B010BD30B50546104600229A42C9
:1084800000D130BD51F82240241A45F8224034BFB3
:10849000012000200132F2E7034600EB81010020B9
:1084A0008B4201D1FBF7F0BC53F8042B1043F7E7E4
:1084B0001FB5089C0394069C0092CDE90134079AED
:1084C000FFF748FF04B010BD30B587B01C460B9DC8
:1084D00003950A9D00920123CDE9014505AA059364
:1084E000FFF738FF07B030BD00220123C0E90023A9
:1084F000704710B5044648B1006818B1E18889009A
:1085000000F0DDFB00220123C4E9002310BD42F28C
:108510001073994270B504460D4602D96FF00F00F2
:1085200070BDC3888B4201D30020F9E7042128469F
:10853000FCF732F906460028F0D0216841B1E28804
:108540009200FFF744F8E1882068890000F0B7FB4B
:10855000E5802660E8E738B504460D4619B9FFF70F
:10856000C8FF002038BDC2888A4207D10068920047
:108570000021FFF737F80123A380F2E7FFF7B9FFE7
:1085800029462046BDE83840FFF7C1BF42F21073CC
:10859000994270B50A46054602D96FF00F0070BDCA
:1085A000C3888B4207D8BDE87040FFF7B0BF296889
:1085B00051F8231011B9013B002BF8D15C1C9442F7
:1085C00038BF144604212046FCF7E6F8064600288A
:1085D000E3D0296839B1A200FEF7F9FFE9882868DD
:1085E000890000F06CFBEC802E600020D7E7884209
:1085F00070B505460E4609D0C988C28841B92AB16E
:108600000123838092000068FEF7ECFF002070BD1C
:108610004C1E8CB90134B6F90430AB80A24212D2A0
:1086200021462846FFF773FF0028F0D131682868FB
:10863000A200FEF7CCFFE9E7336853F82430002BA3
:10864000E8D1013CE5E72868121B9200002100EB0D
:108650008400FEF7C7FFE9E770B50C460121054627
:10866000FFF755FF064688B9EA8801469200286858
:10867000FEF7B8FF84EAE472A2EBE472E40FC4EB05
:10868000C4342B68640001341A60AC80304670BD7D
:10869000C388B1EB431F3FBF03684A0901F01F01C4
:1086A00053F822003ABFC84000F001000020704794
:1086B000C1880068FFF765BC08B5FFF7F9FF073010
:1086C000C00808BD70B50E4612F0030118BF0121A5
:1086D00001EB920105461446FFF73DFF38B9E988E2
:1086E000286823463246BDE87040FFF76CBC70BD79
:1086F00013460A46C1880068FFF78ABC38B50446AD
:108700000D46FFF7D5FFE3882844B0EB431F06D89A
:108710002068E1882A46FFF7E7FC002038BD10F00A
:108720001F0118BF012101EB50112046FFF7EFFE9A
:108730000028EDD0F2E708B50A46C18811B10068FB
:10874000FFF798FC002008BD10B5C38823B9CA887C
:108750005AB9ABB1012017E0026802EB830252F86C
:10876000042C002AF3D1013BF0E70C6804EB8204EF
:1087700054F8044C0CB9013AEAE79342EAD80FD313
:10878000013B5A1C01D1002010BD026852F8234061
:108790000A6852F823209442DCD803F1FF33F0D268
:1087A0004FF0FF30F0E730B5C38823B9CA885AB913
:1087B000002B3DD136E0026802EB830252F8042C14
:1087C000002AF3D1013BF0E70C6804EB820555F871
:1087D000045C4DBB013AEAE7B1F9045003D2B1F9A8
:1087E0000400404226E0B0F90420002A03DD002DF9
:1087F0000CDA01201EE0002D08DD3AB14FF0FF3009
:1088000018E003F1FF330BD2504213E0013B016843
:1088100051F8235054F823108D42F2D9104609E044
:10882000591CF4D1002005E0002BD8D09342D3D9B5
:10883000B0F9040030BD1FB581EAE173A3EBE17329
:10884000C90FC1EBC1314900019301310123ADF8DA
:108850000C10ADF80E3002A901AB0293FFF7A3FF95
:1088600005B05DF804FB90422DE9F04105460F4646
:10887000144602D0884206D127460123AB80FC88EB
:108880003CB9002003E0FFF7B2FE0028F4D0BDE8B9
:10889000F0813B6803EB84034FEA840853F8043CFF
:1088A0000BB9013CECE721462846FFF730FE0028D3
:1088B000EDD12E683A68234631463046FFF74AFC30
:1088C00006EB08030746002FDBD0EA88A24204F13A
:1088D000010608D831462846FFF719FE0028D6D1F0
:1088E0002B6803EB84031A68D21943F8042B2CBFBE
:1088F000012700273446E6E72DE9F041D4880546F4
:108900000E4690463CB9F188A1420ED26FF009079D
:108910003846BDE8F081D8F8003003EB840353F803
:10892000043C002BEFD1013CECE72846FFF7EFFDBC
:1089300007460028ECD1F28894420BD2AE4209D00F
:1089400031682868121B920001EB840100EB84005F
:10895000FEF73DFEEA88F088824207D92B68121A9A
:108960009200002103EB8000FEF73CFED8F80020C7
:10897000316828682346FFF703FC024610B901233B
:10898000AB80C5E72968EB8801EB84011B1B084617
:10899000FFF771FD0028F2D0B8E72DE9F843B1F9EF
:1089A0000440B2F804C01CFB04FC664673438146D5
:1089B0000D4617461CD511462846FFF7C5FEB0F1F7
:1089C00000080DDB3A4629464846FFF795FF98B95F
:1089D000B8F1000F08BF0124A9F8044000200BE003
:1089E0002A464846FFF788FF30B9644224B2F3E7CD
:1089F000FFF739FF0028EFD0BDE8F8830123FFF728
:108A0000CCBF4FF0FF33FFF7C8BF2DE9F341CF884C
:108A10000546884616463FB1D8F8003003EB870379
:108A200053F8043C3BB146B90021284602B0BDE8EA
:108A3000F041FFF711BE013FEDE7791C2846FFF733
:108A400066FD044670B941462846FFF7D0FD04464E
:108A500040B9013E0096D8F80020E98828683B46D6
:108A6000FFF7ABFB204602B0BDE8F08170B50446CD
:108A70000D46104600211646FFF7DDFE002824DBD8
:108A80002A46334621460020FBF700FB054638B155
:108A9000284670BD324621462046FFF7AFFF90B909
:108AA00000212046FFF7C7FE0028F3DB31462046B1
:108AB000FFF779FE0028EBDB324621462046FFF720
:108AC000A0FF0028F2D00546E2E76FF00905DFE7D6
:108AD0002DE9F04F89B0DDE9125806468B4628464D
:108AE000002191460593FFF7A6FE002805DC6FF0F4
:108AF0000304204609B0BDE8F08F2B681B68D90736
:108B0000F5D500214846FFF796FE0028EFDB4846E2
:108B1000FFF7CEFDB0F5006FE9D82846FFF7C8FD96
:108B2000B0F5006FE3D8B9F8061031B9012130462D
:108B300009B0BDE8F04FFFF78FBDE888FFF76FFC85
:108B400004218246FBF728FE0746002800F0AA8091
:108B500000220123CDE906234FEA8A0AB8F1000F6B
:108B60000DD1294606A8FFF740FC044600B3514644
:108B7000384600F0A4F806A8FFF7BBFCB9E7D8F820
:108B80000030002B6ED106AB18462946FFF72DFCAE
:108B900006AB044640B15146384600F090F8D8F88C
:108BA0000030002BA5D1E6E793E8030088E8030036
:108BB00059463046FFF71BFD0446002867D10123C4
:108BC000B38029463046FFF7EEFD002857DAE988E2
:108BD0003046FFF79CFC0446002858D12868FFF770
:108BE000A8FB069B0090029701933168EB882A68E6
:108BF00004900846FFF75CFC059B0698B9F8062030
:108C00003168B3F12A3FEB880192CDE90207D9F828
:108C1000002000922A68084641D1FFF71BFC049B04
:108C2000019700933168EB882A680846FFF74CFCEF
:108C3000BBF904B0BBF1FF3F29D1D9F800301B6864
:108C4000DB0724D5F1883068FFF726FC012259465E
:108C5000FBF70EFA3246B08029463046FFF7CEFECB
:108C6000044614E0E9884046FFF751FC044600281A
:108C700091D198E8030008AB03E9030098E72A467E
:108C800031463046FFF7F2FE044600289FD0514699
:108C9000384600F014F8B8F1000F80D16BE7FFF709
:108CA000C9FBBCE76FF00F0423E713B5049CCDE9C3
:108CB00000344FF02A33FFF70BFF02B010BD10B5A0
:108CC000044608B1FBF75CFD2046BDE81040FBF709
:108CD00069BD00207047704770472DE9F84304468E
:108CE000DDE90876914698460D4651B9B9F1000F75
:108CF00010D1B8F1000F15D1E7B91EBB55BB00204C
:108D000006E00830FFF773FC0028EFD0A0F58140A3
:108D1000BDE8F883494604F12000FFF768FC00280D
:108D2000E7D0F3E7414604F12800FFF760FC002894
:108D3000E2D0EBE7394604F11800FFF758FC0028B1
:108D4000DBD0E3E7314604F11000FFF750FC0028C8
:108D5000D4D0DBE704F10800FFF7AEFC6060CEE79B
:108D600010B5782200210446FEF73CFC0023C4E93C
:108D70001C3310BD4068704710B50446A0B3603086
:108D8000FFF7B7FB04F16800FFF7B3FB04F14800FD
:108D9000FFF7AFFB04F11800FFF7ABFB04F128006D
:108DA000FFF7A7FB04F12000FFF7A3FB04F110007D
:108DB000FFF79FFB04F10800FFF79BFB04F158004D
:108DC000FFF797FB04F15000FFF793FB04F140001D
:108DD000FFF78FFB04F13800FFF78BFB04F1300045
:108DE000BDE81040FFF785BB10BD00BA70476C228C
:108DF0000021FEF7F7BB10B16C21FBF7C1BC704737
:108E00002DE9F04105460E4614467AB3036C03F093
:108E10003F079B18036422BF436C013343645FB375
:108E2000C7F1400842451CD342463844FEF7CFFB09
:108E300029462846FBF70AFEC8B92744A7F1400493
:108E40003F2C46440BD90027F1192846FBF7FEFDBD
:108E500078B94037E31B3F2BF6D83E441C462CB173
:108E6000002722463146E819FEF7B1FB0020BDE895
:108E7000F0814FF0FF30FAE73F2AE4D8F1E773B50D
:108E8000036C03F03F035A1C0D46382A4FF0800153
:108E9000C1540446104400F28480C2F1380200211B
:108EA000FEF7A0FBD4E91060730F43EAC000FFF7A0
:108EB0009CFF04220DEB0201019004F13800FEF743
:108EC00086FBF000FFF791FF04220DEB02010190F9
:108ED00004F13C00FEF77BFB21462046FBF7B6FD84
:108EE0000646002857D1A06CFFF77FFF04220DEB48
:108EF000020101902846FEF76AFBE06CFFF775FF60
:108F000004220DEB02010190A818FEF760FB206D12
:108F1000FFF76BFF04220DEB0201019005F1080041
:108F2000FEF755FB606DFFF760FF04220DEB0201B9
:108F3000019005F10C00FEF74AFBA06DFFF755FF0D
:108F400004220DEB0201019005F11000FEF73FFB3A
:108F5000E06DFFF74AFF04220DEB0201019005F1DD
:108F60001400FEF734FB206EFFF73FFF0422019050
:108F70000DEB020105F11800FEF729FBA36E53B9B2
:108F8000606EFFF732FF042201900DEB020105F144
:108F90001C00FEF71CFB2046FFF72DFF304602B0F9
:108FA00070BDC2F140020021FEF71CFB21462046A5
:108FB000FBF74CFD06460028EDD10146382220463D
:108FC0006EE7002070474FF08053D3F83001421C09
:108FD00004BF4FF0704393F8E00F831F584258418D
:108FE0007047004700F00BB9C00000F1804000F569
:108FF000F830C0F81015C0F814257047FCF770BCA5
:10900000FBF75EBF036803F01F025B0902600CBF41
:109010004FF0A04000207047F7B5019001A8DDE9AE
:10902000084716461D46FFF7EDFF019BB6F1000C01
:1090300018BF4FF0010C00EB83000B1E18BF01237B
:10904000002D43EA4C0314BF4FF00C0C4FF0000C02
:10905000002C43EA0C0314BF4FF4E06C4FF0000CFB
:10906000002F43EA0C03D0F8002714BF4FF4403C14
:109070004FF0000C43EA0C0322EA030301B1097824
:109080000EB13678760019430DB12D78AD0031431D
:109090000CB12478240229430FB13F783F040C43DC
:1090A0003C43C0F8004703B0F0BD1FB50DF10F03FE
:1090B000019300238DF80F1000931A461946FFF70D
:1090C000ABFF05B05DF804FB024611F0010007D0CC
:1090D0004FF0A041D1F820351360C1F8203503B915
:1090E00000207047FCF706B9FCF7E4B80846FCF727
:1090F000D1B84FF080531A695869504370474FF008
:109100008053186970474FF080535869704703685F
:1091100003F01F025B0902600CBF4FF0A04000206B
:10912000704707B5019001A8FFF7F1FF019A0123ED
:109130009340C0F8083503B05DF804FB07B5019013
:1091400001A8FFF7E4FF019A01239340C0F80C3512
:1091500003B05DF804FB37B5D0F818358A69DBB287
:109160008DF807300B6A93423EBF4A699DF807406D
:10917000D4540B6A91F824500C695A1C0A620233C9
:1091800035B1A3428C6938BF0B619C4288BF8B61AB
:109190000D699D4205D9CA68D35CC0F81C35012011
:1091A0000AE08C699C4201D9CB7FF6E7AA42F6D34C
:1091B000A2422CBF0020012003B030BD70B5034691
:1091C0000025C0F80851D3F808310C46FFF7C3FF5B
:1091D00068B9887FFF2801D0FFF7A3FF2046657795
:1091E0002572616850F8083BBDE87040184770BDB3
:1091F000FCF732BD08B5FFF7FBFF002008BD08B142
:10920000F8F780BE7047704740B1C368587810F0D7
:1092100001001EBF1878B0FA80F040097047EFF3E4
:109220001183202383F31288BFF36F8FFEE710B5FD
:10923000D0E9003433B90020E268537843F00103E9
:10924000537010BD204698470028F4D00028B8BFBE
:109250004042E368FF28A8BFFF201870ECE7FEF744
:10926000C1B9FEF7B4B9704708B52024EFF31183F4
:1092700084F31288BFF36F8FFEF776F9F6E790F963
:109280000E308B4201D0FDF77BBA002070470346B9
:109290000020C3E90200C3E9003370473AB18A42B3
:1092A00005D3C0E90212C0E90000002070476FF04A
:1092B00015007047026801238B4022EA0303036014
:1092C00022FA01F000F00100704720B1002211469F
:1092D000783000F01DB9704713B501900846EFF3E0
:1092E0001184202383F31288BFF36F8F01A9FDF748
:1092F00019F884F31188BFF36F8F02B010BD10B559
:10930000FFF7EAFF041E08DDEFF31180202383F34B
:109310001288BFF36F8FFDF7A7FA204610BDEFF359
:109320000580003818BF012070476FF05700704764
:1093300000207047FDF77ABAD0E9003213605A6016
:109340000023C0E90033704708B5FFF7F5FF437B02
:1093500023F0020343730023836008BD38B504463D
:109360000D46FDF7EFF8637B43F002036373E5B14D
:10937000A5602B689D4209D16B68C4E900531C604D
:109380006C6012E06A689A42F6D01B68002BF3D03A
:1093900094F90E2093F90E108A42F3D09142F1DD38
:1093A0005A68C4E9003214605C6038BD10B5EFF350
:1093B0001184202383F31288BFF36F8FFDF7DAF84F
:1093C00084F31188BFF36F8F10BD10B504461830B9
:1093D00000F0C0F8EFF31181202383F31288BFF36C
:1093E0006F8F627B12F0100204D081F31188BFF3FB
:1093F0006F8F10BD2046BDE81040FDF7EFB808B5EF
:10940000EFF31181202282F31288BFF36F8F8368FC
:109410000BB1FFF799FF81F31188BFF36F8F08BD80
:1094200038B50446EFF31185202383F31288BFF388
:109430006F8F437B13F0280F0BD183680BB1FFF7BD
:1094400083FF637B51B903F0FB0363732046FDF791
:1094500091F885F31188BFF36F8F38BD03F0EB03EC
:10946000F3E701211838FFF7DBBF08B50346EFF338
:109470001181202282F31288BFF36F8F006883422C
:1094800007D008B1FFF760FF81F31188BFF36F8F3A
:1094900008BD0020F8E738B5EFF31185202383F3EA
:1094A0001288BFF36F8F0468A0420DD034B12046FC
:1094B000FFF74AFF04F1180000F04CF885F311881B
:1094C000BFF36F8F204638BD0024F7E7EFF311811B
:1094D000202282F31288BFF36F8F027BD2070CD554
:1094E00081F31188BFF36F8F002383F31188BFF3DB
:1094F0006F8F0423184602DF7047437B1B0704D598
:1095000081F31188BFF36F8F70470122FDF766B8B2
:1095100038B5EFF31185202383F31288BFF36F8FE3
:109520000468A04212D09CB1E16662612046FFF758
:109530000BFF04F1180000F00DF82046FDF71AF8B3
:10954000012085F31188BFF36F8F38BD0020F8E745
:109550002046F6E710B5EFF31184202282F312883B
:10956000BFF36F8F03683BB1FDF730FB002084F33E
:109570001188BFF36F8F10BD6FF01500F7E708B5C6
:10958000FDF742FC08BDFDF73FBC10B50446FFF7F0
:10959000E1FFA8B9636A0BB12046984704F11800AF
:1095A000FFF763FF60B1FFF701FFEFF311802023A6
:1095B00083F31288BFF36F8FBDE81040FDF754B9F5
:1095C00010BD00004C6BFF7F01000000F51E000085
:1095D000000000008D1F000044960000F59100007F
:1095E00000000000112A0000589600009930000089
:1095F0006C960000B123000000000000993A0000C2
:1096000000000000C38F0000000000008D6F00000C
:1096100000000000052D000000000000A93100003E
:10962000A8960000E128000080960000A931000003
:109630009496000009240000BC960000A52F0000AD
:10964000D096000068A600004099000058990000DC
:109650001C0600200015002039A90000D099000048
:10966000E899000022060020B8150020EFA90000AC
:10967000289A0000649A000026060020F0150020B9
:1096800015A9000000000000B49900002006002089
:109690000000000005AC0000709A0000209B000054
:1096A00028060020DC04002012AC0000C89A00004C
:1096B000209B00002A0600203C0500209AA80000FC
:1096C00074990000989900001E060020741500206F
:1096D000B3A90000000000000C9A0000240600203E
:1096E000C415002025510000E38F00000000000099
:1096F000537500006C960000FB7C00000000000029
:1097000053750000395C0000E38F0000000000008A
:10971000537500000D570000E38F000000000000AB
:1097200053750000000000005375000000000000A9
:109730005375000000000000537500000000000099
:1097400053750000D0960000152F000000000000A7
:109750005375000000000000537500000000000079
:109760005375000000000000537500000000000069
:10977000293B0000000000005375000000000000BD
:109780005375000000000000537500000000000049
:109790005375000000000000537500000000000039
:1097A0005375000000000000537500000000000029
:1097B0005375000000000000537500000000000019
:1097C0005375000000000000537500000000000009
:1097D00053750000000000005375000000000000F9
:1097E00053750000000000005375000000000000E9
:1097F000537500000000000053750000495C000034
:10980000E38F00000000000053750000000000001E
:109810005375000000000000537500001AA10000FD
:109820000300000083A60000030000003BA100002D
:10983000030000002FA9000003000000A1A9000000
:1098400003000000359D00000300000013AE00007F
:109850000300000064A6000003000000A4A80000AC
:10986000030000001FAC000003000000C1A90000BD
:0C98700003000000FDA900000300000040
:1098800016AE000000010000000000000000000013
:109890000338FDD8704700000300000006000000F8
:1098A000010000000CA00000AC9800000E010000B8
:1098B0000800000000000000000000000000F801A7
:1098C000BC960000010000000000000000E0000065
:1098D000809600000200000000E00000000200008E
:1098E000809600000300000000E000000020070058
:1098F000809600000400000000E20000001E070047
:10990000809600000500000000E20000001E070035
:1099100080960000060000000000F801002007000B
:10992000BC960000070000000020FF0100E00000DE
:10993000BC960000491F0000191F00000000000035
:10994000F92000004520000077A60000212000003B
:10995000E57600007DA60000ED1F00005F760000A8
:10996000BF76000000000000FD7500000000000050
:10997000000000009496000000127A000001000030
:1099800058960000120001000000000000000000D6
:109990000000000000000000117A0000577900006C
:1099A0004378000001240000F97600000100000067
:1099B00000FF0000A92800008D29000009290000EF
:1099C000A1280000912800000400000000FF000012
:1099D000FF07000000000050000000000000000031
:1099E0000060004000000000952A00008D7B000010
:1099F0009B7B0000B37B0000BF7B0000CB7B0000A3
:109A0000112C0000E57B00000000000000000000B9
:109A100000000000000000002D2F0000E92E0000D3
:109A200000000000000000000020004001000000D5
:109A300000000000489A00000000D601000000006D
:109A4000B52F0020B42F002000200040549A0000C1
:109A5000010000005C9A0000020000000400000009
:109A600005000001B57C0000E52F0000A77C000088
:109A70000030024001000000000000FF00FF000075
:109A8000000000000000000101000000477D000010
:109A9000A09A0000FFFFFFFF000000000000000090
:109AA00000300240AC9A000001000000B49A0000AF
:109AB000030000000D0000040E0000051100000668
:109AC0005896000012000100004000400000000015
:109AD000000000FF00FF0000000000000000000187
:109AE000010000003D7D0000F89A0000FFFFFFFF2D
:109AF000000000000000000000400040049B000047
:109B0000010000000C9B0000030000001F00000487
:109B10001E0000051D0000060000000000000000FF
:109B2000B9330000CF7D00000300000006000000F4
:109B3000982F8A4291443771CFFBC0B5A5DBB5E9B8
:109B40005BC25639F111F159A4823F92D55E1CAB2C
:109B500098AA07D8015B8312BE853124C37D0C55BA
:109B6000745DBE72FEB1DE80A706DC9B74F19BC102
:109B7000C1699BE48647BEEFC69DC10FCCA10C24F2
:109B80006F2CE92DAA84744ADCA9B05CDA88F976D6
:109B900052513E986DC631A8C82703B0C77F59BF40
:109BA000F30BE0C64791A7D55163CA06672929146C
:109BB000850AB72738211B2EFC6D2C4D130D385309
:109BC00054730A65BB0A6A762EC9C281852C7292CB
:109BD000A1E8BFA24B661AA8708B4BC2A3516CC7F9
:109BE00019E892D1240699D685350EF470A06A1032
:109BF00016C1A419086C371E4C774827B5BCB03481
:109C0000B30C1C394AAAD84E4FCA9C5BF36F2E681E
:109C1000EE828F746F63A5781478C8840802C78CAD
:109C2000FAFFBE90EB6C50A4F7A3F9BEF27871C6B0
:109C3000C4AD0000D2AD0000E6AD0000F5AD0000FF
:109C400001AE0000CC950000CC950000FC95000012
:109C500004960000449600004496000001000200B3
:109C60001000110012002000210022002300240017
:109C70003000310032003300FFFF77C295F360D22D
:109C8000EF7F3552500F2CB6798025633A205374FC
:109C9000617274696E6720626F6F746C6F61646566
:109CA000720A0025633A20556E61626C6520746FFC
:109CB0002066696E6420626F6F7461626C652069F2
:109CC0006D6167650A0025633A20426F6F746C6F9F
:109CD0006164657220636861696E6C6F61642061A4
:109CE000646472657373206F66667365743A2030BE
:109CF0007825780A0025633A204A756D70696E6789
:109D000020746F2074686520666972737420696DB1
:109D100061676520736C6F740A0025633A204E6595
:109D20007665722073686F756C642067657420684F
:109D30006572650A006D6375626F6F740025633A22
:109D400020696E76616C696420666C617368204975
:109D5000442025643B206578706563746564202524
:109D6000640A0000000000000000007072696D616C
:109D70007279007365636F6E646172790025633A6E
:109D800020426F6F745F696D6167655F63686563CB
:109D90006B2C20706173736564202857616B655567
:109DA00070290A0025633A20496D61676520696E54
:109DB0002074686520257320736C6F74206973208C
:109DC0006E6F742076616C6964210A0025633A2005
:109DD0004661696C656420746F206F70656E2066E3
:109DE0006C6173682061726561204944202564209C
:109DF00028696D61676520256420736C6F74202568
:109E000064293A2025642C2063616E6E6F74206390
:109E10006F6E74696E75650A0025633A2046616944
:109E20006C65642072656164696E67207365637434
:109E30006F72733B20424F4F545F4D41585F494D05
:109E4000475F534543544F52533D2564202D2074A2
:109E50006F6F20736D616C6C3F0A0025633A20467A
:109E600061696C65642072656164696E6720696D03
:109E700061676520686561646572733B20496D6147
:109E800067653D25750A0025633A20496D61676560
:109E90002025642075706772616465207365636F47
:109EA0006E6461727920736C6F74202D3E20707225
:109EB000696D61727920736C6F740A0025633A20B2
:109EC00045726173696E6720746865207072696D90
:109ED00061727920736C6F740A0025633A204572B1
:109EE0006173652074696D65203A202564206D7367
:109EF0000A0025633A20496D616765202564206367
:109F00006F7079696E6720746865207365636F6E22
:109F10006461727920736C6F7420746F207468654B
:109F2000207072696D61727920736C6F743A2030A1
:109F300078257A782062797465730A0025633A205F
:109F4000436F70792074696D65203A202564206D17
:109F5000730A0025633A2055706461746520746942
:109F60006D65203A202564206D730A0025633A2030
:109F700070616E6963210A0025633A2043616E6E49
:109F80006F7420757067726164653A206D6F7265D9
:109F900020736563746F7273207468616E20616CE6
:109FA0006C6F7765640A0025633A2043616E6E6FBB
:109FB0007420757067726164653A20736C6F747396
:109FC0002068617665206E6F6E2D636F6D706174B1
:109FD00069626C6520736563746F72730A00256330
:109FE0003A2043616E6E6F742075706772616465AC
:109FF0003A20736C6F747320617265206E6F7420E9
:10A00000636F6D70617469626C650A003082010A69
:10A010000282010100A6200D370E812C40A82F5E80
:10A0200095DCDD4104298D66B9B075A1807FBBBC8C
:10A03000CAFC9589E1819E517C12B8FB70C92A291E
:10A040008A58D4B2E92DBA3A6AEABA46E7733808B0
:10A050000183A21F723DC397068DD06B2E75DA2542
:10A060003CE800DEDFF220B727A62362C6C86C0DED
:10A07000682D702DAEDCC49AC9984B8D1C0606C99C
:10A08000438A65ED3279C7CBE864F4805D823DDBBD
:10A09000FCA2D574DA99B6F893D03CBB5253690C44
:10A0A00051149E0131E34F66CE5E64287C45586EA4
:10A0B000E5E839BC81910F2AAED7D5BC8B90C41688
:10A0C00059E46ECE1A040109AA58A2F2975F5D1AEC
:10A0D000CE6224883581282AA67C5280EA43320346
:10A0E000A9CB2C401BBDE6F42F851845FEDF34DEDE
:10A0F0009EEE04170A19DA3CA071CE019DB681923A
:10A100008D5337230F4DD5329B217A5B13597B8CAE
:10A11000E8146C9043020301000163627072696E7F
:10A1200074665F7061636B616765002D002B0030A2
:10A130007800305800286E696C2900666C6173687D
:10A14000002A2A2A20426F6F74696E67204D43559A
:10A15000626F6F742076322E312E302D6465762D2D
:10A16000313265356565313036303334202A2A2A5C
:10A170000A002A2A2A205573696E67206E524620EB
:10A18000436F6E6E6563742053444B2076322E39D4
:10A190002E302D3737383762323634393834302064
:10A1A0002A2A2A0A002A2A2A205573696E67205A09
:10A1B0006570687972204F532076332E372E3939E7
:10A1C0002D316638663364633239313432202A2ABD
:10A1D0002A0A0025633A2072302F61313A2020305C
:10A1E0007825303878202072312F61323A202030A3
:10A1F0007825303878202072322F61333A20203091
:10A2000078253038780A0025633A2072332F61347C
:10A210003A2020307825303878207231322F69701A
:10A220003A2020307825303878207231342F6C7203
:10A230003A20203078253038780A0025633A2020EB
:10A24000787073723A20203078253038780A0025EB
:10A25000633A204661756C74696E6720696E737429
:10A2600072756374696F6E206164647265737320C4
:10A27000287231352F7063293A20307825303878AC
:10A280000A0025633A20556E68616E646C6564202F
:10A290004952516E3A2025640A0025633A202A2A41
:10A2A0002A2A2A205553414745204641554C5420DF
:10A2B0002A2A2A2A2A0A0025633A2020204469767D
:10A2C0006973696F6E206279207A65726F0A002562
:10A2D000633A202020556E616C69676E6564206D5D
:10A2E000656D6F7279206163636573730A0025631E
:10A2F0003A2020204E6F20636F70726F6365737316
:10A300006F7220696E737472756374696F6E730A0D
:10A310000025633A202020496C6C6567616C206CD5
:10A320006F6164206F66204558435F524554555213
:10A330004E20696E746F2050430A0025633A202036
:10A3400020496C6C6567616C20757365206F6620B1
:10A3500074686520455053520A0025633A20202036
:10A36000417474656D707420746F206578656375D1
:10A37000746520756E646566696E656420696E73C8
:10A380007472756374696F6E0A0025633A202A2A15
:10A390002A2A2A20425553204641554C54202A2A25
:10A3A0002A2A2A0A0025633A202020537461636B0D
:10A3B000696E67206572726F720A0025633A202009
:10A3C00020556E737461636B696E67206572726F7E
:10A3D000720A0025633A2020205072656369736514
:10A3E000206461746120627573206572726F720AF5
:10A3F0000025633A20202042464152204164647285
:10A400006573733A20307825780A0025633A202056
:10A4100020496D70726563697365206461746120A1
:10A42000627573206572726F720A0025633A20208C
:10A4300020496E737472756374696F6E20627573F0
:10A44000206572726F720A0025633A202020466CE4
:10A450006F6174696E672D706F696E74206C617ABC
:10A4600079207374617465207072657365727661AA
:10A4700074696F6E206572726F720A0025633A20EC
:10A480002A2A2A2A2A204D5055204641554C54202C
:10A490002A2A2A2A2A0A0025633A20202053746196
:10A4A000636B696E67206572726F722028636F6ECE
:10A4B000746578742061726561206D6967687420C5
:10A4C0006265206E6F742076616C6964290A0025CC
:10A4D000633A202020446174612041636365737393
:10A4E0002056696F6C6174696F6E0A0025633A20AB
:10A4F00020204D4D46415220416464726573733A89
:10A5000020307825780A0025633A202020496E7390
:10A510007472756374696F6E204163636573732031
:10A5200056696F6C6174696F6E0A0052657365726B
:10A5300076656420457863657074696F6E202800C5
:10A5400053707572696F757320696E746572727578
:10A5500070742028495251200025633A20535053EB
:10A56000454C20696E20746872656164206D6F646B
:10A570006520646F6573206E6F7420696E64696313
:10A58000617465205053500A0025633A202A2A2A14
:10A590002A2A2048415244204641554C54202A2A18
:10A5A0002A2A2A0A0025633A202020427573206651
:10A5B00061756C74206F6E20766563746F722074A1
:10A5C00061626C6520726561640A0025633A20202F
:10A5D000204465627567206576656E740A002563A0
:10A5E0003A2020204661756C7420657363616C614C
:10A5F00074696F6E20287365652062656C6F7729BA
:10A600000A0025633A20415243485F45584345506C
:10A6100054207769746820726561736F6E202578A5
:10A620000A0A0025633A202A2A2A2A2A2044656237
:10A630007567206D6F6E69746F72206578636570E1
:10A6400074696F6E202A2A2A2A2A0A0025633A2072
:10A650002A2A2A2A2A20257320256429202A2A2A00
:10A660002A2A0A00736F6300636C6F636B40343097
:10A67000303030303030006866636C6B006C66637D
:10A680006C6B00636C6F636B5F636F6E74726F6C87
:10A690000025633A204661696C656420746F20650B
:10A6A0007869742044504420282564290A002563D1
:10A6B0003A2057616974696E6720756E74696C2001
:10A6C000666C6173682069732072656164790A0041
:10A6D00025633A204661696C656420746F20776158
:10A6E000697420756E74696C20666C61736820698A
:10A6F0007320726561647920282564290A00256326
:10A700003A204A454445432049442072656164200B
:10A710006661696C65643A2025640A0025633A2005
:10A72000425020636C656172206661696C65643AB1
:10A730002025640A0A0025633A20534644502072BB
:10A74000656164206661696C65643A2025640A006D
:10A7500025633A2053464450206D61676963202584
:10A7600030387820696E76616C69640A0025633A36
:10A770002025733A205346445020762025752E25F7
:10A780007520415020257820776974682025752030
:10A7900050480A0025633A20504825753A20253054
:10A7A0003478207265762025752E25753A2025751A
:10A7B00020445720402025780A0025633A2025733D
:10A7C0003A20257520256369427920666C6173689B
:10A7D0000A0025633A20556E61626C6520746F2013
:10A7E000656E74657220342D62797465206D6F64B6
:10A7F000653A2025640A0A0025633A2053464450EE
:10A8000020424650206661696C65643A2025640ADE
:10A810000025633A206C61796F75742070616765FB
:10A82000202575206E6F7420636F6D70617469628E
:10A830006C6520776974682065726173652073693F
:10A840007A652025750A0025633A206C61796F7559
:10A850007420706167652025752077617374657356
:10A860002073706163652077697468206465766918
:10A8700063652073697A6520257A750A0025633A35
:10A88000206C61796F7574207365747570206661D2
:10A89000696C65643A2025640A0077323571323577
:10A8A000364030007370695F6E6F720025633A2026
:10A8B000696E76616C696420616464726573733A71
:10A8C0002030782530386C783A257A750A0025636F
:10A8D0003A20756E616C69676E65642061646472AC
:10A8E0006573733A2030782530386C783A257A755C
:10A8F0000A0025633A206E6F7420776F72642D61B1
:10A900006C69676E65643A2030782530386C783A27
:10A91000257A750A00666C6173682D636F6E7472B8
:10A920006F6C6C65724034303031653030300066A9
:10A930006C6173685F6E7266006770696F40353076
:10A940003030303030300025633A204750494F20B6
:10A95000706F7274202573206E6F7420726561644D
:10A96000790A0025633A206661696C656420746F1A
:10A9700020636F6E666967757265204750494F2086
:10A98000686F6720666F7220706F72742025732065
:10A9900070696E2025752028657272202564290A49
:10A9A000006770696F5F686F6773000001020304DE
:10A9B00005060774656D70403430303063303030D8
:10A9C0000074656D705F6E7266350025633A2046CF
:10A9D00061696C656420746F20616C6C6F63617475
:10A9E0006520505049204368616E6E656C0A0075A1
:10A9F0006172744034303030323030300075617202
:10AA0000745F6E7266785F75617274650025633A73
:10AA1000204661696C656420746F20616C6C6F63A3
:10AA2000617465204750494F5445206368616E6EDC
:10AA3000656C20666F722057414B450A0025633ACA
:10AA4000204661696C656420746F20636F6E66696F
:10AA5000677572652057414B452070696E0A002565
:10AA6000633A204353204750494F20706F7274203F
:10AA700025732070696E202564206973206E6F74C1
:10AA80002072656164790A0025633A20557064611B
:10AA9000746520657863656564732063757272659B
:10AAA0006E74206275666665720A0025633A2048F6
:10AAB000616C662D6475706C6578206E6F742073A0
:10AAC0007570706F727465640A0025633A20536C68
:10AAD000617665206D6F6465206973206E6F7420E8
:10AAE000737570706F72746564206F6E2025730AC1
:10AAF0000025633A204C6F6F706261636B206D6F4D
:10AB00006465206973206E6F7420737570706F7246
:10AB10007465640A0025633A20576F726420736974
:10AB20007A6573206F74686572207468616E20386E
:10AB3000206269747320617265206E6F7420737572
:10AB400070706F727465640A0025633A20467265FE
:10AB50007175656E63696573206C6F7765722074BB
:10AB600068616E20313235206B487A206172652031
:10AB70006E6F7420737570706F727465640A00254F
:10AB8000633A204661696C656420746F20696E6960
:10AB90007469616C697A65206E7266782064726986
:10ABA0007665723A20253038780A0025633A2057B6
:10ABB000616974696E6720666F722057414B45204A
:10ABC00061636B6E6F776C6564676D656E7420741E
:10ABD000696D6564206F75740A0025633A205469B5
:10ABE0006D656F75742077616974696E6720666F33
:10ABF00072207472616E7366657220636F6D706C23
:10AC00006574650A00737069403430303233303017
:10AC1000300073706940343030303430303000737D
:10AC200070695F6E7266785F737069007065726DCF
:10AC30000074657374004255473B2063616E27744E
:10AC40002068617070656E007265766572740025AB
:10AC5000633A205365636F6E6461727920696D6138
:10AC60006765206F6620696D616765207061697234
:10AC7000202825642E2920697320756E7265616312
:10AC80006861626C652E205472656174206974205D
:10AC9000617320656D7074790A0025633A20496DEF
:10ACA00061676520696E6465783A2025642C2053BD
:10ACB00077617020747970653A2025730A002563E6
:10ACC0003A20496D61676520696E6465783A202590
:10ACD000642C205377617020747970653A206E6F10
:10ACE0006E650A0004010403040204010401040364
:10ACF000010303040104092040081C400000000077
:10AD0000010000000101000001010101000000003C
:10AD10005465726D696E616C0000000000000054A3
:10AD20005452205245474745530025633A20486115
:10AD30006C74696E672073797374656D0A00556E63
:10AD40006B6E6F776E206572726F7200756E6B6ED0
:10AD50006F776E0025633A203E3E3E205A455048AC
:10AD6000595220464154414C204552524F522025C1
:10AD7000643A202573206F6E204350552025640AC5
:10AD80000025633A204661756C7420647572696EA3
:10AD90006720696E746572727570742068616E6484
:10ADA0006C696E670A0A0025633A20437572726502
:10ADB0006E74207468726561643A202570202825BD
:10ADC00073290A0043505520657863657074696F74
:10ADD0006E00556E68616E646C656420696E7465A2
:10ADE000727275707400537461636B206F76657254
:10ADF000666C6F77004B65726E656C206F6F707359
:10AE0000004B65726E656C2070616E6963006D61E8
:10AE1000696E006F7300737973776F726B710000E6
:10AE200001000000FFFFFFFF13720000B498000054
:10AE3000F775000000000000B522000000000000CF
:10AE4000000000000000000000000000C09A0000A8
:10AE500001000000EC040020EC04002000000000D1
:10AE600001000000FC040020FC04002000000000A1
:10AE700001000000000000000000000000000000D1
:10AE800000000000000000000000000000000000C2
:10AE90000000000000000000949600000000000088
:10AEA000000000000000000000000000189B0000EF
:10AEB000000000004C0500204C05002000000000B0
:10AEC000010000005C0500205C050020000000007F
:10AED0000100000000000000000000000000000071
:10AEE0000000000000000000000000000000000062
:10AEF0000000000000000000A89600000000000014
:10AF000000000000E5750000D78C0000D98C00001F
:10AF1000D38C0000000000000000000000000000D2
:10AF20000000000000000000000000000000000021
:10AF30000000000000000000000000000000000011
:10AF40000000000000000000000000000000000001
:10AF500000000000000000000000000000000000F1
:10AF60000000000008000000FF00000000000000DA
:10AF70000100000000000000FFFF0F001406002089
:10AF80001406002000000000000000000000000087
:04AF900000000000BD
:10AF98000000000000000000396E00000000000002
:10AFA80000000000000000004806002048060020BD
:10AFB800F57600000000000000000000000000001E
:0CAFC800000000000000000015E015E093
:10E000003DB8F396000000000002000044B5040093
:10E010000000000000000000000000000000000000
:10E02000FFFFFFFFFFFFFFFFFFFFFFFFFFFFFFFF00
:10E03000FFFFFFFFFFFFFFFFFFFFFFFFFFFFFFFFF0
:10E04000FFFFFFFFFFFFFFFFFFFFFFFFFFFFFFFFE0
:10E05000FFFFFFFFFFFFFFFFFFFFFFFFFFFFFFFFD0
:10E06000FFFFFFFFFFFFFFFFFFFFFFFFFFFFFFFFC0
:10E07000FFFFFFFFFFFFFFFFFFFFFFFFFFFFFFFFB0
:10E08000FFFFFFFFFFFFFFFFFFFFFFFFFFFFFFFFA0
:10E09000FFFFFFFFFFFFFFFFFFFFFFFFFFFFFFFF90
:10E0A000FFFFFFFFFFFFFFFFFFFFFFFFFFFFFFFF80
:10E0B000FFFFFFFFFFFFFFFFFFFFFFFFFFFFFFFF70
:10E0C000FFFFFFFFFFFFFFFFFFFFFFFFFFFFFFFF60
:10E0D000FFFFFFFFFFFFFFFFFFFFFFFFFFFFFFFF50
:10E0E000FFFFFFFFFFFFFFFFFFFFFFFFFFFFFFFF40
:10E0F000FFFFFFFFFFFFFFFFFFFFFFFFFFFFFFFF30
:10E10000FFFFFFFFFFFFFFFFFFFFFFFFFFFFFFFF1F
:10E11000FFFFFFFFFFFFFFFFFFFFFFFFFFFFFFFF0F
:10E12000FFFFFFFFFFFFFFFFFFFFFFFFFFFFFFFFFF
:10E13000FFFFFFFFFFFFFFFFFFFFFFFFFFFFFFFFEF
:10E14000FFFFFFFFFFFFFFFFFFFFFFFFFFFFFFFFDF
:10E15000FFFFFFFFFFFFFFFFFFFFFFFFFFFFFFFFCF
:10E16000FFFFFFFFFFFFFFFFFFFFFFFFFFFFFFFFBF
:10E17000FFFFFFFFFFFFFFFFFFFFFFFFFFFFFFFFAF
:10E18000FFFFFFFFFFFFFFFFFFFFFFFFFFFFFFFF9F
:10E19000FFFFFFFFFFFFFFFFFFFFFFFFFFFFFFFF8F
:10E1A000FFFFFFFFFFFFFFFFFFFFFFFFFFFFFFFF7F
:10E1B000FFFFFFFFFFFFFFFFFFFFFFFFFFFFFFFF6F
:10E1C000FFFFFFFFFFFFFFFFFFFFFFFFFFFFFFFF5F
:10E1D000FFFFFFFFFFFFFFFFFFFFFFFFFFFFFFFF4F
:10E1E000FFFFFFFFFFFFFFFFFFFFFFFFFFFFFFFF3F
:10E1F000FFFFFFFFFFFFFFFFFFFFFFFFFFFFFFFF2F
:10E20000A8AC00202D830200EFD703001983020081
:10E210001983020019830200198302000000000024
:10E220000000000000000000000000004585020022
:10E230001983020000000000D98402001983020043
:10E240005D870200571A04005D870200452F030016
:10E250005D8702005D8702005D8702005D87020026
:10E260000D1A04005D8702005D870200411A040058
:10E270005D8702005D8702005D8702005D87020006
:10E280005D8702005D8702005D8702005D870200F6
:10E290005D8702005D8702005D8702005D870200E6
:10E2A0005D8702005D8702005D8702005D870200D6
:10E2B0005D8702005D8702005D8702005D870200C6
:10E2C0005D8702005D8702005D8702005D870200B6
:10E2D0005D8702005D8702005D870200FFFFFFFF90
:10E2E0002DE9F00791E8F807B2E802105B1854EB4B
:10E2F0000C04B2E802104D4156EB0C06B2E80210D5
:10E300004F4158EB0C08B2E8021059EB01095AEBE7
:10E310000C0A80E8F80780410130BDE8F00770473B
:10E320002DE9F00791E8F807B2E802105B1A74EBE8
:10E330000C04B2E802108D4176EB0C06B2E8021034
:10E340008F4178EB0C08B2E8021079EB01097AEB07
:10E350000C0A80E8F80780414042BDE8F0077047AA
:10E360002DE9F007524290E87800B1E880071740A5
:10E37000DB1918EA020854EB080419EA020955EB04
:10E3800009051AEA020A56EB0A0678C090E87800F6
:10E39000B1E8800717407B4118EA020854EB0804F3
:10E3A00019EA020955EB09051AEA020A56EB0A06B0
:10E3B00078C080410130BDE8F00770472DE9F007D3
:10E3C000524290E87800B1E880071740DB1B18EA5A
:10E3D000020874EB080419EA020975EB09051AEA48
:10E3E000020A76EB0A0678C090E87800B1E8800768
:10E3F0001740BB4118EA020874EB080419EA020945
:10E4000075EB09051AEA020A76EB0A0678C0804124
:10E410004042BDE8F00770472DE9F00152424FF04D
:10E42000040890E8300091E8C000A31B1340E41AF0
:10E43000F618EB1B1340ED1AFF1830C0C0C1B8F13D
:10E440000108EED1BDE8F001704700BF00B592ECC5
:10E45000080AB1E8805707EE101A53EC102A56EC60
:10E46000114AA7FB0251A8FB020BE7FB6310E9FB73
:10E4700062B041EC145AA8FB0351EAFB6201E7FBCE
:10E4800064B5E7FB6605E8FB661505EE10BAA9FB67
:10E4900003B6EAFB6316ECFB6356E8FB640BE9FB8F
:10E4A000641BEAFB645BECFB646B05EE900AACFB5F
:10E4B000023012EE104AEEFB6250E9FB6460EAFBA8
:10E4C00064B0E7FB6431E8FB645112EE904AE8FB6C
:10E4D0006461E9FB64B1EAFB640106EE103AA7FB54
:10E4E000043213EE104AE7FB6462E8FB64B2E9FB16
:10E4F0006402EAFB641211EE904AE9FB6453EAFB02
:10E50000646313EE904AE7FB64B3E8FB6403E9FB42
:10E510006413EAFB642306EE905A17EE109A99E80A
:10E52000000610EE108AA9FB0854EAFB68B412EE4C
:10E53000108AECFB6804EEFB6814E9FB6824EAFB34
:10E54000683410EE908AEEFB6865E9FB68B5EAFB7B
:10E55000680512EE908AECFB6815EEFB6825E9FB76
:10E560006835EAFB684507EE106A11EE108AAEFBCB
:10E570000876E9FB6806EAFB681613EE108AECFBE6
:10E580006826EEFB6836E9FB6846EAFB685611EE42
:10E59000908AECFB68B7EEFB6807E9FB6817EAFBBB
:10E5A000682713EE908AECFB6837EEFB6847E9FBBF
:10E5B0006857EAFB686700BD2DE9F04F07EE900A47
:10E5C000FFF744FF17EE908A07EE90BAA8EC084ACE
:10E5D00088E8FF00BDE8F08F00B591E89857A3FBED
:10E5E0000352A3FB0401E3FB6420E3FB671042EC4E
:10E5F000145AA3FB0752E3FB6802E4FB6415E3FB38
:10E600006805E3FB6925A4FB07B6E3FB6926E3FB8A
:10E610006A56E4FB670BE4FB682BE3FB6A5BE3FBF6
:10E620006C6B40EC151AA4FB0810E4FB6950E3FB8B
:10E630006C60E3FB6EB0E7FB6721E4FB6951E4FB30
:10E640006A61E3FB6EB1E4FB6E0106EE102AA7FBE4
:10E650000832E4FB6A62E4FB6CB2E4FB6E02E7FBA7
:10E660006E12E7FB6853E7FB6963E4FB6CB3E7FBFF
:10E670006C03E7FB6E13E8FB6E2306EE905AA7FBD4
:10E680000954E7FB6AB4E7FB6C04E8FB6C14E8FB95
:10E690006E24E9FB6E34E8FB6865E7FB6AB5E8FBCE
:10E6A0006A05E8FB6C15E9FB6C25E9FB6E35EAFBB6
:10E6B0006E4507EE106AA8FB0976E8FB6A06E9FBDF
:10E6C0006A16E9FB6C26EAFB6C36EAFB6E46ECFB4D
:10E6D0006E56E8FB69B7E9FB6907E9FB6A17EAFBD5
:10E6E0006A27EAFB6C37ECFB6C47ECFB6E57EEFBE2
:10E6F0006E6700BD2DE9F04F07EE900AFFF76CFF43
:10E7000017EE908A07EE90BAA8EC084A88E8FF0056
:10E71000BDE8F08F30B44FF0000310F8014B11F852
:10E72000015B013A84EA050443EA0403F5D1A3F14D
:10E7300001034FEAD37030BC704700BF4FF00003B5
:10E7400010F8012B013943EA0203F9D1A3F10103C7
:10E750004FEAD370704700BF30B411F8014B12F884
:10E76000015B6C4000F8014B013BF6D130BC7047B7
:10E770002DE9F00791E8F807B2E802105B1854EBB6
:10E780000C04B2E802104D4156EB0C06B2E8021040
:10E790004F4158EB0C08B2E8021059EB01095AEB53
:10E7A0000C0A8941B3F1FF3374F1FF3475F1FF3581
:10E7B00076F1000677F1000778F1000879F1010998
:10E7C0007AF1FF3A51F100015B184C414D4156F18D
:10E7D000000657F1000758F1000859EBD1795AEBC0
:10E7E000010A80E8F807BDE8F00770472DE9F00757
:10E7F00091E8F807B2E802105B1A74EB0C04B2E877
:10E8000002108D4176EB0C06B2E802108F4178EBD6
:10E810000C08B2E8021079EB01097AEB0C0A894185
:10E820005B184C414D4156F1000657F1000758F175
:10E83000000859EBD1795AEB010A80E8F807BDE8E6
:10E84000F007704718EB040859EB05095AEB060A64
:10E850005BEB070B5FF0000C4CF1000C18EB0508AC
:10E8600059EB06095AEB070A5BEB070B50EB0C0060
:10E870005FF0000C51EB0C0152EB0C0263414CF1C8
:10E88000000CB8EB070879F100097AF1000A7BEB7C
:10E89000040BA841B141A241B3416CF1000CBBEBA8
:10E8A000050BB041B941AA41BB416CF1000C4CF0E1
:10E8B00001068CF0020718EB060859EB6C095AEBBD
:10E8C0006C0A7BEB6C0B70EB6C0471EB6C0572EB00
:10E8D000670653EB6C076CEB6C0C18EB0C0059EBF8
:10E8E0000C015AEB0C025BF1000354F1000455F1EA
:10E8F000000556EBDC7657EB0C0770472DE9F04F1F
:10E9000007EE900AFFF7A2FD59EC168A17EE10AA3F
:10E91000FFF798FF59EC148A5BEC15AAFFF792FFFA
:10E9200017EE908A88E8FF00BDE8F08F2DE9F04FE0
:10E9300007EE900AFFF750FE59EC168A17EE10AA60
:10E94000FFF780FF59EC148A5BEC15AAFFF77AFFFA
:10E9500017EE908A88E8FF00BDE8F08F064B074A63
:10E960005B7802604FF420728280C371082200231A
:10E9700082710372704700BFD013002061E2010072
:10E98000064B074A9B7802604FF494728280C371F1
:10E990000822FF2382710372704700BFD01300204A
:10E9A000CFDD0100F8B5C41D002824F0070405469A
:10E9B00014BF2046002000F035FB061E02DA6FF07F
:10E9C0000B00F8BD0DB9F442F9D4284FB979787924
:10E9D0003B7AFA79033103300CF073FE0028EEDB4A
:10E9E00039787B7826440336002D194426F0030637
:10E9F00000FB01F114BF3046002000F09FFC3044C2
:10EA00000DB90028DBDBBA780346B2B1F97BFB789D
:10EA100011441944FF29D2DC0330002D20F00304F7
:10EA200014BF204600207A89C9B200F0F7FC031E0B
:10EA3000C5DB23440DB9002BC1DB397B81B1BA782A
:10EA400072B10733002D23F0070414BF20460020C5
:10EA500003F058FF031EB2DB23440DB9002BAEDBDD
:10EA6000002D0CBF18460020ABE700BFD0130020DC
:10EA70001FB572B6184B9D6AE5B9BFF34F8F1749A2
:10EA8000174BCA6802F4E0621343CB60BFF34F8FA9
:10EA900000BFFDE7B2FBF6F2DCB20133002AF9D188
:10EAA00004F110036B4403F80C2C0A2234B901A8BA
:10EAB000A847E2E7024600230A26EDE7631E04AEFC
:10EAC000DCB256FA83F3B0FBF2F602FB16003030EC
:10EAD00003F80C0C3046E9E7D013002000ED00E00D
:10EAE0000400FA0507B50C4B1A7A8DF80120DA7983
:10EAF0008DF8002068469A795B79ADF80420ADF86E
:10EB0000023002F075FB18B1D9210320FFF7B0FFE6
:10EB100003B05DF804FB00BFD013002038B50546F4
:10EB200070B30AF075F910B94FF0FF3038BD0FF02F
:10EB30008DFCB0F5FA7FF7D8144C1548A562002576
:10EB400000F0E8F926222946204684F82C500AF0E5
:10EB500067FD01236370A3701B23637140F21B33B5
:10EB6000E380022323721F23638108232373EFF3BF
:10EB7000108472B600F028FD2CB962B62046D5E7A5
:10EB80006FF01500D2E72846D0E700BFD013002071
:10EB9000E5EA000010B500283CD1214C94F82C3057
:10EBA000032B34D059B1002A37D00239052931D886
:10EBB000DFE801F003142230252813786370002069
:10EBC000FFF7F0FE0028B7BF0123022384F82C30A2
:10EBD0006FF00B00A8BF84F82C3010BD9378E3B120
:10EBE000D378D3B113781A2B17D953781A2B14D999
:10EBF0001368C4F80530E2E71378A370DFE71388E1
:10EC00006381DCE71388FF2B07D82373D7E74FF026
:10EC1000FF30E2E76FF02C00DFE76FF01500DCE774
:10EC2000D0130020F8B50D46064630B329B311F0D5
:10EC3000070422D1124F97F82C30012B02D16FF02C
:10EC40000B00F8BD032B02D14FF0FF30F9E700F0C5
:10EC50009DF80028F8D02846FFF7A4FE0028EEDB38
:10EC60000FF035FB3046214602F056FBFFF73AFF26
:10EC7000032387F82C302046E3E76FF01500E0E728
:10EC8000D013002010B5074C94F82C30032B03D17F
:10EC900002F05AFB03F020F90CF007FE002084F884
:10ECA0002C0010BDD013002050B1074B03F114020B
:10ECB00053F8041B40F8041B9342F9D1002070471D
:10ECC0006FF01500704700BFE586050010B5074BD3
:10ECD00093F82C403CB902F0E9FA0120044900F015
:10ECE00099F9204610BD4FF0FF30FBE7D01300200C
:10ECF00081E9000010B5074B93F82C403CB902F0B5
:10ED0000E9FA2046044900F085F9204610BD4FF08D
:10ED1000FF30FBE7D01300205DE9000010B5054B84
:10ED200093F82C401CB902F08DFA204610BD4FF02C
:10ED3000FF30FBE7D013002010B5054B93F82C40B3
:10ED40001CB90DF03CFE204610BD4FF0FF30FBE734
:10ED5000D013002010B5054B93F82C401CB90DF0D2
:10ED600031FE204610BD4FF0FF30FBE7D0130020EE
:10ED7000024B02681A600020704700BF0014002098
:10ED8000014B1B68184700BF00140020024B186895
:10ED9000003818BF01207047001400202DE9F74308
:10EDA000294E0446071D2848376003F0ADF80228B5
:10EDB000054607D1244920460BF08BFF284603B0B7
:10EDC000BDE8F083042838D13378072B18D13E20D2
:10EDD00000F050F878B9F378327901A943EA0223B8
:10EDE0006846ADF800300CF052FA0028DBD0532111
:10EDF0000820FFF73DFE052000F07CF80028EAD04F
:10EE0000314620460BF0CCFFB0F5817F01D3722153
:10EE1000EEE70028C7D094F8008094F802904046AE
:10EE200000F028F80028BED0B8F13E0FC6D1484601
:10EE300000F060F80028C1D1B5E70828BED102492A
:10EE400020460BF075FFB9E704140020074B4FF084
:10EE5000FF3141F6FF72C3E9001205490022C1E902
:10EE600000221F21C3E90212704700BFC004002026
:10EE7000481400203F280CD801380B4BC0F3421235
:10EE800000F01F0053F8223023FA00F000F00100D8
:10EE90007047FF2806D04038C0F34212034B00F001
:10EEA0001F00EFE701207047C00400204814002035
:10EEB0000146074B006849681A4603C240F48C2299
:10EEC0001A6041F0107242F4FF625A60704700BF4E
:10EED000C00400200246024B0068516803C370471B
:10EEE000481400200246024B0068516803C3704773
:10EEF000C80400200138064BC0F3421203EB820322
:10EF000000F01F009B6823FA00F000F0010070473A
:10EF1000C0040020014B1860704700BF501400204F
:10EF200007B5FFF793FF0DF09CF9044B1B6813B175
:10EF300001909847019803B05DF804FB501400203D
:10EF40000B880288F0B5C3F30E049EB204F11403DB
:10EF5000C57CC35A02352A442B4497B213FA82F374
:10EF6000013B4288B3FBF7F313FB07439BB29A4282
:10EF7000044A93BF22EA0603324013439BB20B803C
:10EF8000F0BD00BF0080FFFF08B54B1E062B04D864
:10EF90004FF4D1711520FFF76BFD0A4B994202D94E
:10EFA00040F2A311F6E719B900B10160084608BDA7
:10EFB00028B103680022C3E901211A1D1A60043137
:10EFC000F4E700BFFAFFFF7F10B5114B00EB4104DF
:10EFD0001A786389B3FBF2F303FB0223013A1A4464
:10EFE000B2F5706F027928BF00231A448378B2FB10
:10EFF000F3F0194403FB1020091AB1FBF3F003FBF3
:10F00000101313446FEA43436FEA5343638110BD07
:10F0100054140020024B03EB80004160704700BF96
:10F02000541400202DE9F04F10F0070A85B0054672
:10F0300004D040F261111720FFF71AFD554F07F178
:10F040000C06B1460446B0464FF0010B57F8043B9E
:10F050008DF80BA03BB101A898479DF80A30082B0A
:10F0600001D9E821E7E79DF80B1081BB05B13160BC
:10F07000B94506F10406E9D12DB3DFF81CE1002300
:10F080008EF800301E46022258F82200013A60B184
:10F0900090F804A08178BAF1FF0F66D14FF0000715
:10F0A0008E4207713CBFCEB20123511CECD10BB193
:10F0B0008EF80060022640F6FF6A58F82670002F8E
:10F0C00065D1013EF9D2601B05B0BDE8F08F9DF817
:10F0D0000AC0BCF1020FE64601F1050238BF4FF04D
:10F0E000020E0EF1FF3004EB42040444CEF10000A6
:10F0F0002040BDF808406444013CCCF1000C04EA17
:10F100000C04B4F5803F4FEA420301D3F82192E7A3
:10F1100075B1C31A336099701C8083F803B09DF8F1
:10F120000C201A71019A1A814FEA124CA3F806C0FA
:10F1300004FB01049CE758F82C90B9F1000F06D0AD
:10F1400099F804B0D34504BF99F802904F440CF1EC
:10F15000FF3CBCF1000FEEDA3944FF29A0D90BB116
:10F160008EF8006040F2271165E794460027F0E72B
:10F1700007EB41033846A3F80AA0FFF725FF09F182
:10F180000109BB785FFA89F18B42F1D899E74FF01A
:10F190000009F6E75814002054140020F8B54FF683
:10F1A000FF730380184B03EB810105460869B8B172
:10F1B00086780379B3FBF6F206FB1233DBB219460D
:10F1C0000A1D00EB4202B2F902705488002F09DBDD
:10F1D0000131B1FBF6F206FB1211C9B28B42EFD13D
:10F1E0000020F8BDFF29FBD0C4F30E03C4782B80A8
:10F1F00024B94FF4D5711720FFF73AFC5380BDE8CE
:10F20000F8400CF03DBA00BF541400201D4B03EB36
:10F21000810170B50C69054644B3030404D54FF46D
:10F22000DC711720FFF724FC014620460CF00AFA97
:10F23000FF28014604D02046BDE870400CF020BAFB
:10F24000A078B5FBF0F300FB1353DBB219460A1D9F
:10F2500004EB4206B6F90260002E09DB0131B1FB76
:10F26000F0F200FB1211C9B28B42F0D1002070BD48
:10F27000FF29FBD08B4204EB42021CBF0023E3704A
:10F280005580D8E754140020094B03EB810110B5D9
:10F290000C69014620460CF0D5F9FF28014604D040
:10F2A0002046BDE810400CF0EBB9002010BD00BFB7
:10F2B00054140020F8B5104B03EB810107460C698C
:10F2C000014620460CF0BEF9FF28054611D0E6881D
:10F2D000238953EA064606D0014620460CF0D0F9B1
:10F2E00001463846B04720462946FFF76DFE00200C
:10F2F000F8BD0520FCE700BF5414002038B50E4BC4
:10F30000827903EB82030446186908B9052038BDE9
:10F310008278E1799142F9D24B1CE37100EB410311
:10F320005D89B3F90A30002BF3DBA5800CF0A8F956
:10F3300020600020EBE700BF5414002070B50446A5
:10F3400010F003000E4603D04F211820FFF790FB6A
:10F35000FFF71AFE054624B1034831460460FFF763
:10F3600013FE284670BD00BF701400202DE9F3473E
:10F370001C4C9DF82CA0904622681E4607469DF81E
:10F3800028300D461AB961211820FFF771FB1A4683
:10F390000921404601930BF0DBFF52461FFA80F92A
:10F3A000092130460BF0D4FF19FA80F120680CF0E7
:10F3B0001EF9019B386018B9286002B0BDE8F087DB
:10F3C00000EB09042C603868414609220BF079FFF4
:10F3D000286853460922314602B0BDE8F0470BF0D9
:10F3E00070BF00BF7014002070B50E4604460BF0CD
:10F3F000C2FF054630460BF0BEFF044B2A182146DB
:10F400001868BDE870400CF016B900BF70140020F9
:10F41000014B18680CF0DFB8701400201F2AF8B5F3
:10F4200004460ED89200033222F00303B3F5803F66
:10F430002ED2194DB4B1A00711D05F210920FFF7DA
:10F4400017FBFF2A4FEA420304D9FF329A42A8BFB2
:10F450001A46E8E77C2BB8BF7C231A46E3E72970FD
:10F460006C602B8122F0030201EB81031204D800AF
:10F4700001276B68120C0025EEB28E4200D3F8BD56
:10F4800014B126181F705E60104401352833F3E76D
:10F490004FF0FF30F3E700BF7414002038B5144A72
:10F4A000147853680021C8B2844203D8AB210920E4
:10F4B000FFF7DEFA1846013105782833002DF2D027
:10F4C0000021817001241289447044688161C16106
:10F4D000920800F12001051D21F8022B994245F800
:10F4E000044B1444F8D100234361037038BD00BFBE
:10F4F000741400202DE9F8434B7880460C4602F046
:10F50000040602F0FB07D3B1DFB12E4BD4F8049010
:10F510001D89B7BB01236370AD08A761E76104F1E2
:10F5200020034A46211D04F1280023F8025B98427B
:10F5300041F8042B2A44F8D10023636101E0002F35
:10F54000E3D0FF23A370002E18BF0226A3191B7D52
:10F55000032B03D1022F1CBF0136F6B2A3190122DF
:10F560001A7506F10C0204EB8606002324F812300B
:10F570007268A370C8F80020A8F804304046BDE8BF
:10F58000F883002114226170A0180AF049F8B5F53B
:10F59000FF7F0FD26B08ED1AADB209EB0502C4F87C
:10F5A00004902584A2606384C4F80C90A584226131
:10F5B000E384C6E7B5F5EE6F4FF0FF03EBD940F2F9
:10F5C0007265EAE774140020134B012200214FF00A
:10F5D000FF309A60C3F80012C3F80803C3F800159F
:10F5E000C3F804259A60C3F80803C3F80015C3F8EC
:10F5F00004250A490A4A03F580334FF40040C3F852
:10F600000825C1F88000BFF34F8FBFF36F8FC1F89B
:10F610008001C3F80825704700F0004000E100E0D9
:10F620000000F63F0A46192302F8033B0448C3686A
:10F63000C1F803300369536043699360704700BFAA
:10F6400080140020024B5A8C02435A845B6A18478C
:10F6500080140020014B00215B6A184780140020B1
:10F6600010B5154C05F0C6FD05F044F9208DFFF7E7
:10F67000F1FF237E63B12246104952F80C3BE36050
:10F680006368536004F11900A36893600DF035FFBF
:10F690000B4B228D93E8030003F0BCF9236B188811
:10F6A00003F0E4F8A36B94F8341094F8350098470D
:10F6B000002384F83C3010BD8014002025F60000A3
:10F6C000AC140020034B93F83C300BB1FFF7C8BFDC
:10F6D000704700BF8014002070B51D4C256B636C13
:10F6E000236495F89430064694F848000BB1031D46
:10F6F000D8B295F869102EB9FF2803D195F8683073
:10F700008B4201D005F004FC95F89430D3B1E06C45
:10F7100005F010FE012384F86830D5E93E23E16C42
:10F72000206CC4E9182305F09BF816B9304605F0A3
:10F7300041FE95F86810002005F086FE022384F84B
:10F740003C3070BD206C05F0F5FD05F0D3F8ECE71A
:10F750008014002008B5094B93F83C20022A04D0FD
:10F7600040F253212720FFF783F9DA7A42F00102B1
:10F77000DA72BDE80840FFF773BF00BF80140020B5
:10F7800010B50E4CA26F137803F00303032B04D1C2
:10F79000D378022B01D1002010BDE06F0BF07EFE6C
:10F7A0000028F9D1A36F1B7803F00303032BF2D0D9
:10F7B00001F0BEFE80F00100C0B2EDE78014002031
:10F7C0002DE9FF41434C94F83C30256B012B064654
:10F7D0000F465FFA83F804D040F2A4412720FFF7D8
:10F7E00047F995F884303BB1002185F88410042056
:10F7F000FFF728FF85F88680A16F0B7803F00303DD
:10F80000032B05D195F88A3013B90220FFF71AFFB0
:10F81000A26F137803F00303032B02D053781BBBB2
:10F82000012385F88A3095F89430BBB1D5E93E01C3
:10F83000236B94F848200392C4E918014FF00108A3
:10F8400093F8690084F868800CF031F800210346D1
:10F850000091039A2049404604F0BCFF36B104B041
:10F86000BDE8F041FFF7FCBE0223DAE7002FF6D037
:10F87000D4F88030304698470028F0D094F83430DF
:10F88000002BECD194F88430DD06C3F3001001D5D1
:10F89000FFF776FF636CD4F888201B78C3F300135E
:10F8A0002AB9B4F88C2013B1B2FA82F35B09628CE6
:10F8B000910709D5A36FDB78022BD0D1002004B0CB
:10F8C000BDE8F041FFF708BF002AC8D10343F5D1D6
:10F8D000C5E700BF80140020D014002010B5064BEF
:10F8E00093F83C2002F0FF0422B91C7603F08AF85A
:10F8F000204610BD0C24FBE7801400200A4B0B4A65
:10F9000070B506460D461A60FFF7E8FF18B1E12111
:10F910002720FFF7ADF8064C012104F18E000DF011
:10F92000C8FC6664E56470BD08050020F4000100B1
:10F9300080140020024B012283F8B020704700BFE2
:10F9400080140020F0B5814D85B002AE86E803003A
:10F9500095F83C100A9F01F0FF0411B90AB103B1F8
:10F9600027B940F26F112720FFF782F896E80300CD
:10F9700005F12C0C8CE8030085F8B04085F8344084
:10F9800085F8B14085F8354085F8B24085F8B34038
:10F990006C842C852C6BC5F880306A62AF6305F0EF
:10F9A000F5FA04F0A7FF94F96C0005F08BFB606A90
:10F9B00005F0B2FCE06905F08BFB94F8A40005F0BB
:10F9C000ADFB2B6B93F8AF310BB105F0CDFA94F88A
:10F9D00069209D21012005F0F9FB5D4B186805F0B9
:10F9E000A1FC2369EB676369C5F8B43094F87730FC
:10F9F00073B9226F62B1B4F8BE10B4F888308B428C
:10FA000006D1B4F874100B44A4F8BE30012313607F
:10FA1000504E04F5807304F58877186859683246AB
:10FA200003C20833BB421646F7D1D4F810314A4A14
:10FA3000C5F86930D4F8143153602B6B93F88E20DD
:10FA400093F86860A2F12501012903D993F88F107A
:10FA500025295DD193F856322BB1012E03D0012B0D
:10FA600014BF0226012604F13007314638460DF056
:10FA7000D6FD31460DF07AFAA38F94F869109842BA
:10FA800028BF184685F8B80038460DF0B1FD94F847
:10FA9000691094F89470B4F84460042908BF0321F5
:10FAA0000DF064FA0FB9043080B2B04228BF30467E
:10FAB00094F89430C6B285F8B96085F8486093B17F
:10FAC000D4E93E2394F869000127C5E9182385F895
:10FAD00068700BF0ECFE0022034600921D4932468E
:10FAE000384604F077FE0120FFF7F6FD00232B6077
:10FAF0006B60AB60B4F888306B8023882B8094F8FF
:10FB0000A4302B71A36F0BB101221A6005B0F0BDB8
:10FB1000203A012A0CD823290CD093F8363113F05F
:10FB2000010211D19B079ED5012E18BF02269AE72C
:10FB3000232905D193F8362193F861301340EEE77D
:10FB4000032E08BF04268EE716468CE7801400209B
:10FB500008050020D0140020E914002008B50C4B43
:10FB600093F83C201AB9BDE80840FFF779BD93F837
:10FB70003C20022A04D040F235212720FEF778FFEE
:10FB80001B6BD3F8C801BDE8084005F0E5BB00BF1A
:10FB900080140020014B1876704700BF80140020AD
:10FBA000014B93F8B200704780140020024B188D6F
:10FBB000C0F3C020704700BF80140020014B93F8B1
:10FBC000B1007047801400202DE9F3411E4D8207DB
:10FBD0002C6B06460F4622D5D5F8883023B940F263
:10FBE00095412720FEF744FFB5F88C20296C184674
:10FBF000033291F8018009F09DFC0DF1020201A988
:10FC00002864D5F8B4000BF0DCFC01980BF0C3FCC1
:10FC1000012238604146D5F8B4000BF089FCF307A7
:10FC20000ED5D4E93E32013342F10002C4E93E323E
:10FC300094F88C30012B0CBF0023012384F88C3006
:10FC400002B0BDE8F08100BF801400202DE9F04F24
:10FC5000AB4C002387B0CDE9043394F83C30276BDC
:10FC6000022B81468A4604D04FF4A3612720FEF779
:10FC7000FFFE238D590606D44020FFF7EBFC238DB1
:10FC800043F04003238597F89430B9F1000F00F05A
:10FC90002881B3B104F060FE04F044FE88B9236CFF
:10FCA0005A7872B11B7897F88C20C3F3C0039A423C
:10FCB00007D1012384F83530FFF7D2FC07B0BDE847
:10FCC000F08F236C5978A4F88C1009B3D4F8B400E1
:10FCD0000BF005FCC4F88800238D97F88B2043F4C3
:10FCE00000732385236C1B78C3F380039A4200F0D2
:10FCF000B980256B95F88A30002B3DD0022B11D1AD
:10FD0000E06F04A90BF082FB28B940F20E41ADE789
:10FD1000C4F88810E0E7D5E93C32013342F1000233
:10FD2000C5E93C3295F88630002185F88A1023B168
:10FD300085F886101020FFF785FC95F885309BB17B
:10FD4000002685F8856001F0DDFB10B940F2254101
:10FD50008CE731460820FFF775FCD5E93C320133CA
:10FD600042F10002C5E93C3295F88B30012B0CBF03
:10FD70000023012385F88B30238D43F40063238512
:10FD80004FF0000B216C97F88C200D78C5F3C00361
:10FD90009A4240F0988005F00305032D266B63D04E
:10FDA000002D6CD196F88C30013B18BF012386F8EA
:10FDB0008C30236C5B7833B1D6E93E32013342F1AB
:10FDC0000002C6E93E3297F893308BB1D7E93C2365
:10FDD000002697F8680084F86860C4E918230BF0DF
:10FDE00066FD484900960346FB22304604F0F2FCCB
:10FDF000BAF1000F40F08880628C94F8B13012079D
:10FE000003D5A26FD278022A7ED0012B7CD8D4F8F9
:10FE1000803001209847002876D094F83480B8F1DB
:10FE2000000F71D1266B94F8483096F894208DF825
:10FE30000D80002A40F0B380FF2B96F8681003D1A4
:10FE400096F869308B4202D0FF2005F061F896F8F1
:10FE50008A30032B00F23881DFE813F0A400D500CC
:10FE60001D012E01CB468DE7238D012043F48053E5
:10FE700086F8840023850025FFF7E4FB92E74D78A0
:10FE8000002D8FD0238D96F8945043F48053238512
:10FE900004F0E8FF042894F8B93006D1002D14BF0F
:10FEA0001B221F22934228BF1346226C52789A428B
:10FEB0000BD8D4F88850002D85D094F8B03073B1A9
:10FEC0002020FFF7C7FB00257DE794F834300120A0
:10FED00043F0100384F8343006F08EFBF3E74D4610
:10FEE00060E70BB104F06EFD94F8B130013384F893
:10FEF000B130238D002543F480632385AB4662E750
:10FF000080140020D014002005F0BEFA4FF0010A42
:10FF10001DB105A90220FFF757FEBBF1000F0DD060
:10FF2000B4F80720B4F805301343B7F8882013431A
:10FF30001EBFB4F809300133A4F80930B9F1000F3D
:10FF400000F0CA80B4F805300133A4F8053000236E
:10FF500084F8B130634802F077FC049830B10BF0BC
:10FF60001AFB216B0022027202F01EF8059B33B1CE
:10FF7000216B00221A720C22059801F0E3FFBAF1FE
:10FF8000000F7FF499AE238D1B063FF597AE8020BE
:10FF9000FFF760FB238D43F0800323858EE6043357
:10FFA000DBB249E794F8B830ADF80E304E48A6F809
:10FFB000583001F097FA50B1A16F4FF48070FFF7FD
:10FFC00041FB012386F8853084F8B3301DE0E06FF3
:10FFD0000DF10D020DF10E010BF0F5F9A06790B1D6
:10FFE00096F8D1307BB99DF80D302BB90380837022
:10FFF000A06F01210DF05DF9BDF80E10A06F0DF09E
:020000040001F9
:1000000025FA0123E0E7394BA36796F88B30A26FFE
:10001000DB0003F00801137803F0F3030B4396F8B9
:100020008C10890001F004010B4323F010031370BE
:10003000FFF7A6FB0028A06F037818BF4FF0100849
:1000400048EA030880F8008096F89330002B3ED0F1
:100050004378002B3BD0E06C05F06CF9002384F86A
:100060006830D6E93C23A16FE06CC4E9182304F0A2
:10007000F7FB96F86910012005F0E6F9A26F1188E8
:10008000A4F8841091781A4A012384F8B230917050
:1000900084F83C303CE7B6F85830E06FADF80E30ED
:1000A0000DF10D020DF10E010BF08DF9A067002886
:1000B000A7D140F2F321D9E50B4801F013FA00284B
:1000C0009FD140F2FD21D1E540F20B31CEE505F0A4
:1000D00031F904F00FFCCCE7B4F807300133A4F891
:1000E000073037E7AC140020F81400200E1500206C
:1000F0000415002055F700004DFC0000C1F700007A
:10010000C5F600000B2808B504D940F2C13106201D
:10011000FEF7AEFC014B33F8100008BD946B0400F1
:100120002DE9F04F2DED028B8BB00446154602935E
:10013000894690F869B00CF08CFC064694F8B00142
:10014000FFF7E0FF94F88F300393304485F001030C
:1001500086B2059355BB94F8F431032B26D1039B4B
:100160000D2B23D1B4F854324B451FD1D4F8FC31B8
:10017000C4F8E831A369B4F8CC21C4F8EC31B4F880
:1001800042321344C4F8F031204604F043FAD4F864
:100190005832A362B4F85632A385D4F85C32A36116
:1001A000D4F860322362022384F8F431B4F8407248
:1001B000B4F88880A9EB07073FB204F50473002F59
:1001C00008EE103AB7BFD4E98A23029BC4E98E2314
:1001D00001230493CD4BA9EB08081B780FFA88F88C
:1001E000B8BF474603F0FF05002B53D00EF028F9A7
:1001F00000286FD0B4F8E031012B6BD994F8F431BA
:10020000022B67D094F80A52002D63D194F8B00104
:10021000FFF778FF94F8F43100F5C860012B86B23F
:10022000D9B24AD194F89230D4F828A0032B3ED109
:10023000D4F8EC5155443146D4F8EC010EF0FAF8FC
:10024000D4F8E831C4F8E801A0EB030AD4F8F0319F
:100250003146284603FB0AFA0EF0ECF8D4F8F851C0
:10026000C4F8F801451B3146A0690EF0E3F8AA4432
:10027000B4F8CC51D4F8F0314544ED1BDB432B44AA
:10028000D4F8FC51451B05FB03A50123C4F8FC0170
:1002900084F80A3294F8F431DFF870A2032B00F2EC
:1002A0008C81DFE813F0190014016900350128463C
:1002B0000CF084FE00EB0A05BDE7A06931460EF0A4
:1002C000B9F8B4F8CC51D4F8FC314544ED1BC31A4D
:1002D0005D43DAE70025DDE7012100200CF06EFE2A
:1002E0008046A06A314640440EF0A4F83146C4F876
:1002F000F801A0690EF09EF807A9C4F8FC0108A84F
:1003000005F0CAF8079B0093D4E98E01DDE90823C4
:1003100008F062FC074620460BF0EDFAD4F84432B0
:10032000A66A94F869001E4405F0FCF9D4F8F811A7
:10033000A38D943E761AB044A8EB070800F523403D
:1003400030314FF47A7703EB4101A130B0FBF7F085
:10035000A8EB000794F869000BF0B9FAD4F844321E
:10036000FB1A2230B3F5917FCAF8040058D240F24C
:10037000C6413020FEF77CFBA36AD4F8EC0131467D
:1003800018440EF057F83146C4F8F801A0690EF091
:1003900051F8C4F8FC0120460BF0ADFAB4F8CC31AA
:1003A000A66AD4F8EC71002B40F08D80029B002BE4
:1003B00000F0898094F8690005F0B4F93E44D4F85F
:1003C000F871943ED4E98A23F61BD4F83072804643
:1003D0003E4494F86900B61A05F0A4F94FF47A7314
:1003E00000F2E73708F52340B7FBF3F73744A130B5
:1003F000B0FBF3F0D4F8F811D4F8E831D4F8F021D8
:10040000303102FB0311A38D3F1A03EB410194F835
:1004100069000BF05CFA0123CAF8040084F8F43197
:10042000A6696FF4F4731E44D4F8FC31F61ADAF8B6
:1004300004309E4228BF1E46D4E98E327F1BDF194E
:1004400042F100024FF00008C4E98872C4F8C861A4
:1004500084F8108204F130000DF0C8F8B4F8B81137
:10046000A4F84092D4E98823A1EB09090FFA89F98D
:10047000C145C4E98E23C8BF022384F81882C8BFCF
:1004800084F81832039B30440D2BC4F81402029BED
:1004900000F09680002B40F0948094F8F431002B0B
:1004A00000F0AD80A169D4F8FC3118EE100AC91A29
:1004B0000CF02BFD80B2002800F0A180169B03B148
:1004C00018800120ABE0D4F8F801374492E7D4F863
:1004D000FC21A369D4F8F001D4F8E8119B1A5F431A
:1004E000B4F8CC319844C3439844D4F8F83130334D
:1004F00001FB0033A18D94F8690002FB083301EB86
:1005000043010BF0E4F9CAF8040089E73C15002028
:10051000A369D4F8FC219B1A5F4394F88E30252BF5
:1005200003D094F88F30252B0AD1B4F85432A9EBBC
:1005300003031A0404D494F85732002B18BF9B46C7
:10054000049B63B3B4F8CC314BBBD4E98A23D4E920
:100550008C0182428B4102D340F21A5109E794F890
:10056000690005F0DFF8D4F830220646D4E98A01A4
:10057000A2F194031B1A3B4494F86900049305F01C
:10058000D1F8049B00F2E7374FF47A7206F5234066
:10059000B7FBF2F71F44A130B0FBF2F03F1AB4F8FA
:1005A000CC11D4F8FC31414459433031490058460C
:1005B0000BF08DF91C4B586032E740F23251D8E60F
:1005C000EBB1B4F8E01121B3B4F8E22194F8E431CE
:1005D000A4F8E22102FB0333994202F101000EDD8F
:1005E00094F818325BB1002384F81832A4F8E201C1
:1005F00001F070FD00F00700013084F8E40118EE0E
:10060000101A94F80B0207F0B1FB20B940F27B51AD
:10061000AFE60A46DAE7059B84F8083200200BB003
:10062000BDEC028BBDE8F08F3C1500202DE9F041B8
:1006300004460D46164690F8F83003F0FF071BB14C
:100640000C273846BDE8F0810146454807F042FADC
:1006500020288046F4D05822394604F1D00008F012
:10066000DFFF84F8D080C4F8D450FF2384F8F8303A
:1006700035B101F047FD00F00700013085F8E401D5
:1006800002234FF00008A4F8083184F800810DF02F
:10069000DFFE9E3085B220460DF07EFC014670B331
:1006A0000CF0D7F900F5CD6081B230460DF0C2FEF6
:1006B0003044C4F804010EF02DF8281841F100016F
:1006C000C4E94401012084F8D800A4F826800DF084
:1006D00021FDDB3E361AC4F8DC604FF0FF326FF0CC
:1006E0000043C4E9462394F8D00004F5807107F074
:1006F0003DFB48BB40F2C1113020FEF7B9F920465E
:100700000DF06FFBDFF85C80DB30C4F80401B8F853
:10071000080048B1E08C38B101F0F4FCB8F80830BA
:10072000B0FBF3F202FB130005440DF0F3FF2D18AC
:1007300041F10001C4E94451002ECED0751941F1B8
:100740000001C4E94651CEE7D4E944230021C4E9BD
:100750003A23C4E93C2320460DF03BFC71E700BF7F
:10076000C9BB01003C150020F0B5002385B0CDE9E0
:10077000003301238DF806306846FEF7BFFD70B1E7
:100780001B4E0123B3720027CDE9027702A8FEF7C2
:10079000B5FD0546A8B10023B37205B0F0BD0098C1
:1007A0000BF0CBFAE8E790F80B0208F0D3F894F8D6
:1007B0000B0284F8F45107F0B9F9202384F80B32C6
:1007C000E2E7029B002BE1D093F80B22202ADDD038
:1007D00018884FF6FF739842DDD02946FEF754FD86
:1007E00004460028DFD140F22B113020FEF740F9FB
:1007F0003C150020054B00220121DA7219709A7213
:1008000042F210721A81FFF7AFBF00BF3C15002003
:10081000014BD872704700BF3C15002008B504F0AA
:1008200027FB044BDA6882422ABF987A002080F0C6
:10083000010008BD3C1500202DE9F34704460629B8
:1008400000F2C680DFE801F0047C69798085BF0092
:10085000D0E98A23D0E98C0182428B414BD294F8B3
:100860000A32002B47D094F8F431032B43D194F88B
:1008700069A00CF0EEF8074694F8B001FFF742FCCF
:10088000D4E98A12D4F83032D4F8C86181460744DA
:100890005046A3EB010804F03DFF361A504604F021
:1008A00041FF00F523404FF47A72A130B0FBF2F023
:1008B000321AA2F17401A2F1D403BFB2490809F5BA
:1008C000C8699D317B431FFA89F9B3FBF9F36033A3
:1008D0005A08A1EB5303984502D31144884501D926
:1008E0000DF0B0FDA06939460DF0A4FD0023C4F859
:1008F000FC0184F80A32384B9B7A03F0FF0263B99B
:10090000B4F8BC11009201232046FFF709FC38B16E
:1009100040F2CA613020FEF7ABF8042384F8F431CA
:1009200004F0BAFC06F08EFFB4F88820A4F8062282
:100930000023A4F8423284F8093202B0BDE8F087FF
:10094000032380F8F431F8E704F0B2FAC4E98C012B
:10095000F3E78569D0F8FC31DFF87C809D4288BFE1
:10096000ED1A98F80B3098BF00251BB9036B9D4218
:1009700028BF1D4604F13000D4F8C8710CF036FED3
:100980000744022007F06AFEEE1B26EAE67686425E
:1009900028BF06460221304607F0B4FE00B93744AE
:1009A00040F2D312394620460CF071FED4F8C8311B
:1009B000C8F80C00A069184407F000FE0028BCD15C
:1009C00040F27931A6E702B0BDE8F0470AF093BFE4
:1009D00040F265719EE700BF3C1500202DE9F84309
:1009E00006460C4615467ABB04F042FAD4E944891F
:1009F000074684F8D85084F8F8500121D4F8D40080
:100A000000F0D6FFD4F8D400C0E98A8994F8D02049
:100A100080F80B22C0E98E89C0F844720BF086F88A
:100A200020B140F20A713020FEF722F804F034FCC5
:100A300006F008FF074994F8D000324605F0CCFDD7
:100A400028B94FF4EF61EEE740F28F71EBE7BDE8B4
:100A5000F88300BF1FB90100014B1881704700BF28
:100A60003C150020F0B5070CA7F5AA42144B543AE8
:100A7000012A03EA90231FD927F4004042F6AA2254
:100A8000801A18BF01200022162116461F2487EA6B
:100A9000060562EA0505013510D0DD03ADB245EA71
:100AA0005606E503ADB2013945EA52024FEA530357
:100AB0004FEA5404EBD1F0BD0020E4E70020FAE750
:100AC000E0FF3F00304BF0B51A88B0F85C70B0F82A
:100AD0005A605D88974228BF1746964228BF16463F
:100AE0001B2E85B00C462ED0B5F5A47F2DD040F638
:100AF00048039D4201A928BF1D460BF07EFABDF8B0
:100B00000A309F4228BF1F46BDF80C30E780AB4239
:100B100028BF2B462381BDF806309E4228BF1E46C3
:100B2000BDF8083066809D4228BF1D46A580FF2382
:100B30002370E3881B3B9BB2E02B08D940F2F751AE
:100B40003920FDF795FF1B2FCED105B0F0BD63888E
:100B50001B3B9BB2E02B02D940F2F951F0E723890D
:100B6000A3F5A4739BB2B3F5E06F02D940F2FB5139
:100B7000E6E7A388A3F5A4739BB2B3F5E06FE4D9CD
:100B800040F2FD51DCE700BF4C15002010B50121FB
:100B90000020FEF779FB044670B90121FEF736FB11
:100BA000044620B940F23D313920FDF761FF034B87
:100BB00093F904100DF0D9F8204610BD4C15002013
:100BC00008B50CF055F900F0FFFD00F0EDFB0CF05E
:100BD0006CFC00F08DFF01F0A7FE00F0A1FF084BB8
:100BE0001B224FF4A4711A805980064B06499A8043
:100BF00000221960DA825A821A835A7408BD00BF33
:100C00004C1500207419002003021B00044B41F610
:100C10004C52C3E902221B221A74FFF7D1BF00BF56
:100C2000741900202DE9FF41344DAB68044640F8AB
:100C3000303F0BF0B9F8064600F0A6FB2B7C84F899
:100C400038302F4B668710F0200F1B681DBFAA8815
:100C50006988A4F85A101B2208BFA4F85A20A4F8E7
:100C60005C201BB194F96C1020889847AE7CEF7C17
:100C7000B5F8148041F64C53A36116B900F08AFB15
:100C8000064677BB00F086FB074666B358B303A958
:100C900020468DF80C608DF80D70ADF80E800CF0CC
:100CA00089F9AB886A8869780191033329780091C2
:100CB00003329BB292B204F1140104F11000FEF76A
:100CC00055FB236913B940F2CE5114E0636913B99F
:100CD00040F2CF510FE0002004B0BDE8F0810920C0
:100CE000FAE7002ED3D120880021FEF7E3FA00288E
:100CF000F5D040F2B9513920FDF7BAFE7419002041
:100D00000C050020F7B505460E460DF065F80028E5
:100D100073D028460DF040F940B1B6F80130013BE0
:100D20007F2B03D91224204603B0F0BD28460DF0D6
:100D300037F908B90C24F6E728460BF0EAF8002842
:100D4000F8D128460DF002F804460028F2D12846D2
:100D500002F0AAFA0028E5D0B6F80170F17842F264
:100D60001072284657430DF004F928460DF00CF98F
:100D7000014658B93A462846FFF758FC0446002871
:100D8000D1D041F683113920FDF772FE21460DF1D5
:100D90000600FEF703FA064668B3214600F008FE97
:100DA000BDF806303380284631460DF003F9284659
:100DB0000DF0FCF898B928460DF0FAF801463046D7
:100DC000FFF730FF04460028ADD13A4631462846A9
:100DD000FFF72CFC044620B141F6A611D3E7012110
:100DE000EDE7074B9B68002B9DD0024606F59571F9
:100DF0003046984797E70D2495E7422493E700BFD4
:100E00004C150020034B5A8802801B788370002009
:100E1000704700BF7419002037B583781A2B054638
:100E200009D8042B05D9012202FA03F3134A13420D
:100E300005D112241AE0292B01D03B2BF9D12888A7
:100E4000B0F5706FF5D269460CF052F888B9019B85
:100E500093F8282102F0FF046AB9AA7883F82921BF
:100E6000FF2283F8282168460CF0FAFA204603B0E6
:100E700030BD0224FAE70C24F8E700BF2000380454
:100E80000188A1F11B039BB2E02B0CD84288A2F58C
:100E9000A4739BB244F24810834204D8034B002051
:100EA00019805A8070471220704700BF4C150020EF
:100EB000034B1A885B88028043800020704700BF84
:100EC0004C15002038B504784278857804F0010389
:100ED00052EA030104F0020401D1112038BDBCB96B
:100EE000002DFAD0002B08BF144601E0002425464F
:100EF00020460BF04DF80028EFD028460BF048F8BC
:100F00000028EAD0054B00209C74DD749882E5E748
:100F1000002BEBD114461D46EAE700BF74190020F0
:100F200013B5008869460BF0E3FF18B10224204690
:100F300002B010BD019A92F8F431DBB292F8B02001
:100F4000002AF3D113F0FB0FF0D0019890F83A315A
:100F50000BB13A24EBE790F8DC3003F0FF04002BF0
:100F6000F7D190F8D3309B0706D1FF2380F83A31B0
:100F700068460CF075FADAE70249D4300CF0BDFA95
:100F8000D5E700BF23DC0100F0B50778EF2F85B06F
:100F900004460D4603D91225284605B0F0BDB0F829
:100FA0000130ADF80C309DF90C209DF80C30002A72
:100FB000F1DB9DF80D209107EDD1DA063FD49E06B6
:100FC00003F0030238D5002AE5D11807E3D463788B
:100FD000190711D42179E278E07942EA0122617996
:100FE00042EA0142A17941EA0021207A41EA004126
:100FF0008A42D0D81F2ACED9627A013A062ACAD8A4
:10100000A27A032AC7D813F0040102D1023A012AB6
:1010100003D8E27A012ABED811B9A27C032ABAD831
:1010200013F01001227D19D0012AB4D1227E012AA9
:10103000B1D8B1B91125AFE7032AC6D1ABE713F098
:10104000600FA8D103F00F0203F00703052BBED0F9
:10105000931E012BBBD9002A9DD1B8E7022AE5D106
:1010600099E7DA071FD46378227D03F01801082975
:101070001ED1022ADED11B0709D4E279A37943EA03
:101080000223227A43EA0243B3F5804FD2D8BFB29B
:1010900001213846FEF7F8F8064678B10AF039FF24
:1010A000B8B10C2578E700F031F90028DBD1C1E7B1
:1010B000022AE0D0A27E002ADDD0BBE7012138461B
:1010C000FEF7A4F8064650B3164B93F904100CF043
:1010D0004CFE30460CF055FF21462870E074304637
:1010E0000CF09BFE637E0546002B3FF455AF0028B5
:1010F0007FF452AF316B02466846FEF7FBF9306B66
:101100002A4601210AF025FB316B68460422FEF7CE
:10111000F1F9306B2A4629460AF01BFB3CE707250C
:101120003AE700BF4C15002070B50579042D8AB050
:10113000034658D84488B4F5804F54D82B48465DB0
:10114000284400214279857AC07BADF8041042F032
:10115000100242EA460242EA850242EAC00202F076
:101160001F028DF80420BDF80420ADF80D201A8868
:101170008DF80F208DF81240120A240A8DF81110F4
:101180008DF814108DF810208DF813405A7B8DF8CF
:1011900015205A798DF816209A79D3F807008DF822
:1011A0001720B3F80B209B7B8DF81E307F238DF822
:1011B0001F3001238DF80C1006908DF82110ADF82A
:1011C0001C208DF820308DF8223003A88DF82310D4
:1011D0008DF824108DF825108DF8261001A9FFF741
:1011E000D3FE0AB070BD1220FBE700BFAC6B040059
:1011F0000278034672B1427862B142881A2A09D94C
:1012000082881A2A06D9044A006810609B88938055
:10121000002070471220704774190020024B0268AA
:101220009A600020704700BF741900200378A3F172
:101230000A02112A9DBF024A00201374122070472F
:101240007419002008B5052000F090F803F012FA98
:10125000014B024A9A6008BD4C150020C50A0100E6
:1012600008B502F009F8FFF7C5FABDE808400148E3
:1012700001F0ECBF5815002010B50B4C012384F889
:10128000023102F001F80DF00AF80BF0EFFD04F264
:1012900003112046FEF732FB00200AF0F9F9BDE801
:1012A000104000F029BE00BF5815002010B5064CB4
:1012B000064904F502700BF091FB04F50370044934
:1012C000BDE810400BF08ABB581500201005002027
:1012D0001805002010B5094C094904F502700BF0FF
:1012E0007DFB04F5037007490BF078FB04F50470EF
:1012F0000549BDE810400BF071BB00BF5815002038
:10130000280500203005002020050020014B93F81F
:10131000020170475815002010B5074C00F0C8FDB9
:10132000D4F808020BF052FBFFF770FC00F002FF4C
:10133000012384F8143210BD58150020014B93F896
:10134000140270475815002010B5074CD4F80C0251
:101350000BF03CFBD4F810020BF038FBFFF730FC2D
:10136000002384F8143210BD58150020C208054926
:10137000012300F0070003FA00F08B5C1843885447
:10138000704700BFD0040020014BD3E90001704733
:10139000D0040020034B1868C0F30020400040F048
:1013A00001007047D004002008B50DF04FF8084A3E
:1013B000002332F82310814205D302EB83039B788C
:1013C000044A137008BD01330C2BF2D10023F7E758
:1013D000C06B04006D17002010B544682388A4F882
:1013E000783194F8683084F87711012B06D0022BFD
:1013F00004D040F217310620FDF73AFB84F87A3129
:1014000094F86930012B01D0022BF2D184F87B31A2
:10141000044904F5B7700CF070F8002384F83431F7
:1014200010BD00BF57CA0100406808490388A0F8F2
:101430006A3190F8603080F86C3190F8613080F853
:101440006D3100F261100CF052B800BF6DCA01009E
:10145000044B002283F822204FF6FF729A84DA842C
:101460001A8570476E170020054B9A8C824201BF87
:10147000002283F822204FF6FF729A84704700BF43
:101480006E170020014BD884704700BF6E170020F4
:10149000084B998C4FF6FF72914206D193F82220A7
:1014A000012A04D00360012070470023036000205C
:1014B000704700BF6E170020064B93F82220012AC8
:1014C0001FBF0120DA8C83F822009A8408BF002015
:1014D000704700BF6E170020014B1885704700BF92
:1014E0006E170020064A918C138D994205D192F80F
:1014F000223013B10260012070470020704700BF06
:101500006E170020094B998C1A8D914201D0002052
:1015100070474FF6FF729A8493F82220002AF6D083
:10152000002283F822200120704700BF6E170020A0
:10153000054B998C1A8D914203BF93F82200B0FAA3
:1015400080F04009012070476E17002050B90A4A08
:101550001346012003F8010B0868C2F801008A88CD
:101560009A807047012805D1034B0A689A608A88DF
:10157000D8719A81704700BF9817002048B90A4B6C
:10158000187880B1D3F80120B3F805300A608B8059
:101590007047012806D1044BD87920B19A680A60B7
:1015A0009B89F4E7002070479817002020B9054B6D
:1015B000187800F00100704701280ABF014B002095
:1015C000D879F6E798170020F7B500228B888DF8B8
:1015D0000600ADF8043008680C4B8DF80720019D1B
:1015E0001C78014603F5AC73D0B2844201D80820C0
:1015F00009E0D3E90076AE4208BF8F4203F1080349
:1016000002F10102F0D103B0F0BD00BFA817002025
:1016100030B5094B01465C78002203F58173D0B2E6
:10162000844201D8082005E013F8015B8D4202F1E5
:101630000102F4D130BD00BFA8170020F0B5254D40
:1016400095F8984189B0224605F29911684607F04D
:1016500071FF214668460BF02AFC0446B8B300EB44
:101660004001C9B202A8FDF78BFB601E95F8A1618D
:10167000C0B2012495F8982105E0731CB3FBF2F188
:1016800002FB1133DEB206F120030DEB030111F86A
:10169000203C002BF1D100EB400220326A4406EBE3
:1016A00046032B4412F8187C83F8A27112F8177CB9
:1016B00012F8162C83F8A37183F8A42101F8204CAA
:1016C0000138AB19C0B2FF2883F89941D2D109B0D3
:1016D000F0BD00BFA817002070B5064688B00C46C4
:1016E000002A4FD02A4A92F8A131D01890F89911C7
:1016F00021B94FF480712820FDF7BAF903EB4301BB
:101700001144013391F8A251E57091F8A35191F879
:10171000A41161710021257180F8991192F8981136
:10172000B3FBF1F001FB103382F8A13192F8C23122
:1017300023B9184902F5DD700BF0DCFE657905F080
:101740003F0545F0400565710D220021684607F010
:1017500067FFE3788DF80F3023798DF80E3004AAF7
:101760000423694630468DF80D5007F087FC9DF83C
:101770001F3023709DF81E3063709DF81D30A370DC
:1017800008B070BD03216018FDF7FAFAD6E700BF74
:10179000A81700203D160100044B5A78824286BFEC
:1017A0001B1893F84A010020704700BFA8170020BB
:1017B000044B5A78824286BF1B1893F842010020DE
:1017C000704700BFA8170020064B00224FF461713C
:1017D0001A8083F8C32183F8C421A3F8C61183F8C3
:1017E000C2217047A8170020014B83F8C40170473D
:1017F000A8170020014BB3F8C6017047A8170020B6
:1018000030B50A4B5C7884420ED9184490F8020136
:101810002B3003EBC004A5790D7053F83000106035
:10182000A3889380012030BD0020FCE7A81700208A
:101830000246074810B590F8C34124B1417821B160
:10184000023002F03DFF204610BD0C46FBE700BF12
:10185000A81700202DE9F74F2F4C00921A46637805
:1018600083428046894654D9231893F8425185F023
:101870000105E9B193F84A31D3B945F002070135C2
:10188000C2B9F9070BD5062101FB084104EB08108A
:1018900001F5857182300092FFF71EFF009ABB07A9
:1018A00033D504EB081049460230FFF715FF2CE052
:1018B0002F46E5E794F8A1614FF0010A002DE0D032
:1018C00004EB060B9BF8991199B9009B0192D3B1D7
:1018D00000F000FC06EB460121444FEA102C81F891
:1018E000A201019A81F8A3C1000C81F8A4018BF830
:1018F00099A194F898110136B6FBF1F001FB10663E
:10190000F6B2013DDAE747F00407384603B0BDE818
:10191000F08F0027F9E700BFA8170020074B5A787F
:10192000824209D91A1892F842212AB9062202FBEA
:10193000003000F58570704700207047A817002020
:10194000064B5A78824281BF1B1893F83A01B0FACD
:1019500080F0400998BF0020704700BFA817002002
:1019600030B50024A0F84240B0F8464042F210756D
:101970004C43B4FBF2F4A0F84640541E05FB03436D
:10198000B3FBF2F3A0F84430084BB3FBF2F301339E
:10199000A0F84A30838F05FB0344436BB4FBF2F499
:1019A00059438463B1FBF2F2426330BD005A6202D4
:1019B00070B504460D4649BB4FF4207207F030FE67
:1019C000012384F896306FF0360384F8E330042363
:1019D00084F8E4306FF03B0384F8E5306F2384F83B
:1019E000E6306FF03F0384F8E7302B2384F8E230D1
:1019F000FE2384F81E317F2384F88D30202384F861
:101A0000E85084F8E95084F80B3270BD012922D1E6
:101A10000023A0F8CC3180F8C331154B8269134400
:101A2000B3FBF2F3C0F8B83040F6B833A0F8BC30DE
:101A30001146438C8030FFF793FF07F037FC30B13D
:101A4000E069FFF70FF810B984F8AF51DDE7002324
:101A500084F8AF31D9E70229D7D1B0F86232D0F893
:101A60005C228169BDE870408030FFF779BF00BF1C
:101A70007FC3C901034B80F86C101B680BB1008851
:101A80001847704738050020074B93F90030184479
:101A9000142804DC10F17F0F03DB40B270471420E0
:101AA00070476FF07E0070477019002007B57F23E4
:101AB0000DF107008DF8073003F0BAFC9DF90730EF
:101AC00068B10A4A5078404243FA80F0142808DC92
:101AD00010F17F0F07DB40B203B05DF804FB18463E
:101AE000FAE71420F8E76FF07E00F5E770190020A0
:101AF000024B00221A705A70704700BF7019002004
:101B0000054BFF221A70054A0168116001791171B5
:101B100000221A70704700BF72190020D8040020FC
:101B200007B5064B186800901B798DF8043068469D
:101B3000FFF7E6FF03B05DF804FB00BFFA8605007F
:101B4000437843B1C2783A2A07D80549885CC31A5A
:101B5000584258417047184670470120704700BFEF
:101B6000F06B04003A2908B5C17003D8064B5B5CE2
:101B7000437008BDFF2904D04FF489612A20FCF787
:101B800077FF0123F4E700BFF06B04002DE9FF4766
:101B90008A4602A9154699460BF0AAF9064600287E
:101BA0003CD1039F35B9012487F89540204604B005
:101BB000BDE8F087D7F810802946404609F0A2FB1F
:101BC00004460028F2D0174B5B88AB4228D301466D
:101BD00001AA404609F0D9FC97F895300198002BEE
:101BE0000CBF514602210BF064FB01982A4649467E
:101BF000033007F09FFC2946404609F0C8FB044625
:101C000018B97A212B20FCF733FF02A80BF028FC2F
:101C1000039BA3F8BA6187F89560C7E70124C5E77D
:101C20003446C3E774190020024B987DC04300F08E
:101C30000100704774190020034B987D80F002006A
:101C4000C0F34000704700BF7419002083230B705D
:101C5000014B1B78CB707047901900207FB505466B
:101C60000C4621B94FF48B711020FCF701FF03885B
:101C70008B8000234B724669304609F078FC0146A0
:101C800010B940F21F11EFE701AA304609F07DFCC0
:101C9000E08010B94FF49271E6E7FB2802D94FF4C7
:101CA0009371E1E701980BF00CFB012801D00228A9
:101CB00005D12072206828B940F23D11D4E74FF4D5
:101CC0009B71D1E70199E288033107F033FC30467C
:101CD00009F063FC10B94FF4A171C5E7002130464B
:101CE00009F0B9FB10B940F24711BDE70A4BDA7DA4
:101CF00082B11A8B2888013A02A91A830BF0F8F8EE
:101D000010B14FF4A871AFE7039AB2F8A6300133CF
:101D1000A2F8A63004B070BD741900202DE9F74375
:101D200006460D464FF0050800274FF003092B69C2
:101D300043B11B7A33B12C69A4B90022104603B019
:101D4000BDE8F0836C68237A012BF6D0EFF31083A3
:101D500072B66A6812686A6003B962B6237A002BA9
:101D6000E5D02C61237ADBB284F80880013B0B2B91
:101D700065D8DFE803F0610620335E643C64646488
:101D80006451636823B94FF4EE711020FCF770FEC4
:101D90003146204698470422EFF3108372B6217A29
:101DA0000529C8B201D0002852D127722F61002B1B
:101DB0004AD162B648E0636813B940F2E511E4E73E
:101DC000314620469847C0F30723012BADF80400A5
:101DD000C2B237D0022BDFD12F6135E0636813B96F
:101DE00040F2EF11D1E7204698470022D4E763681C
:101DF0000BB9DB21C9E70B2232701988A6F8031052
:101E000001220024B27072711869B471214609F080
:101E100022FB2C61042291E7606810B940F21A217C
:101E2000B3E70E4B31461B68984700232B61022213
:101E300084E740F22321A8E740F22621A5E740F2FB
:101E40002921A2E784F80890002A3FF470AF75E7D3
:101E5000002B7FF46CAF62B669E700BF3C05002041
:101E600038B5124C231D14220021184607F0D8FB68
:101E700003460125257414220433002104F11800BF
:101E8000C4E9013307F0CCFB84F8245004F11C03AF
:101E9000C4E906330023E362236384F83430C4F8D2
:101EA0003530C4F8393084F83D3038BD9019002001
:101EB00010B5084C2378FF2B04D04FF4B7711020D5
:101EC000FCF7D6FD07F022F92070BDE81040FFF7BF
:101ED000C7BF00BFDD04002010B5034C207807F019
:101EE00031F9FF23237010BDDD040020014B187869
:101EF00007F038B9DD040020014B024A1A60704730
:101F00003C0500205D1C010038B50B4D05F11801A2
:101F10000446FFF703FF70B9AB681B7A0C2B04D1A2
:101F2000064BDA7D0AB11B8B2BB120460449BDE874
:101F30003840FFF7F3BE38BD901900207419002017
:101F40009419002010B51346027A22B140F2C9213B
:101F50001020FCF78DFD0A46BDE8104001460148FF
:101F60000BF0A5BA94190020044890F834301BB93E
:101F700003492C300BF0B8BA704700BF901900200D
:101F8000A1D401000346064890F83E203AB190F8EB
:101F90003D2022B900F8353B02490BF0A5BA704745
:101FA000901900204D1C010010B50A46037A23B198
:101FB00040F2D1211020FCF75BFD0146BDE8104046
:101FC000014807230BF073BAA81900201346027AC0
:101FD0000AB1037270470A46014601480BF067BA1E
:101FE000941900201B234FF01B1283840384826109
:101FF0008382C260038539B94FF4A473034AC38452
:102000004384C261C3820261704700BF4801480136
:102010000346F0B4B3F85420B3F84840B3F8446032
:10202000DF8FB3F84250944228BF14460846B3F8F5
:102030004C20B3F85610DC878A4228BF0A46B3F812
:102040004610A3F84220914238BF1146A64238BF3D
:102050002646A742A3F84460A3F846101FD1AA1A47
:1020600018BF0122B3F84A50B3F85040B3F8527089
:102070009E8FB3F84010A54228BF2546B3F84E40C6
:102080009D87BC4228BF3C46AE42A3F8404002D1E7
:10209000A14200D12AB1F0BC03490BF02EBA0122B3
:1020A000E0E7F0BC704700BF01D501000B8BA2F840
:1020B0000B304B8BA2F80D308B8BA2F80F30CB8BF3
:1020C000A2F809000249A2F8113010460BF00FBA2D
:1020D00051D50100094AD2E90003434083EAB01117
:1020E00081EA43214FEAF3435360054B11605843A3
:1020F0004FEAF06000EB8000704700BFD01900206D
:10210000BB79379E094AD2E90003434083EAB01104
:1021100081EA43214FEAF3435360054B1160584372
:102120004FEAF06000EB8000704700BFE004002041
:10213000BB79379E10B50A4C09480821FCF720FEF0
:10214000D4E900231343F7D0064CFFF7DBFF2060F0
:10215000FFF7D8FF236860600343F6D010BD00BFCF
:10216000E0040020D0190020174B184A9A60184A42
:102170005A60184A1A60184A9A62184ADA62184A6B
:10218000DA60184A9A61184A1A63184A1A62184A99
:10219000DA64184A9A64184A5A62184B184A9A60C4
:1021A000184A5A62184ADA62184A1A61184A5A6179
:1021B000184A9A61184A1A63184A9A64184ADA64E3
:1021C000184A9A63704700BF4005002019D80100E3
:1021D0004FD80100C7D801004FDA0100A3DA01008F
:1021E0002D250100B9DA01009D270100112601000B
:1021F00099DB0100B5DB0100692601002C060020F7
:102200003BD8010059DB0100DBDA01007FDA010075
:10221000FFDA0100B125010041DC0100EDDB010026
:10222000DBDB01003FDB0100044B054A5A65054B2F
:10223000054A1A65054A5A65704700BF40050020E7
:1022400087D901002C0600206DD90100F7D90100C3
:10225000054B064A9A65064A1A66064B064A9A656F
:10226000064ADA65704700BF40050020B5CB010083
:102270004BCC01002C060020F1CA010031CE010038
:10228000252A70B505460C4618D8012A19D9023AF4
:10229000232A16D8DFE802F01A1525242433153531
:1022A000152439444815154D242467676D74151598
:1022B000151515151515151515808990FF2A00F0AF
:1022C000828040F2FE315120FCF7D2FB0278436855
:1022D000012A02D193F8203101E093F829312371CA
:1022E00070BD4168204601F5EB710BF054F8696848
:1022F000204601F58A71BDE870400BF04EB8436886
:10230000E8E7BDE8704000F011BA0E230B715923C5
:102310004B7100238B716B23CB7110230B72DFE7A2
:10232000436893F81A31DAE7BDE87040084600F0D8
:10233000EBB90378466873B996F820315BB196F82B
:102340001D1120460BF07AF896F81C112046BDE8C6
:1023500070400BF077B896F81B1120460BF06EF822
:1023600096F81A11F2E741682046BDE870400BF07C
:1023700008BA436893F83621227193F8373109E09F
:10238000436893F83421012AF4D093F864200A7149
:1023900093F865306371A3E7104B1B68002B9FD047
:1023A00002462320BDE8704018470C4B1B68002BE9
:1023B00096D002462420F5E7084B1B68002B8FD0EF
:1023C00002462520EEE74368204693F84F22D3F8D3
:1023D0005012BDE870400AF078BF00BF1807002017
:1023E0003A289ABF024B53F820000020704700BFE4
:1023F000400500203A289ABF024B53F820000020E5
:10240000704700BF2C060020F7B545682E690446CA
:102410004FF6FF770DF102010DF101023046ADF8E4
:10242000027008F0D0FF01A9304608F0EFFF40B17C
:10243000019809F0B0F8616800220272FFF7B4FD5C
:10244000E8E7044905F1A80003B0BDE8F0400BF04F
:102450004EB800BFB3D70100F0B5044685B00D46B5
:10246000FF2600F8856C10F8863CF3B1174F3B78D7
:102470001BB148211F20FCF7FBFA0C21381DFCF78B
:102480007FFC3E70002304F8853C2A46072302F8AF
:10249000033BD4F80930C5F80330D4F80D3053604D
:1024A000D4F81130936005B0F0BD01A80C21FCF701
:1024B00067FCA4F5A873039A1A6001AB03CB44F838
:1024C0008E0C44F88A1C04F8866CDBE7D8190020CF
:1024D00010B5054C23782BB90C21201DFCF750FCBE
:1024E000FF23237010BD00BFD8190020024690F8CA
:1024F000DE31BBB990F8DF3103F0FF010BB10020F2
:102500007047094B18780028F9D01970D968C2F8BB
:102510001411043303CBC2F8D601C2F8DA11FF2339
:1025200082F8DE3101207047D819002038B54268A2
:1025300092F88F3004460D463BB1132B05D0113B6A
:102540000B2B94BF0820012038BD92F8D23013B96C
:1025500020460BF0D4F86168284601F5E7710AF0CF
:102560000FFF6168284601F588710AF010FF616865
:102570000B88A1F86D32284601F26F210AF0F8FEAF
:102580006168284601F277210AF0F7FE63680025AA
:1025900083F8DE516068054900F519700AF0A4FF60
:1025A0006368152283F88F202846CDE7592401005F
:1025B00038B5436893F88F201C2A044604D040F2B3
:1025C000BB111F20FCF754FA93F8D2101D8800228B
:1025D00083F8D12003F5D17069B10B4983F8D2207B
:1025E000A3F8AC5183F8AB210AF07EFF63680022A8
:1025F00083F88F2038BD012283F8AB11A3F8AC51CA
:10260000024983F8AE21EFE73BDA01002DDA010041
:10261000436830B5D3F8804014F001001FD14D68F5
:10262000104A8968A3F8CE002A40C3F8E220C2F31A
:10263000076242F0080221F41E5121F0100183F8D4
:10264000E52093F8D0200904090C013244F001047C
:10265000C3F8E61083F8D020C3F8804030BD0120D5
:10266000FCE700BF2FC904F710B5406890F88E3022
:10267000042B2FD14C688A68184B22F41E52234039
:10268000C0F8E23022F01002C3F3076343F00803FE
:102690001204120C80F8E5300023C0F8E62080F820
:1026A000CC3080F88E3090F8842102F0FF049AB983
:1026B0000388A0F8863180F885414B68C0F88831DE
:1026C0008B68C0F88C31064900F5BE700AF00CFF2B
:1026D000204610BD0124FBE71C46F9E72FC904F78B
:1026E0001DDB0100406890F8843153B90388A0F8DD
:1026F00086311A2380F88531024900F5BE700AF050
:10270000F3BE70471DDB010010B50446FEF73CFE2A
:1027100021F41E51044B21F0100109040340090C5F
:102720006360A16010BD00BF2FC904F737B50C4628
:102730004568FEF729FE0A4B95F8E22021F41E5168
:1027400021F01001034009040093090C13408DF897
:10275000003001916B4603CB6060A16003B030BDD7
:102760002FC904F7DB0410B5144604D5037D13B15B
:102770000023436310BD436B013343630BF043FA03
:10278000D0E90D239A42F5D3002343630249204642
:10279000BDE810400AF0B1BE8BDB010038B54468DB
:1027A00094F88E30012B0D4603D0D4F88030980772
:1027B00045D494F8D330990719D428460AF0F0FD8F
:1027C00084F8DD00B5F80530A4F8DE30B5F8073040
:1027D000A4F8E03094F8D33043F0020284F8D32018
:1027E000DA0711D5174904F1D4000AF086FE94F8EF
:1027F000D330DB0718D4D4F8803013F0020208D0AD
:1028000055214020FCF734F994F83A31002BE9D1F6
:10281000EDE743F00203C4F8803094F8D030A4F818
:10282000CE20013384F8D03094F88E30012B4FF055
:10283000000003D184F88E0084F8CC0038BD01205C
:10284000FCE700BF23DC010070B545680446FFF7D4
:102850002DF9054B85F88D001B6801461BB12046FC
:10286000BDE87040184770BD20070020024B1B6870
:1028700003B11847704700BF1C070020F0B5204D7A
:102880002B7800241470CBB3013B6F68DBB21D1BA7
:10289000012D0BDC07EBC40557F834606D688D42E1
:1028A00008BF864212D114700120F0BD1D196E10B0
:1028B00007EBC60E57F836C0DEF804608445C5F352
:1028C00047058E412CBF2B462C46E0E7B04271EB0A
:1028D000050502D214700020E7E707EBC30457F8A0
:1028E000335064688C4208BF854201D11370DBE726
:1028F000A842A14128BF01331370ECE71846D4E782
:10290000F819002010F0070208B503D06321482011
:10291000FCF7AEF818B1034B197258601A70C80072
:1029200008BD00BFF8190020014B00221A70704743
:10293000F8190020014B187A704700BFF8190020E1
:102940002DE9F7430BF0A7F90DF1070206460D46F6
:10295000FFF794FF98B910490A780B7A93420ED08A
:102960004C6813466FF060479DF80700984209D302
:1029700004EBC003C3E9006501320A70012003B013
:10298000BDE8F083D81904EBC000D0E90089013B11
:10299000C0E90289DBB2E7E7F819002037B50BF090
:1029A0007AF90DF10702FFF769FF0446A0B10C4A5E
:1029B0009DF8070013785568013BDBB213701A1AB3
:1029C000D2B2411CD200834238BF002205EBC101C4
:1029D00005EBC00006F06AFD204603B030BD00BF25
:1029E000F81900200A46822302F8033B04480368D2
:1029F000C1F803304368536083689360704700BF39
:102A0000011A002002481622002106F009BE00BF6C
:102A1000011A002082B002AB03E903000B48437D9A
:102A200093B1530610D50A880280D1F83022B1F84C
:102A300088304260D1F83422054982604380022206
:102A40000C3002B0FFF7C2BA02B07047011A002082
:102A5000E529010038B5074D044600F15101286809
:102A60000AF09DFB94F850102868BDE838400AF041
:102A7000A4BB00BF181A0020F8B504460E466588AE
:102A8000407F15F0040508BF2946134618BF04F11E
:102A90005F013246FEF7DEFEC20705460BD5012375
:102AA00084F85030607FFEF739FF0368C4F8513076
:102AB0008388A4F85530AB070CD5094E0127306840
:102AC00084F85E7004F15F010AF070FB30683946EB
:102AD0000AF07CFB85F00400C0F38000F8BD00BF65
:102AE000181A002038B5C38D0E4D0133C385AB7C59
:102AF00004462BB102F08EFC01F014FE0023AB74EF
:102B000000232B7194F879302BB101212046BDE8C8
:102B1000384009F0BFB9637C13B1E28D9A42F4D218
:102B20000021F3E7181A002010B5094C2379012B76
:102B300002D02379022B05D1A37C1BB102F06AFCE1
:102B400001F0F0FDE069BDE81040FFF7CBBF00BF2A
:102B5000181A002070B5294C2379012B07D023794E
:102B6000022B04D040F63C412D20FBF781FFA0B999
:102B70000125A37C1BB102F04DFC01F0D3FD002D1B
:102B80003AD0E06909F0FEF8002830D002F032FBBC
:102B9000236ABDE870409B6818472168E26911F814
:102BA000095B02F15103E80992F850200AF061F93B
:102BB0000028DDD0206800210AF02DFB0028D7D0A6
:102BC0002379E069012B05D02379022B02D040F64E
:102BD0001541C9E72379226A03F180435269013B19
:102BE00005F00F0152F8233098470546C1E7E06928
:102BF000BDE87040FFF776BF70BD00BF181A002017
:102C0000074A0346D06903B909B9FFF76BBF1379C7
:102C1000126A03F180431269033B52F823301847CC
:102C2000181A00202DE9F043032985B00546904687
:102C30007BD090F878300529DBB202D14288D007EA
:102C40005FD5002B5DD10127DFF8E89099F812607D
:102C5000B6B10AF043F9082888F8000014D002AA97
:102C60000DF10701FEF7CCFD20B940F685612D205E
:102C7000FBF7FEFE9DF8070002A90BF018F80646C8
:102C800098F80030082B08D1D9F8001011F8030B80
:102C9000C0F380100BF00BF80646D9F8001095F839
:102CA000572011F8030B05F15803C0F380100AF008
:102CB000E0F8D9F80010044611F8030BC0F38010B7
:102CC0000AF002F98146FEF73BFE40B1B9F1080F68
:102CD0001CD04846FEF760FD80F00100C0B298F8B5
:102CE0000020082A16D09CB96B7F991A4B424B41A1
:102CF0006A88520706D420B99EB9EB7C9BB1BB42CF
:102D000011D00023184605B0BDE8F0830020E6E7A7
:102D10000123EDE714B180F00104E4B204F00103F3
:102D2000E6E73346EEE70123ECE743889B07E8D567
:102D3000022789E7181A00202DE9F04F85B00823F3
:102D40000DF10702052104468DF80730FFF76AFFF1
:102D5000064620B90026304605B0BDE8F08F7A4F10
:102D60003968FA7C11F8030B07F11403C0F38010E3
:102D70000AF07FF880460028ECD13B68216A1846AB
:102D800091F8962010F8035B02EA551202F0010256
:102D900081F89620D3F80320C1F803208288A1F897
:102DA00007201946226A11F81F0BC0F3801090709B
:102DB00009798DF80C10D3F80F10D3F81F00D161EA
:102DC000597D0290187D090441EA0021D87C014315
:102DD0005162B3F8191040F2E24909FB01F1916127
:102DE0009D7DC5EB451105EB810505EB85056D0066
:102DF0009585B3F8171009FB01F19162B3F81B1028
:102E00001184B3F81D10518493F8243003F01F018E
:102E10005B0982F8A21082F8B031256A94F912B0E9
:102E200002A905F196000AF012F940F20113A5F883
:102E300068304FF0FF0A85F86AA0414605F130007E
:102E4000FFF7D0F859462846FEF714FE236A84F8A7
:102E500083801A88A4F8842084F8A1A04FF6FF721A
:102E6000A4F8A2209A69B2FBF9F2A4F89A201A8C6D
:102E7000A4F89C205A8CA4F89E2093F8B02184F8E2
:102E8000A020227F9DF8070004F18E015AB394F828
:102E90005020012A27D194F8562002F0C002402A7F
:102EA00021D1D4F85120C4F88E20B4F855208A805E
:102EB0009A7884F88720082803F1030504F1880232
:102EC000D3F8033004F1940134D0C4F89430AB88C3
:102ED0008B8004F18701FEF793FC40B940F69B31EB
:102EE0002D20FBF7C5FD0022C4F88E20DFE794F803
:102EF000873043F0020384F88730144904F17A00E4
:102F00000AF0F2FA236A12491A88A4F8BB2093F84F
:102F1000963084F8BD3004F1B2000AF0E5FA0D4BAA
:102F2000206A1B6800223A71002B3FF414AF21463F
:102F3000984710E7C4F88830AB8893800023C4F822
:102F400094308B80D9E700BF181A0020F1DC010013
:102F5000C3DC010028070020032973B5044604D010
:102F6000052952D0012002B070BD08230DF10702DF
:102F70008DF80730FFF756FE0028F3D0237C284D4C
:102F800003B39DF8070094F8C630DBB9237884F8C2
:102F9000C730082804F1C90228D004F1C801FEF79F
:102FA0002FFC20B940F6FB612D20FBF761FD94F862
:102FB000C83043F0020384F8C8301A4904F1BE0057
:102FC0000AF092FA2B68062204265A701E702046D8
:102FD000FFF740FD94F84020E16B28680AF00CF9F7
:102FE00028682E7102F0A6F90020BCE72868034685
:102FF00013F8031BC1F3801184F8C810D0F8031034
:10300000C4F8C9109B889380D7E7074B1B6823B18E
:10301000984780F00100C0B2A5E71846A3E700BFBB
:10302000181A0020D9DC010024070020F8B5044656
:103030000F4619B300F1280528460BF044F8A0B953
:1030400063881A072ED528460BF054F80646284602
:103050000BF039F8301AC0B20BF05CF8444A9368B0
:103060001844906028460BF00AF828460BF00CF83C
:1030700002F054F82179252001F04AFF3C4D94F8E4
:103080005E2028680023037043706388103B0D2B7B
:103090005ED8DFE803F0595D550C5D405D5D5D5D18
:1030A0005D5D5D402046BDE8F840FFF71BBD06238F
:1030B0004370202303702046FFF7CCFC638823F085
:1030C00008039BB2152B05D094F83820616B286853
:1030D0000AF083F8286802F02DF9032321792B7177
:1030E000002002F021F8064607B9E86063881B0754
:1030F00004D50BF00CF83044C4F8E0006388103BB2
:103100000D2B30D8DFE803F0322F29292F292F2F5C
:103110002F2F2F2F2F290C2343702123037042B10F
:1031200004F15F010AF042F8012128680AF04EF824
:10313000C1E704F158010AF039F894F85710F4E7A0
:10314000062303704370B6E7022303700623F9E7F2
:1031500040F226612D20FBF78BFC21790120BDE890
:10316000F84002F071B940F6AA41F3E7F8BD00BF9C
:10317000181A002038B54388102B044604D1BDE846
:1031800038400121FFF752BF0B4DAB7C23B101F05A
:10319000AFFA402002F032F9286802F0CBF86088DC
:1031A00010F0040002D1217902F04EF9002002F063
:1031B00001F901232B7138BD181A0020024B01219F
:1031C000D869FFF733BF00BF181A002010B5134CA1
:1031D000A37C1BB102F01EF901F0A4FAE06908F02B
:1031E000D1FD70B12379E069012B0FD12379226AD7
:1031F00003F18043D268013BBDE8104052F8233010
:103200001847E069BDE81040FFF76CBC2379022B3A
:10321000ECD040F643312D20FBF72AFC181A002091
:1032200010B50948037903F0FF0453B91822214669
:10323000043006F0F5F902F0EDF801F073FA2046DB
:1032400010BD0C24FBE700BF181A002010B5094C74
:10325000002323712060FFF7E3FF20B140F2F62145
:103260002D20FBF705FC236A13B940F2F921F7E79B
:1032700010BD00BF181A0020014B024A1A627047A5
:10328000181A002068350100034B044A1A60044BE9
:10329000044A1A60704700BF24070020392D01003E
:1032A00028070020DD0901002DE9F041067DB31E4D
:1032B000DBB2012B04468CBF4FF000084FF0010831
:1032C0007EB3B71E18BF0127012B36D800F1580175
:1032D00090F8570009F0F8FD082805462DD0FEF7B4
:1032E00067FA58BB657784F81C8084F85070FEF745
:1032F00081FA05460BF00EFA174BA5FB033518189B
:1033000045EB01050022C4E9120584F85E20114650
:103310002046FFF7B1FB70B940F293412D20FBF737
:10332000A7FB3746082504F151010020FEF726F9D6
:103330000028D7D10020BDE8F0810825022EF2D068
:10334000E37E002BF6D0D4F81530C4F85130B4F831
:103350001930A4F85530C5E740420F00F0B5464E8D
:10336000327987B0044602F0FF0312B90278FF2ACF
:1033700004D140F6A9112D20FBF77AFB3382B3600C
:103380007371B37180F879303C4B02933C4B0393DB
:103390003C4B0493336A02A85B68059301F0C2FFBB
:1033A00001F0F4FD02F036F801F0BCF9364801F006
:1033B0008FFE364801F0B0FF04F1280001900AF0BA
:1033C0005EFE01980AF060FE01F0A8FE217925203A
:1033D00001F09EFD94F9120001F074FE04F1340135
:1033E000206B08F0D3F904F13C010746206B08F08C
:1033F000F2F9054617B194F82430C3B90DB194F829
:103400002550237F13B963885B0709D5D4E91212CD
:103410006FF000439A4208BFB1F1FF3F09D185B96F
:1034200030680330FEF704FAB07407B0F0BD012530
:10343000E7E70BF06FF9D4E91223904271EB030335
:10344000EDD3012205EA02012046FFF715FB68B122
:10345000FEF7D0F905460BF05DF90D4AA5FB0232E7
:10346000181842EB0102C4E91202D9E7002DD7D0A7
:1034700040F6DE117FE700BF181A0020CD310100B1
:10348000552B0100012C0100D6BE898E55555500E3
:1034900040420F00F7B50446FFF760FF00212046C9
:1034A000FFF7C4FD04F1680009F0D9FC236F0BB1EC
:1034B00001221A606388DB0721D50023114E256A9B
:1034C000CDE90033FF23F37405F10A076846FBF7E3
:1034D00015FFA0B9009CA542F8D06A7A607A3B46F5
:1034E00004F10A0109F0C5FC0028EFD0A378F374B9
:1034F000D4F803007061044BB4F807209A8003B03D
:10350000F0BD00BF181A00202C1A0020024BD86111
:103510001B6A1B68184700BF181A002043881B0746
:1035200010B5044611D5036A0A493C2280F883206D
:103530001B88A0F88430FF2380F8A1304FF6FF737A
:10354000A0F8A2307A3009F0CFFFFF2384F8793059
:1035500010BD00BFF1DC0100592F010075310100E1
:1035600049DD010043DD010095340100292B0100F4
:10357000BD310100643501005C35010058350100A2
:103580000138022808B503D9C3212F20FBF770FAB0
:1035900013290A4B05D811290CD8102907D0D1219D
:1035A000F3E71529FBD103EB4003D88801E033F89A
:1035B000100008BD03EB40039889FAE72C6C040067
:1035C000F8B52F4B1A88402842EA00021A8005D12C
:1035D00004219868BDE8F840FDF72EB9802801D194
:1035E0000521F6E700F00302032A04D140F6CA11D0
:1035F0003120FBF73DFA10F0020418BFD960C5076F
:1036000005D5CA781961062A0DD00B2A18D02CB11D
:10361000DA68D278052A1FD00B2A2AD0820644BF46
:1036200008221A75F8BD9A6892F88F101829EED101
:10363000002600270121C2E93C6782F89310E6E7E3
:103640009A6892F88F10122901BF002182F8931016
:10365000012182F8D210DAE79A6892F88F101629C1
:10366000DCD100240025C2E93E45012182F89410F6
:10367000D4E79A6892F88F101129CFD10021F5E78D
:103680003C1A002013B5044601A8FDF701FF20B93C
:1036900040F2CA713120FBF7EBF922220021019898
:1036A00005F0BEFF0198032109F003FE019803789D
:1036B00023F0100303702146FEF754FA01990648DF
:1036C0002246FEF7DDFDFDF7F7FE10B940F2D4719A
:1036D000E0E702B010BD00BF401A002070B5274CD3
:1036E000A36893F8566293F85752002E3FD193F88F
:1036F0006810002D3DD193F8692083F8681083F895
:103700006920FF2283F86A201D4B1B680BB1A0685B
:103710009847A36893F83431012B02D056EA050389
:1037200003D018480021FDF757FEA068303009F09B
:103730005DFF0546A06800F24511FEF769FCA06830
:103740000621FDF779F8A068303009F04FFF854277
:10375000044610D202F060FF0146601B322838BFD9
:10376000322004F0CFFFB0FA80F0400970BD31463E
:10377000BFE72A46C1E70120F8E700BF3C1A002056
:1037800030070020401A0020002908BF1F211728F9
:1037900010B503460BD80D280DD90E3809280AD8C4
:1037A000DFE800F00B0909090B090B09110BA0F167
:1037B0002303022B23D9002010BDBDE810400021B7
:1037C00018460AF0ABBC114CA36893F88E20212A4E
:1037D00009D1201DFDF700FEA368002283F88E208A
:1037E00083F8CC20E7E72E2AE5D193F88F30A3F1B8
:1037F0002002062AF0D92E2BEED02A21E9E7044B2D
:103800001B68002BD7D0BDE8104018473C1A002099
:103810002C070020114B09790246986890F88E30E9
:10382000212B11D02E2B0FD0282B0FD0042B0FD0F3
:103830000F2B0FD01D2B0FD090F88F30232B14BFE0
:10384000FE201720FFF7A0BF1620FBE72320F9E793
:103850000E20F7E71220F5E71420F3E73C1A0020CA
:1038600008B50C4B9B6893F81E21FE2A04D040F249
:10387000D9713120FBF7FCF883F81E0111B9A3F8C8
:10388000CE1008BD0022A3F8C820012283F8CC2066
:10389000F7E700BF3C1A00200D4B1A7D9AB940B9DA
:1038A0009B68B3F858109A8F91420FD81846FCF7CE
:1038B000B5BF1A88120708D59B6893F8900007389F
:1038C00018BF01207047002070470120704700BFDB
:1038D0003C1A002070B54368D3F8803013F0300FE5
:1038E00086B004460D4655D1084609F073FD30B93F
:1038F0002946204606B0BDE8704009F02EBF284694
:10390000666809F063FD0590284609F05BFD0490A8
:10391000284609F05DFD0390284609F055FD303634
:10392000DDE9033200900599304609F071FE1A4B2B
:103930001A88920710D5DA68D278142A0CD16268F6
:10394000D2F8803043F01003C2F88030204609F0EE
:10395000D6FE002006B070BD626892F88E101D2958
:10396000EDD092F82B21002AE9D1626892F82A2141
:10397000002AE4D16168D1F8802042F02002C1F829
:1039800080209A68114602F5A77231F8300BFEF7D5
:103990008DFBDBE70120DDE73C1A002010B5164B5C
:1039A000DB681979436893F88E20092A09D193F8C6
:1039B00019218A4205D1002283F88E2083F8CC2079
:1039C00010BDD3F8802012F0080407D022F00802BE
:1039D000BDE81040C3F8802009F09BBEFF2905D147
:1039E000332283F88E2083F84C42E9E740F2DE412F
:1039F0003120FBF73DF800BF3C1A002010B50B79D1
:103A00004268172B92F88E2004460CD80D2B0CD947
:103A1000A3F10E01092908D8DFE801F0090707071B
:103A2000090709071009232B26D0002010BD2246C4
:103A30000121BDE8104018460AF070BB212A01D0D0
:103A40002E2AF2D1204609F051FE636893F88F20A8
:103A5000222AEAD093F8E32022F0010283F8E3203F
:103A6000626892F8E33023F0080382F8E3301A2109
:103A70002046FDF7B1FCD8E7282AD6D1024B1B68B7
:103A8000002BD2D09847D0E7340700207FB5844C74
:103A90000546002840F0B88023881B0735D5A36869
:103AA00093F81E21FE2A04D14FF4AA613120FAF7BF
:103AB000DFFFFE2283F81E2193F88F201A2A07D1F8
:103AC00083F8D100201D09F024FEA36883F88F50ED
:103AD000A36893F88E20332A42D03F2A49D0202A67
:103AE0000AD193F88F20A2F12001062901D92E2AAC
:103AF00034D12E2283F88E20A36893F89020072AD1
:103B000002BF0222627583F81E212388DE0734D4A7
:103B10002388580700F1A680990713D5E368DE785B
:103B20000D2E00F0A780112E00F0A680072E00F0C9
:103B3000A5803046FEF75EFC0346002800F0A0801A
:103B4000584898472388DA065ED5A36893F88F20F3
:103B50000A2A59D10B2283F88F2055E02122C9E788
:103B6000012283F84D22002283F88E2083F8CC2096
:103B7000C2E74C4809F0BAFDBEE7A368216993F893
:103B80008F30113B0B2B0CD8CB78023BDBB2092BCF
:103B900000F28280012202FA03F340F23332134230
:103BA0007AD008460191FDF7CBFF019918B93D483D
:103BB00009F0D3FD4BE0CE78012E01D9162E11D19C
:103BC000A368019193F88E0009F0B8FD019948B1FE
:103BD000A36893F88E20202A04D0212A10D12E2207
:103BE00083F88E20112E37D028D8072E36D00D2EF0
:103BF00036D030460191FEF7F3FB0199034621E0F0
:103C0000162E0CBF20250225237D1B0713D5A36884
:103C100093F88F30113B0B2B40D9002603A90320CA
:103C20000396FBF7D1FF039B2BB11E720C22A168F8
:103C30000398FEF787F9284604B070BD142ED8D13A
:103C4000194B1B68002BB2D02169164898470028F1
:103C50003FF45EAF0546D7E7144BF5E7144BF3E7A7
:103C6000144BF1E7A26892F89020062A04BF0122C3
:103C7000627551E7104B63E7104B61E7104B5FE74C
:103C8000FF2E06D1A268332182F88E1082F84C02F2
:103C900058E740F2445109E70825B5E70825CAE787
:103CA0003C1A0020401A00203C07002031E20100AD
:103CB000FD39010015380100C1E10100DFE101001B
:103CC0009D3901002DE9F041A54CB4F800800E4665
:103CD000A16818F4007F0ABFB1F8C22000230132A6
:103CE00001F1800507461ABFA1F8C23081F8C7313B
:103CF000A1F8C22028460AF08AFA28B1434601F505
:103D00009E722846FEF72EFD238803F4C06333B16C
:103D1000A06890F89230002B4AD0032B4ED0A168B7
:103D2000238891F89220012A04D11D0544BF022264
:103D300081F89220002F40F0AD8058065DBFB1F8A9
:103D4000E021013292B23A46A1F8E02103F00A02E2
:103D50000A2A0DD1E268D278022A09D123F0080399
:103D600030462380FFF792FE08233043C6B22380FB
:103D70003046FFF78BFEA36893F81E213043FE2ADE
:103D8000C6B24FD1002E4DD193F89020063A012AA9
:103D900048D993F82831B3B1A36893F82921A3F83F
:103DA000C66083F8202101210220FFF759FD39E088
:103DB000012180F89210FCF73FFDB0E7022380F864
:103DC00092300121F7E7A06890F88F30A3F1100539
:103DD000EDB20C2D11D8113B0B2B00F25681DFE810
:103DE00013F00C015401540154010F011701540147
:103DF00054015401540154014201D0F88030D907D4
:103E000002D531460920D0E79A0740F19A80314621
:103E10000C20FFF725FDA26892F8D33043F0010390
:103E200082F8D330A568B5F8C03195F8C481013364
:103E3000A5F8C031B8F1000F00F0E581FBF7B6FE40
:103E400010B10023A5F8C031A16891F89280B8F1B3
:103E5000010F40F20E8291F89030072B40F0EB8179
:103E6000B1F8C230022B40F20482B1F8C4500135DF
:103E7000ADB2B1F888302B44A1F8B83191F8C53112
:103E8000002B00F0FF810123A268B2F888100B44D8
:103E9000A2F8BC312288A36855065BBFB3F8CC21D9
:103EA000B3F8BE1100225218A3F8CC2193F82831A0
:103EB0002BB9A36893F89030063B012B07D8A36871
:103EC000B3F8C620B3F8BE110A44A3F8C620A3680D
:103ED00093F8CC0030B1B3F8C820B3F8BE110A444F
:103EE000A3F8C82093F9D0100029C1BFB3F8CE20A1
:103EF000B3F8BE515219A3F8CE2093F8B1205AB9A5
:103F0000002F40F05982627D022A40F00E8293F821
:103F10002021062A18BF1622A36893F8B0302BB9C7
:103F2000A368104883F8B120FEF76EFAA0680AF083
:103F3000BFF9A368002283F8C321BDE8F041FDF773
:103F4000E1BA590702D5314613202EE71A070BD5DF
:103F500090F8183180F820313146072025E700BF5E
:103F60003C1A0020401A002013F0300F3FD090F888
:103F70002B31002B40F02682A36893F82A31F3B14D
:103F8000A06890F88F30252B00F5957100F256222D
:103F90002BD090F88E30A3F1250CDCF1000343EB1D
:103FA0000C0309F027FBA268D2F8803023F020032D
:103FB00043F01003C2F88030002382F82A31A06851
:103FC000D0F88030DA0640F1FD8100F24511FEF7AD
:103FD0001FF8A368B3F85220A3F82021B3F85620A5
:103FE000A3F8222100211520DFE60123D9E75B0693
:103FF00040F1E88100212420D7E600210B20D4E6FF
:10400000FEF774FA00283FF40DAF00210420CCE63F
:1040100090F84832012B08D100210520FFF720FC41
:10402000A368002283F84822FCE6A36893F848328C
:10403000022BD8B27FF4F6AEA36893F8D2500622D2
:104040001DB183F820210021E8E78C48032109F005
:104050006FFBA36893F8E23013F0040F294614BFF6
:1040600011200D20DAE7002106209EE693F8342186
:10407000022A02D10021172097E693F83421012A61
:1040800003D193F83531002BF4D0A36893F88E2038
:104090006AB993F88F20103A0C2A40F2A38193F862
:1040A000C020002A00F09E81012112207DE6092A0D
:1040B00040F0948193F8192183F8202101214CE7E5
:1040C000A36893F83A319BB1A36893F8D33013F007
:1040D00003050DD101210C20FFF7C2FBA36893F863
:1040E000D32042F0010283F8D32083F83A519BE7B2
:1040F000A36893F82A3153B3A36893F82B3133BBE9
:10410000A06890F88F30252B00F5957100F25622AB
:104110001BD090F88E30A3F1250CDCF1000343EBAB
:104120000C0309F067FAA368002283F82A21012111
:104130001420FFF795FBA368B3F85220A3F82021C1
:10414000B3F85620A3F822216CE60123E9E7A3681F
:1041500093F83421012A4CD193F83531002B48D102
:10416000A16891F88F30A3F12002062A41D92E2BA5
:104170003FD091F86850012D06D0022D04D040F2B6
:1041800017310620FAF774FC91F86900012801D074
:104190000228F4D1022D91F836210AD0012A14BF49
:1041A000002201223AB90A3B042B12D90121162020
:1041B000FBE5022AF3E7022891F8372117D0012AFC
:1041C00014BF00220122002AEDD02C480021FDF767
:1041D00003F9A36893F88E20002A7FF423AE93F8A6
:1041E0004C32002B3FF41EAE0121FF20DDE5022AF8
:1041F000E6E7234B1B68002BEBD020489847FE28AE
:10420000E7D00121D1E5FBF7CBFC08B1A5F8C081CF
:10421000FBF7D4FC00283FF417AE95F8C731013303
:10422000DBB2022B85F8C73182BF0023A5F8C0316D
:1042300085F8C73108E691F8C0301BB191F88E308F
:104240000F2B16D1B1F8C450B1F8C23001F1800083
:10425000ED1A033D09F0DBFF68B1D1F8B830D1F8B1
:10426000B420033B9B1A9D42A8BF1D46012D3FF77A
:10427000FFAD0125FDE52B46F5E700BF401A002004
:1042800038070020012D7FF6FEAD91F88F3013B175
:104290000B2B7FF4F8AD91F88E30002B7FF4F3AD4B
:1042A00091F89030002B7FF4EEADB8F1020F7FF45F
:1042B000EAAD91F8C731002B7FF4E5AD086907F04E
:1042C000E6F800283FF4DFADA26892F81E31FE2B1D
:1042D0007FF4D9ADB2F8BA31012B7FF6D4ADB2F884
:1042E000C011138C9942BFF4CEAD5B1A013DADB243
:1042F0009BB29D4228BF1D466B1C9BB292F8772053
:1043000072B9A1680A6F5AB1B1F8BE20B1F888102D
:10431000521A91B212B2002A02DD9342A8BF0B4694
:10432000A268012182F8C211AEE5012A09D193F8F1
:104330009120002A7FF4F0ADA0680021FCF77CFA00
:10434000F7E55EB1F00635D4310735D4B20635D481
:10435000B30735D140F64C11312013E738B1B3F82B
:10436000C800B3F8CA20904201D32222D4E5002924
:1043700005DDB3F8CE10B3F8CA209142F5D2B3F8F8
:10438000C610B3F8C42091420BD2A36893F89210E0
:10439000B3F8C22051B1B3F8C4309342CCD808224C
:1043A000BAE593F82831002BDFD1EEE7052AC3D90F
:1043B0003E22B1E51E22AFE53D22ADE52322ABE56D
:1043C0002A22A9E5A36893F88F20222A3FF44EAE53
:1043D000312A7FF45AAE00211120E6E40C2D3FF67D
:1043E000F8AE1FE50C2D7FF61DAD93F83B31002B89
:1043F0003FF466AE01210E20FFF732FAA3680022D7
:1044000083F83B2110E600BF73B5664D00240126FA
:104410002E71A8602C802C756C75FF2380F8C33139
:10442000AB681888FDF72EF8AB681888FDF754F8CC
:10443000AB68B3F8BA21EAB193F81E21FE2A19D16C
:1044400093F82831B3B1AB6893F89020063AB242A2
:1044500010D993F82921A3F8C64083F8202102201F
:104460003146FFF7FDF9AB68022083F8C241FFF740
:1044700009F904E0AB6893F81E01FE28F7D1AC6897
:10448000B4F8BE31B4F8C021013B12FA83F2A4F8AB
:10449000C021B4F8C22099B212FA83F3A4F8C23052
:1044A00004F1800009F0B3FE20B1D4F8B4300B441D
:1044B000C4F8B430B4F8BA31012B9CBF0133A4F86E
:1044C000BA31002609B184F8C76194F88F3084F8B6
:1044D000C261A3F10A02012A1FD8B4F88830B4F8E7
:1044E00054229B1A190432D404F2562104F1960086
:1044F00008F0ADFDAB6883F88F60FF2283F8EA20F7
:10450000A968B1F8BE2101F1800008F0E6FDA0B372
:1045100040F6D7013120FAF7ABFA252B17D1B4F8C2
:104520005422B4F888309B1A1A0410D484F88F608F
:10453000FFF7D4F8AB68014630B983F8340102B014
:10454000BDE87040FFF7BEBB83F83461D8E794F84C
:104550008E3003F0FD03252BD2D1B4F88830B4F8A7
:1045600054229B1A1B04CBD4002384F88E30FFF70F
:10457000B5F801460028C3D1E1E70B4B0B49009386
:1045800003C90B4B0B4AFBF7DDF9AB6893F88F308F
:10459000113B0B2B04D802B0BDE87040FBF7CAB941
:1045A00002B070BD3C1A0020C53C0100401A00203A
:1045B00099380100C135010038B50446084694F821
:1045C000483213B10C25284638BD94F88F30153B7E
:1045D000012BF7D894F86C3203F0FF05002BF1D1D2
:1045E000A1B194F8DE3123B940F6A1113120FAF7D8
:1045F0003FFA074B9968052301F5807201F5E771D1
:1046000004F03CFD012384F84832DCE70223FAE79A
:104610003C1A0020D0F85C328269934210B50446FF
:1046200004D1D0F86012026A914215D02288A4F811
:104630009A2140F2E242B3FBF2F3A4F89C31B4F8C1
:104640006032A4F89E31B4F862320949A4F8A0316E
:1046500004F5C87008F051FF02212046FDF7A8F9C3
:10466000002384F88F30032384F8923010BD00BFFC
:10467000A7D8010008B5FDF7D7FD024B024A1A6022
:1046800008BD00BF3C070020D5380100064BD3F819
:10469000000138B1D3F8040120B1D3F80801B0FA11
:1046A00080F04009704700BF00F00040034B00223B
:1046B0001A705A7010229A70704700BF541A002066
:1046C00070B50646022014460D4600F09FF9064BD1
:1046D00001221A70054B033CC3F81045C3F8086566
:1046E000C3F8045570BD00BF541A002000F000400C
:1046F00008B5022000F08AF9084B01221A70084B15
:104700000022C3F80021C3F80421C3F8082103F5EF
:1047100080334FF40002C3F8042508BD541A00206A
:1047200000F000400D4A08B513787BB10C4B4FF4F4
:104730000001C3F80815FFF7A9FF60B1012353700A
:10474000084BD3F80034937000231370BDE8084081
:10475000002000F05BB950701023F4E7541A0020D9
:1047600000F0014000F000400A4B1A786AB10A4B91
:10477000D3F800215AB1D3F8040120B1D3F80801CD
:10478000B0FA80F04009C0B27047587870470220F4
:10479000704700BF541A002000F0004008B5074BD6
:1047A0001A783AB1FFF772FF30B1054BD3F8000425
:1047B000C0B208BD9878FCE71020FAE7541A002030
:1047C00000F00040024B00221A705A709A70704735
:1047D000571A00202DE9F04104461C4D01201E46C9
:1047E0008846174600F012F904F003002E7140EAE3
:1047F0000643174E43F08073C6F80435C6F80885A3
:1048000004F028FD30B9D6F8183523F0FF033B43F8
:10481000C6F818350F4B104AC3F8082514F0FB0FE3
:1048200001BF0E4AC3F89825FC3AC3F89C25012223
:10483000022C6A70EC7007D8054B2A700021C3F86F
:104840000011C3F800121A60BDE8F081571A002069
:1048500000F0004000F001400000020200F10040C2
:10486000214A537870B523B94FF404713C20FAF70C
:10487000FFF81E4BC3F80C15C3F81005D5780124BA
:104880009470C5B912780AB9E121EFE7184AC3F864
:1048900004514FF40035C2F80455D3F8006116B145
:1048A0005C60C2F808550B7803704B780433437092
:1048B0008B78837070BD042D4FF0000106D1147009
:1048C000C3F80411C3F800421C60F3E7127812B970
:1048D00040F20D11CAE7C3F80411054B4FF0007206
:1048E000C3F80425E6E700BF571A002000F0004097
:1048F00000F00140084B1A784AB10849084AC1F84B
:1049000008250022C1F89825C1F89C251A700022BC
:104910005A709A70704700BF571A002000F001408B
:104920000000020208B50A4B1B7823B940F2762139
:104930003C20FAF79DF8074BD3F8042112B940F256
:104940007721F5E7D3F80004003818BF012008BD2F
:10495000571A002000F00040164B1B7870B523B9A1
:1049600040F287213C20FAF783F8134CD4F8043145
:10497000BBB90223C4F80433104B114E1D691A69E8
:1049800042F0100205F010051A61D4F804314BB161
:1049900025B90A4A136923F0100313610223C4F8EE
:1049A000083370BD4FF40043C6F8803109F0E0FED3
:1049B000EBE700BF571A002000F0004000ED00E0D8
:1049C00000E100E0014B01229A60704700F00040D6
:1049D00008B50B4B4FF40042C3F88020BFF34F8F54
:1049E000BFF36F8F074B0022C3F80025C3F80025E3
:1049F000FFF780FF044B4FF40002C3F8082508BD01
:104A000000E100E000F0004000F0014038B5144C37
:104A10000023C4F80035C4F800350546FFF76AFFE7
:104A2000104B4FF40002012DC3F8082503D0022DCE
:104A300008D085B938BD0223C4F800350A4BC4F844
:104A40001435F7E70321C4F800150749C4F8141515
:104A5000C3F80425EEE782213D20FAF709F800BFEC
:104A600000F0004000F001405C1A0020024B0022E0
:104A70001A809A701A717047681B002038B5144D5F
:104A800095F841200346084622B940F64F013E20E2
:104A9000F9F7EEFF6BB9012AEC6B95F8401005D1E0
:104AA00000F05CFE2044AB6AC01A38BD09F02CFC53
:104AB000F8E7012B0AD1012AEC6B95F8401002D1DE
:104AC00000F03EFEEEE709F02AFCEBE70020EAE703
:104AD000681B002008B5094B012883F82000084B0B
:104AE00006D0022808D040F675513E20F9F7C0FFE5
:104AF0000322C3F8102508BD0422FAE7681B002032
:104B00000010004008B5144B93F84D30D90721D55B
:104B10009A0711D5114BD3F8002242F00102C3F8D5
:104B20000022D3F8503503F0F603022B12D140F2E5
:104B30000D613E20F9F79CFF5B070BD5084B094A36
:104B4000C3F8AC25A3F5B833D3F8403113B140F224
:104B50001461EEE708BD00BF681B00200010004094
:104B600000F001400810004007B50B4A01AB92F974
:104B7000212000F037FE9DF9040000F0D9FD9DF8DA
:104B8000050000F0A3FE20B140F2DE513E20F9F70F
:104B90006FFF03B05DF804FB681B002008B50346F7
:104BA0000F4863B92831C1600E4900F077FE01302B
:104BB000012814D940F235713E20F9F759FF012B35
:104BC0000AD12931C160074900F06EFE0130012889
:104BD00005D940F23F71EFE740F24371ECE708BDC1
:104BE000E80400204C6C040008B50C4B9B78012BAA
:104BF00009D100F05FFE013001280ED94FF40A619F
:104C00003E20F9F735FF022B07D100F059FE0130A5
:104C1000012802D940F6A601F2E708BD681B002072
:104C2000044B03441A7E044BC3F80825C3F854050B
